:1000000000400020458000008580000087800000BF
:1000100000000000000000000000000000000000E0
:1000200000000000000000000000000089800000C7
:1000300000000000000000008B8000008D800000A8
:100040008F800000195B0000F18300008F800000AA
:100050008F800000000000008F8000008F80000073
:10006000A1390000C58700008F8000008F8000004C
:100070008F8000008F8000008F8000008F80000044
:100080008F800000758400008F8000008F8000004A
:100090008F8000008F8000008F8000008F80000024
:1000A0008F8000008F800000000000000000000032
:1000B0000000000000000000000000000000000040
:1000C00010B5064C2378002B07D1054B002B02D02E
:1000D000044800E000BF0123237010BD700200201F
:1000E0000000000094F50000044B10B5002B03D075
:1000F0000349044800E000BF10BDC04600000000F6
:100100007402002094F50000164B002B00D1144B14
:100110009D46402292029A1A924600218B460F4633
:100120001348144A121A0CF081F90F4B002B00D01F
:1001300098470E4B002B00D0984700200021040068
:100140000D000D48002802D00C4800E000BF0CF064
:100150002DF92000290008F09DF90CF001F9C046A6
:100160000000080000400020000000000000000027
:1001700070020020CC2F00200000000000000000D2
:1001800002000120104011D1042A0ED91368180969
:1001900080B2002809D001388000031D11180979A8
:1001A000002902D001309842F8D170470020FCE7C6
:1001B0000378002B03D05AB2002A01DB01307047CC
:1001C0003F229343C03B59424B41C01803789343AD
:1001D000802BF4D10130F9E710B500240378002B0F
:1001E00001D1200010BDFFF7E3FF0134F6E770B541
:1001F000002204000D00411C092003F0F9FE002834
:1002000006D001236200134343600023A34200DBB6
:1002100070BD9A00A958821891600133F6E770B555
:10022000012803DC1C2001F06DFA70BD01230D686C
:1002300011201D42F7D04868184206D1042804D97D
:100240000F2302681340042B01D00E20EBE703F0CC
:100250002DFD6D100400002D03DDFFF7BDFFA8424A
:1002600006DA1220DFE72000FFF7A2FF0400013DBD
:10027000012DF8D120787F2809DDDF280BDCF82359
:100280003F22DB00800118406378134018430123AC
:1002900040001843C9E7EF280BDCFC226378120109
:1002A0009B0113403F220007000C0343A07810403D
:1002B000ECE7F72812DCFC22637892021B03134060
:1002C000E0228004520310403F221843E378134099
:1002D000FC220343A07812018001E8E7012040429C
:1002E000D5E7F8B54D680F00EB0706D4042D04D907
:1002F0000F232E683340092B03D00B2001F002FAA4
:10030000F8BD6B683609B6B25C10731EA3420FD8F5
:100310000321200009F046FF6421642803DC01006A
:10032000032800DA03212800891903F093FE050051
:100330002B6800201B099BB2013B9C42E0D23A682B
:10034000A31C9B005A510123013464001C436C60C0
:10035000D6E7F0B585B0012803DC1C2001F0D2F906
:1003600012E001274B683A000093022806D08B6800
:100370003B4203D05F10002F00DC17000125009BDB
:100380002B4203D00120404205B0F0BD009B042B5E
:10039000F8D91B680C680F261900314004292DD1AB
:1003A0002C4205D1042C03D923681E40042E01D011
:1003B0000E20D3E70098FFF7E3FEB842E2DB009897
:1003C00003F074FC0600200003F070FC03780100C9
:1003D000002BD7D0781E30180CF0DEFB041ED1D0D5
:1003E0003378002B01D0A64202D36800012521E01A
:1003F0003000FFF7DDFE01350600F1E709293ED1A7
:10040000009B5B685B1001939F42BBDC2C422ED1AA
:10041000042C2CD923683340042B28D1200003F06E
:1004200045FC039602907E1C009AB300D05884428B
:1004300002D178002843A7E728420ED104280CD91E
:100440000368039A1340042B07D103F02FFC01002B
:1004500002980CF06BFB0028EBD0019B37009E420A
:10046000E1DD8FE71F00019B9F4200DD8AE77B1CD7
:1004700000999A008A58A242F4D17800B6E703297D
:1004800000D07FE71A0992B25B0F92000B40D31A9B
:1004900001939F4200DD75E72C4229D1042C27D916
:1004A00022681640032E19D1100980B2520F800025
:1004B0003240251D801A019B2E181B1A0193009BA8
:1004C000781E0433019A904200DD5BE72A00191878
:1004D000B2420FD316D10130400087E7042E07D176
:1004E000200003F0E3FB05002000FFF749FEE2E7F0
:1004F0000F2033E70C78A4461478A44502D10131CB
:100500000132E5E70130DDE7F0B50D0085B00128E7
:1005100004DC1C2001F0F6F805B0F0BD01270868E6
:10052000384206D1042804D90F2102680A40042A5F
:1005300001D00E20EEE76A681740FAD1042AF8D9F4
:1005400013680B40042BF4D103F0B0FB040068687F
:1005500003F0ACFB02900CF0F3FA039000280FD1EB
:100560002000FFF739FE0190019B0122591C092050
:1005700003F03EFD364E3060002815D10020CBE759
:10058000029920000CF008FB001B4342434120006D
:100590000193019B5E1C0028E6D0039B0299C018C2
:1005A0000CF0FAFA0196F4E70122019B5B00134379
:1005B0004360039B002B18D12000FFF7F9FD019B3E
:1005C0000500BB4201DC3068A6E7291B200003F0D0
:1005D0008DFD0028D2D0BB1C32689B0098502800AB
:1005E000FFF7E6FD01372C00E9E7019B012B02D163
:1005F0002B68836090E7029920000CF0CDFA01256A
:100600000700019B002F13D0AB42DCDB391B20001D
:1006100003F06CFD0028B1D032680135AB00985072
:10062000039B0299FC1820000CF0B6FA0700E8E7DB
:10063000AB42C8DB20000CF083FA0100200003F07D
:1006400055FD00289AD001353368AD00E850BAE76F
:10065000E40F002010B503F00DFB43000120184308
:1006600010BD0000C30711D404280FD90F2302685E
:100670001340032B0AD119400133591AC0234907EB
:10068000DB051940024B1A40114301607047C04618
:10069000FFFFFF9F70B5002805DC1C2001F032F839
:1006A0000500280070BD01220C68144201D10D2004
:1006B000F4E701281CD04B681342F8D05B101320DC
:1006C000FF2BEBD81A0619040A431A431B021343E3
:1006D0006410E243D2171440E11C89101A00032071
:1006E00003F086FC051EDCD02100FFF7BBFFD8E736
:1006F0000023EDE7F7B507000E001C20012F06DDF3
:100700004C68012322001A40009203D10D2000F012
:10071000F9FF53E0022F02D08A681A42F6D0012373
:1007200035681D4200D0A9E0042D00D8A6E01C4188
:10073000002C00DC1C000F2029680840092828D163
:100740006B685B100093022F05D0B368009A5B10B2
:100750009A4200DD0093009B01221D1B0135EB43F3
:10076000DB171D40691C092003F042FC071E09D05D
:1007700001236D001D430300326808334560009972
:10078000A14201DA3800FEBD0134A100515802C374
:10079000F5E7042845D1280003F088FAFFF71CFD8F
:1007A0000190022F04D0B3685B10984200DD0193E2
:1007B000019BA34204DA002003F08CFC0700E1E770
:1007C000280003F073FA0700009BA34221DB2800F6
:1007D000009703F06BFA05003800FFF7E9FC019B76
:1007E00001340700A342F7DA009BC41A200003F08B
:1007F00071FC071EC6D003F059FA0190306803F06F
:1008000055FA2200009B591B411801980BF0F2FD8C
:10081000B8E73800FFF7CCFC009B070001330093DA
:10082000D2E703282AD10B099BB2490F9B00014054
:10083000591A022F04D0B2685210914200DD110003
:10084000A14205DA00220320110003F0D1FBB5E735
:1008500003200E1B331DD9170140C918891000222F
:1008600003F0C6FB071E00D18CE7013631000334CC
:10087000FFF7F8FE381D29193200C7E7212046E7A7
:10088000F7B5002804DC1C2000F03CFF040014E055
:100890000D6801272E003E4011D03D41FF2D01D9AA
:1008A0001320F1E700223900032003F0A1FB041E0E
:1008B00003D03900FFF7D6FE25712000FEBD042DC0
:1008C000EED90F232A681340042B1BD12800FFF711
:1008D00057FCC31C07000320D9170140C918891011
:1008E000320003F085FB041EE7D03900FFF7BAFEA3
:1008F000280003F0DBF9231D01003A0018000BF07B
:1009000079FDDAE7092B1FD103206B6832005B10F9
:1009100001930333D9170140C918891003F068FB0C
:10092000041ECAD00199FFF79DFE019B9E42C4DAC6
:10093000B300EB189B683B4204D05B10FF2BAFD891
:10094000A21913710136F0E7032BA9D12C00B4E7EB
:1009500010B57F2902DC0170013010BD1A4B99429D
:100960000CDC40238A115B42134303703F230B408E
:1009700080214942194341700230EEE7134B9942FE
:1009800010DC20230A135B4213433F2480220370B0
:100990008B1152422340214013430A43437082701B
:1009A0000330DAE70A4B9942D7DCF0230370603B4F
:1009B0004370113B8A11FF3B1A4382703F22114062
:1009C0001943C1700430C8E7FF070000FFFF0000B3
:1009D000FF0F0100F0B50D0085B0002803DC1C20DE
:1009E00000F090FE0DE009680122080010400AD0D6
:1009F00002AC11412000FFF7ABFF011B200003F008
:100A000075FB04001AE004293FD90F230C6823402A
:100A1000092B3AD14B685B10019303239C46019B41
:100A20009A420EDD03F056FB041E07D02E68012506
:100A300003F03CF92F00019B9D421DDD200005B015
:100A4000F0BD01329300CC580123234001D127206F
:100A5000C6E764107F2C0DDD0D4E0223B44209DD84
:100A60000C4E6346B44205DD00270B4EE30FA64251
:100A70007B419B00C018D2E70135AB00F1583942E9
:100A8000E5D04910FFF764FFD5E70B20A8E7C04683
:100A9000FF070000FFFF0000FF0F010010B5012459
:100AA000044002D04410200010BD042810D90F23A8
:100AB00002681340042B07D103F0F8F821000A2242
:100AC0000CF006F90400EEE7032B01D10430F5E742
:100AD0000D2000F017FEE6E710B5040001200840E5
:100AE00010D104290DD90F230A681340042B08D113
:100AF000080003F0DBF8010020000CF017F8434277
:100B0000584110BD0020FCE7F7B50E00012803DCBA
:100B10001C2000F0F7FDFEBD4D68EB0706D4042D48
:100B200004D90F222B681A40092A01D00B20F0E7C4
:100B30006A681B099BB25410A34200D85C1E0127AF
:100B400031680F404810002F35D12648FFF7C4FF09
:100B500001230190002813D131682348FFF7BCFF1F
:100B6000002811D0002C0DD00122631C013C9440C0
:100B70009B005A5114436C6004E00137BA00AB503B
:100B8000BC42FADA0020C6E701233068184223D1BC
:100B9000042821D902680E331340042B1CD1FFF71F
:100BA0007DFF002807D131681048FFF795FF002826
:100BB00012D01220ADE70028FBDD8442F9DB830070
:100BC000EB180433844209DC0123621C013C9C4085
:100BD000920053511C43CEE711209AE75A68013026
:100BE0001A60EEE7CFDA0000D3DA0000D8DA0000AE
:100BF000002310B50C000B70C30705D50D4942103A
:100C000020000BF057FF08E00B49002802D0042811
:100C100004D10A4920000BF06DFF10BD0428FCD957
:100C20000F2302681340042BF7D103F03FF8044967
:100C30000200E5E76CE60000DADA0000E0DA000026
:100C4000E5DA0000F0B593B0060002911C20012EF9
:100C50001DDD029B01251B681C002C4000D0ADE06F
:100C6000042B00D8E6E01A680F231A40092A4AD15B
:100C70000394039A029992008A5817002F4005D1D5
:100C8000042A03D910681840092806D0222000F051
:100C900039FD0190019813B0F0BD52685210A418AC
:100CA000039A013203929642E3D1611C012203F0C0
:100CB0009FF90190002802D100230193EAE7019BEC
:100CC0006400190025435D600831029ABB00D058CA
:100CD00002684368120992B25B109A4200D8531E10
:100CE0000022934209DCDA43D21713409B00C91853
:100CF000039B01379F42E8DBCCE794000519AD6800
:100D000001320D51EDE72700032A59D10193029AD0
:100D1000BB00D3582B42B9D1042BB7D9186801991D
:100D20000140032939D1020992B2430F92000B40CE
:100D3000D31A1C190137BE42E9D10320E31CD9178D
:100D40000140C9188910002203F052F901900028CF
:100D5000B2D000252100FFF785FC019B1E1D029AE1
:100D6000AB00D45801231C421FD1042C1DD90F21E4
:100D700023681940032918D1180980B25B0F80003D
:100D80000B40C01A0023834213DBC343DB17184018
:100D900001353618BD42E2DB7CE7042900D075E757
:100DA0001800FFF7EDF92418C4E72000FFF7E8F971
:100DB000E8E7E2181279F2540133E4E700273C0037
:100DC0000F25029ABB00D3580122134234D1042BC1
:100DD00032D9186801002940042935D11800FFF7DD
:100DE000CFF924180137BE42EBD1200003F072F98D
:100DF0000190002800D15FE7029FB600BB19041DD7
:100E0000029301233D681D4229D1042D27D90F26C5
:100E10002B681E40042E37D12800FFF7B1F90600D9
:100E2000280002F043FF0100200032000BF0E2FA3C
:100E3000A41922E02700C3E7180005A9FFF7D8FE90
:100E400005A80BF07DFECCE7032900D01EE70209C0
:100E500092B2430F92000B40D31A1C19C2E705A9A6
:100E60002800FFF7C5FE05A80BF06AFE05A90500DE
:100E7000020020000BF0BEFA6419029B0437BB424B
:100E8000BFD10023237005E7032EF6D11A0992B2D1
:100E90005B0F92001E40961B291DC5E7F0B50D00A3
:100EA00097B0002806DC1C2000F02CFC070038005E
:100EB00017B0F0BD0C68012123000B40009306D150
:100EC000042C04D922680F331A40092A01D00B20C0
:100ED000EAE7626852100392002A03DC009803F0EC
:100EE000F9F8E3E7504A019201280BD068680842FC
:100EF00008D1042806D902681340042B02D102F05D
:100F0000D5FE019001980BF01BFE06000F27039BF6
:100F10000834013B05935E43039B02909B00E3185A
:100F2000049301232068184273D1042871D9016801
:100F30000B003B409C46042B03D1FFF721F9861997
:100F400009E0032B6CD162460B099BB2490F9B0051
:100F500011405A1A9619049B0434A342E1D130007F
:100F600003F0B8F8071EA2D02B680793029B002B52
:100F700003D0686802F09AFE0190380002F096FEF5
:100F80000400009B079A9B00D3189E68300002F073
:100F90008DFE0123334005000693002B01D1042E62
:100FA00004D809A93000FFF723FE09AD28000BF093
:100FB000C7FD069B0490002B0ED1042E0CD90F21E7
:100FC00033681940032907D11A0992B25B0F9200C6
:100FD0000B40D31A351D04932000049A29000BF00E
:100FE00009FA049BE418029B002B0AD0059B009A87
:100FF000934206DD2000029A01990BF0FBF9029B57
:10100000E418009B01330093009A039B9342B8D1EC
:101010004DE709A9FFF7ECFD09A80BF091FD8EE75C
:1010200002F044FEF9E7C04601E0000010B50122DD
:10103000002400280BDD0B681A40141E03D05C103E
:10104000E343DB171C400122904200D04A68611C38
:10105000092002F0CDFF002803D0012364001C43C7
:10106000446010BD0A6870B510000125284034D1D5
:10107000042A32D90F24136849681C40092C17D15F
:1010800054681B099BB22C41A34200D85C1E8442C9
:1010900005DC02200133984206DB00200FE08500CA
:1010A0005519A9600130F2E7840011510130F2E7CF
:1010B000032C12D1294203D1132000F023FB70BD71
:1010C0004910FF29F8D81B099BB204329B00D318A2
:1010D0009342E2D911700132FAE70B2000F012FBC3
:1010E000DBE700000123F7B500254E680C00334014
:1010F0000193AB420ED11D00042E0BD90F22336891
:101100001A40092A26D172681B099BB25510AB42BE
:1011100000D85D1E27687C10FB0746D439003D4887
:10112000FFF7DAFC002826D00BF060FC290009F05C
:101130001FF94C1C019B002B00D069E0042E67D9DD
:1011400032680F331340092B3BD10134A400A4595A
:101150002000FEBD042A04D13000FFF711F805007D
:10116000D8E7019D032AD5D11D09ADB25B0FAD00B3
:101170001340ED1ACEE739002748FFF7ADFC0028F1
:101180001DD1042F16D90F233A681340042B11D117
:101190003800FFF783FC041E07D139001F48FFF712
:1011A0009BFC002806D0122005E0002CFBDDA542A8
:1011B000C0DAF8E7112000F0A5FA0400C8E72C0017
:1011C000B8E7042B1CD1300002F070FD0500012CA3
:1011D0000EDCFEF7EDFF461B300002F07BFF041E25
:1011E000B6D002F063FD320029000BF003F9AFE73F
:1011F0002B78013C002BD6D02800FEF7D9FFE5E77D
:10120000032B05D13419E37801245B001C439FE7CD
:101210000B20D0E7C8DA0000D3DA0000D8DA0000EB
:10122000F7B54D680E002A0001210A402FD1042D88
:101230002DD90F242B68B7681C40092C14D169687C
:101240001B099BB24C100192A34200D85C1E31686E
:101250003448FFF741FC00282DD00F232A681340A3
:10126000092B1DD1012317E0032C10D10F4203D10C
:10127000132000F047FAFEBD7A100192FF2AF7D83A
:101280001A0992B25B0F92001C40141BDFE70B207F
:10129000EFE701339A00AF509C42FADA0020EAE708
:1012A000032BFBD12B0001335A1BA242F6DC6A460A
:1012B0001279DA70F7E736687010F30719D4310045
:1012C0001948FFF709FC002822D1042E1ED90F234C
:1012D00032681340042B19D13000FFF7DFFB0028E0
:1012E00007D131001148FFF7F7FB00280ED012207C
:1012F000BFE70028FBDD8442F9DB0F232A68134097
:10130000092B07D1013080004751C7E71120B0E712
:101310002000F2E7032BC1D16B461B792D18EB702F
:10132000BCE7C046CFDA0000D3DA0000D8DA00000C
:1013300070B501240868204207D1042805D90F257B
:1013400001680D40092D02D14468200070BD032DB5
:1013500008D10A0992B24B0F92002B40D31A5B00BE
:101360001C43F2E7042DF0D102F0A0FCFEF734FF9D
:1013700040000443E9E7000010B5034A0D2103488B
:1013800004F09EFC10BDC04660DA000058DA000090
:1013900000207047042070470120704710B50020DE
:1013A00002F098FE10BD002070470020704700201A
:1013B00070470020704700207047002070470020D1
:1013C000704700207047000010B5034A0C21034805
:1013D00004F076FC10BDC0466CDB0000CCDB0000E6
:1013E00070470378002B03D05AB2002A01DB01308A
:1013F00070473F229343C03B59424B41C01803788A
:101400009343802BF4D10130F9E70000F8B50127B0
:10141000060014000800394227D104293FD90F23C0
:101420000A681A40042A3AD13C4213D1042C11D93B
:1014300022681340042B0DD102F038FC0500200077
:1014400002F034FC010028000BF070FB00282EDBBA
:101450001FD127E0E30722D502F028FC0A22002151
:101460000BF036FC0500601010E0174015D1042A7F
:1014700015D90F2312681340042B10D120004D10F2
:1014800002F014FC0A2239000BF022FC85420EDB2C
:1014900008DD002E09DC00200CE04D10E3E70F22F0
:1014A000054B1A700136022EF5D8042002E0042004
:1014B00076173040F8BDC046B0020020F8B50600EF
:1014C00000242B4BE500ED182B79032B09D00134B8
:1014D000FF2CF6D1300004F007FC041E46D1013C7D
:1014E00044E030000BF02CFBE3B2020031001800A6
:1014F00004F07AFC002839D12A6851688842E6D085
:101500008300D3189B680130F02BF7D101238000B2
:10151000083012181A42DAD1042AD8D90F211368D8
:1015200019400429D3D11B0998B20123013080004E
:1015300010181842CBD10428C9D90F2203681340D0
:10154000042BC4D102F0B2FB0327050009212800B7
:101550000BF0DEFA0028BAD0013F451C002FF5D170
:10156000310028000BF018FB8542B0D12000F8BDF7
:10157000A025002010B50124044002D04410200012
:1015800010BD042810D90F2302681340042B07D183
:1015900002F08CFB21000A220BF09AFB0400EEE71C
:1015A000032B01D10430F5E70D22014B1A70E6E759
:1015B000B0020020012210B5024018D1042802D93F
:1015C00003681A0992B201230B4012D1042902D9EF
:1015D0000B681B099BB20024934206D104309B0088
:1015E0000431C318984206D30124200010BD002204
:1015F000E9E70023EFE704780A78002C01D1002AFC
:10160000F2D0013001319442ECD00024EDE700002B
:10161000F7B50700009101933049314B002A02D001
:1016200002220A70013A00261A601B68CE54BE429C
:1016300000DBF7BD009AB300D058294B274D1C683A
:10164000C8239B0065191C1B0123184206D0254A9C
:101650004310210028000BF0FBF909E0224A002882
:1016600002D004281BD1214A210028000BF0F0F9F8
:101670001A4C20000BF064FA194A019B1060002BF1
:101680000BD07B1EB34208DD194B984205D8431C92
:101690001360202222540022E2540136C7E70428B6
:1016A00019D90F2301680B40042B04D102F0FEFA74
:1016B000104A0300CDE7092B03D143680E4A5B10A3
:1016C000C7E7032B08D10A0992B2490F92000B40D9
:1016D000D31A0A4ABDE70123094ABAE7B10200203A
:1016E000D40500206CE60000DADA0000E0DA000041
:1016F0001F03000097EC00003CDE00004BDE000002
:1017000056DE0000014B187000207047B002002028
:1017100070B502F06BF8094C0100251D1F2228004E
:101720000BF026FA28000BF00BFA04230430800893
:10173000000118432060200070BDC0468C020020CC
:10174000C368F0B59D00836889B05D190300183344
:1017500006930369069A9F00069B0290DF1943696E
:1017600001939B00D3180393D04B1B78002B26D1F9
:101770007F222B68CE491C1213409B005B58043516
:1017800001929F46029B587804F04AFF0023029A78
:10179000137027E0C54B1B78002B10D12B68019AE2
:1017A0001C121340C24A9B009B580435E9E7069B74
:1017B0003A1DD11ABD4BD82928DD1A221A70029B76
:1017C000BA4C9B6821780193EA1A029B92109B788D
:1017D00012021A43029B587804F02AFF0023029A4F
:1017E00023701370029B069A9B680193ED1A029B6B
:1017F000AD10DD60069BFE1A029BB6101E61039BB6
:101800009B1A029A9B10536109B0F0BD39001B78F6
:1018100017000C60002BD2D12B68019A1C121340C8
:10182000A34A9B009B580435ABE7069B3A1DD11A8F
:101830009E4BD82902DD1A221A70C0E738001B78A7
:1018400017002A68291D0260002B01D00D00B6E7A1
:101850006B68019A1C121340954A9B009B580835EF
:101860008FE7069B3A1DD11A904BD82902DD1A2228
:101870001A70A4E73900A4001B782C1917000C601B
:10188000002B9CD12B68019A1C121340884A9B00A4
:101890009B58043575E7069B3A1DD11A834BD8290E
:1018A00002DD1A221A708AE739001700814AA40063
:1018B000A2581B780A60002B00D080E72B68019AA1
:1018C0001C1213407A4A9B009B58043559E7043F89
:1018D000784B3A68A400E250744B1B78002B00D080
:1018E0006DE72B68019A1C121340714A9B009B58AC
:1018F000043546E76F4BA400E058FFF73BFE6B4B07
:1019000006001B78002B09D1043F3868FFF732FE30
:101910000123861976001E43664BE650634B1B7805
:10192000002B00D04BE72B68019A1C121340604A31
:101930009B009B58043524E7069B391DCA1A5B4B54
:10194000D82A02DD1A221A7039E70698039C012270
:10195000A04202D222000C3A126838001B780F0015
:101960000260002B00D02AE72B68019A1C1213405A
:101970004F4A9B009B58043503E7069A3B1D991A72
:101980004A4AD82902DD1A23137018E706990398EA
:10199000814218D202000C3A12684749521064186A
:1019A000A41AA40022583A601F00404B1B78002B59
:1019B00000D004E72B68019A1C1213403C4A9B009C
:1019C0009B580435DDE6182111700022EBE7069BD9
:1019D000039A934219D213000C3B1B68364A5B10E2
:1019E000A418043FE41A3A68039BA400E2502F4B6A
:1019F0001B78002B00D0E2E62B68019A1C121340E2
:101A00002B4A9B009B580435BBE61822274B1A70C3
:101A1000EDE7069B039A934228D2274B043FE61832
:101A200014000C3C23685B10F31A9B009858FFF7D6
:101A3000A1FD04903868FFF79DFD2468049B6410A5
:101A4000341B1E18012376001E43039BA400E6509E
:101A5000164B1B78002B00D0B1E62B68019A1C12A4
:101A60001340134A9B009B5804358AE618220F4BFB
:101A70001A70EDE7069B3A1DD11A0C4BD82902DDEE
:101A80001A221A709BE639001700039AA400A25884
:101A90001B780A60002B00D091E62B68019A1C127B
:101AA0001340034A9B009B5804356AE6B0020020AD
:101AB0003CDC0000982D0020FDFFFF3F043F039B0E
:101AC0003A68A400E250D64B1B78002B00D076E693
:101AD0002B68019A1C121340D24A9B009B58043574
:101AE0004FE6039BA4001C192368043F38685E106E
:101AF000FFF740FD0123361876001E43C84B2660D1
:101B00001B78002B00D05AE62B68019A1C12134058
:101B1000C44A9B009B58043533E6069BA4003F1B38
:101B2000BF4CBB420CD82378002B00D047E62B6873
:101B3000019A1C121340BB4A9B009B58043520E6B7
:101B4000B94802F0A3F82378002B00D037E62B68C1
:101B5000019A1C121340B34A9B009B58043510E6AF
:101B6000A300ED18002C00DA3CE6AD4B1B78002BEF
:101B700000D024E62B68019A1C121340A94A9B004E
:101B80009B580435FDE5043F3B68042B04D1A300BA
:101B9000ED18002C00DA25E6A14B1B78002B00D0B5
:101BA0000DE62B68019A1C1213409E4A9B009B581D
:101BB0000435E6E5043F3B68042B04D0A300ED1890
:101BC000002C00DA0EE6964B1B78002B00D0F6E5D1
:101BD0002B68019A1C121340924A9B009B580435B3
:101BE000CFE501233E1F306818420AD01841013862
:101BF000002809DB01234000A40018432D193060A0
:101C0000F0E5FFF7B7FCF2E7854B1B78002B01D01E
:101C10003700D4E52B68019A1C121340814A9B00BF
:101C20009B5837000435ACE5FF20610040000140BF
:101C3000FE38FF380143396002993B00896824125D
:101C400004916D1A0299AD1089782D020D438540DB
:101C500005437D6006991700039A521A921082403C
:101C600002439A60029B029A9C70E4B26F4BE400BC
:101C7000E35893606A4A1278002A03D008331D00A3
:101C800003979CE51D00019A9B680C351C121340BC
:101C9000644A9B009B58039773E53B1F1C68039A9B
:101CA000069B934232D10A20E30711D4042C18D9A1
:101CB0000F2322681340042B16D1200001F0F6FFF9
:101CC0000AF03EFFC8239B00984200D91800063056
:101CD000643004F0BDF800280FD1043D069B039347
:101CE00080E50720042CF3D02000431E9841FA23FE
:101CF0004042FF3318400730EAE7029B2100587842
:101D000004F0A8FC0023029A1370E7E7039B039AF0
:101D10000C3B1B6802995B109B00D31A0C3B1C60A8
:101D20001F1D1300083B1B685A108A70D2B23F492E
:101D3000D2005B0055589B0A029A9B009560ED18F3
:101D4000039B069A043B1B685B109B00D31803930C
:101D5000334B1B78002B00D031E52B68019A1C1205
:101D60001340304A9B009B5804350AE53B1F186816
:101D7000FFF700FCA40006003F1B1E2827DC0028FC
:101D80000DDC274B1B78002B00D018E52B68019A3F
:101D90001C121340234A9B009B580435F1E401F0C8
:101DA0000BFD033E361801F007FD214B801B9842C6
:101DB000F9D81B4B1B78002B00D000E52B68019A4B
:101DC0001C121340174A9B009B580435D9E4012389
:101DD000029A137001F0F0FC029B0A3886195E60CB
:101DE00000E53B1F1868FFF7C5FBA40006003F1B7A
:101DF00000280DDC0A4B1B78002B00D0DFE42B6899
:101E0000019A1C121340074A9B009B580435B8E402
:101E1000084B984210DD1D22014B1A70CFE4C046DA
:101E2000B00200203CDC000068DE0000A02500209D
:101E30003F420F0080EE36000123029A137001F03A
:101E4000BBFCFA239B005E430A3E3018029B58609D
:101E5000C8E4A300FF1A002320001A003900FFF78E
:101E6000D7FBD74ED74C3168200002F03FF9D64B54
:101E700031681860200004F0ADFA3168200004F0E9
:101E8000F0FBD24B1B78002B00D098E42B68019A12
:101E90001C121340CE4A9B009B58043571E4CB4B77
:101EA000A4001B783F1B002B00D088E42B68019A0C
:101EB0001C121340C64A9B009B58043561E40298EB
:101EC00004F02AF8C14B1B78002B00D077E42B6874
:101ED000019A1C121340BE4A9B009B58043550E4E3
:101EE0003B1F1B68002B58D13B0001260C3B186898
:101EF00006402FD046103A0001217300083A0B43E8
:101F00001360002E00DC95E0012173000B433A1FA3
:101F100013603B00083B1B680B419B1B04933B0079
:101F20000C3B186808423BD0049BA4005B188B4014
:101F30000B43039AA350A54B1B78002B00D03EE423
:101F40002B68019A1C121340A14A9B009B58043530
:101F5000FFF717FC04281BD90F2302681340092B35
:101F600002D143685E10C6E7042B08D101F09EFE43
:101F70000378002BBFD0FFF734FA0136F8E7032BC4
:101F800006D11609B6B2520FB6001340F61AB2E7E0
:101F900019228E4B1A70FFF712FC5B105E1EB0E721
:101FA000042842D90F2302681340092B05D1049B52
:101FB000A40002339B001B58BBE7042B2BD1039BCF
:101FC000A4001B19079301F071FE0600049C013464
:101FD000012C10DC3000FFF704FA831B1800049377
:101FE00002F078F8041E0ED001F060FE049A310071
:101FF0000AF000FA07E03178013C002906D11222EC
:102000000C00724B1A70079B1C6094E73000FFF7BE
:10201000E8F90600DCE7032B07D10122049BA400AA
:10202000C01803795B00134383E71922674B1A70CA
:10203000FFF7C5FB04357EE7A300069AFB189B1A41
:10204000D82B08DD1A22614B1A70FFF7B8FB01226A
:102050001C003A600437631E002CF8DC5B4B1B78D5
:10206000002B01D0FFF7ABFB2B68019A1C12134029
:10207000574A9B009B580435FFF783FB069A3B1D8C
:102080009B1A524ED82B03DD1A233370FFF797FBB0
:10209000069B039AA40093422AD23B1F1868FFF7BD
:1020A00069FA011E21DD039B0C3B1A685210824223
:1020B0001BDB9007801A474B4018C018039B800019
:1020C000C2583B1B1A60414B3F1B1B780437002B47
:1020D00001D0FFF774FB2B68019A1C1213403C4A95
:1020E0009B009B580435FFF74CFB20233370EAE735
:1020F0001823FBE7344BA4001A683B1B1F001A602F
:10210000324B04371B78002B01D0FFF758FB2B68AC
:10211000019A1C1213402E4A9B009B580435FFF76E
:1021200030FB3A1F1368042B02D13A00A4002D198A
:10213000264B1B78002B02D01700FFF740FB2B68C3
:1021400001991C120B4022499B005B581700043573
:10215000FFF717FB043F3B68042B04D00023A400C7
:102160003B602D190437194B1B78002B01D0FFF76A
:1021700026FB2B68019A1C121340154A9B009B58A2
:102180000435FFF7FEFAA3009C46F81A002C23DC66
:102190001C2200260D4B1A706346FF1A0B4B06607B
:1021A0001B780437002B01D0FFF709FB2B68019A3D
:1021B0001C121340064A9B009B580435FFF7E1FAB6
:1021C000D4050020B102002008000020B002002049
:1021D0003CDC0000FCFFFF3F002103685B10012690
:1021E0008A008258164003D10D22D54B1A70D3E7CE
:1021F0005210934200DD130001318C42EFDC5E008F
:1022000001231E43C8E7A3009C46F81A002C17DCE4
:102210001C220026CA4B1A706346FF1AC84B066080
:102220001B780437002B01D0FFF7C9FA2B68019AFD
:102230001C121340C34A9B009B580435FFF7A1FAB8
:10224000002103685B1001268A008258164003D1E2
:102250000D22BB4B1A70DFE75210934200DA1300D5
:1022600001318C42EFDC5E0001231E43D4E73B00CA
:102270000122083B1968A40011421DD03B1F1B68B6
:10228000134219D0114113410022994200DA04325D
:102290003B1B1A60AA4B3F1B1B780437002B01D055
:1022A000FFF78DFA2B68019A1C121340A54A9B0078
:1022B0009B580435FFF765FA02203B1F1A6840421D
:1022C000FFF7A4F83E1B3060E4E73B000120083B29
:1022D0001968A40001421ED03B1F1A6802421AD09E
:1022E00001415010CB0FD217884253413A1B9B003B
:1022F0001360934B3F1B1B780437002B01D0FFF773
:102300005EFA2B68019A1C1213408E4A9B009B5860
:102310000435FFF736FA01203B1F1A684042FFF7E9
:1023200075F83E1B3060E4E73B00083B18683B1F34
:102330001968A600BE1B0423814202D0042802D8DB
:102340000023336016E001231842F9D10F230268FD
:102350001A40042AF4D1033A1142F1D10429EFD9E9
:102360000A681340042BEBD1FFF724F9431E984170
:1023700080003060724BA4001B783F1B0437002B99
:1023800001D0FFF71CFA2B68019A1C1213406D4A0A
:102390009B009B580435FFF7F4F93B00083B186895
:1023A0003B1F1968A600BE1B0023814202D00428EF
:1023B00002D80423336016E001231842F9D10F2319
:1023C00002681A40042AF4D1033A1142F1D10429D7
:1023D000EFD90A681340042BEBD1FFF7EBF8434227
:1023E000584180003060564BA4001B783F1B0437D7
:1023F000002B01D0FFF7E3F92B68019A1C12134060
:10240000504A9B009B580435FFF7BBF93B00012263
:10241000083B1968A40011421ED03B1F1B681342E1
:102420001AD05B104A10D80FC9179A4241413B1B82
:1024300089001960424B3F1B1B780437002B01D0E9
:10244000FFF7BDF92B68019A1C1213403D4A9B000F
:102450009B580435FFF795F93B1F1A680120FEF7DA
:10246000D5FF3E1B3060E5E73B000122083B1968C1
:10247000A40011421DD03B1F1B68134219D011410B
:1024800013410022994200DD04323B1B1A602C4BA1
:102490003F1B1B780437002B01D0FFF790F92B6806
:1024A000019A1C121340274A9B009B580435FFF7E2
:1024B00068F93B1F1A680220FEF7A8FF3E1B306038
:1024C000E5E73B1F1B68A400043B5A1E93413A1BDF
:1024D00017009B0013601A4B04371B78002B01D0A8
:1024E000FFF76DF92B68019A1C121340154A9B00E7
:1024F0009B580435FFF745F93B00083B1868FFF788
:1025000039F83B1F06001868FFF734F80121A400D2
:102510003B1B1F00321852000A431A60084B043755
:102520001B78002B01D0FFF74AF92B68019A1C1287
:102530001340044A9B009B580435FFF722F9C0461C
:10254000B00200203CDC00003B00083B1868FFF7AD
:1025500011F83B1F06001868FFF70CF80121A400D2
:102560003B1B1F00321A52000A431A60E44B043727
:102570001B78002B01D0FFF722F92B68019A1C125F
:102580001340E04A9B009B580435FFF7FAF83B00E4
:10259000083B1868FEF7EEFF3B1F06001868FEF7C1
:1025A000E9FF02000121A4003B1B1F0072435200FF
:1025B0000A431A60D24B04371B78002B01D0FFF777
:1025C000FEF82B68019A1C121340CE4A9B009B58C0
:1025D0000435FFF7D6F83B1F1868FEF7CBFF061E41
:1025E00017D11F23C64A1370A4003B1B1F001E6097
:1025F000C34B04371B78002B01D0FFF7E0F82B68A2
:10260000019A1C121340BF4A9B009B580435FFF7E8
:10261000B8F83B00083B1868FEF7ACFF310007F044
:10262000C1FD012346001E43DEE73B1F1868FEF78D
:10263000A1FF061E17D11F23B14A1370A4003B1B34
:102640001F001E60AE4B04371B78002B01D0FFF734
:10265000B6F82B68019A1C121340AA4A9B009B589B
:102660000435FFF78EF83B00083B1868FEF782FF41
:10267000310007F07DFE01234E001E43DEE73B1FC5
:102680001868FEF777FFC217801850400122A40097
:102690003B1B1F00400010431860994B04371B7808
:1026A000002B01D0FFF78BF82B68019A1C12134006
:1026B000944A9B009B580435FFF763F8A300FE1A69
:1026C0003068012C25D1FEF755FF012307900493B4
:1026D0000AF08CF90799002900DC012107F048FE77
:1026E000049BA400C918012349001943844B3F1BD4
:1026F0001B7831600437002B01D0FFF760F82B689E
:10270000019A1C1213407F4A9B009B580435FFF727
:1027100038F8FEF72FFF04907068FEF72BFF049B3C
:102720000130C31A0793D3E7A300FE1A310020003B
:10273000049301F061FE049B3060FF1A704B043774
:102740001B78002B01D0FFF73AF82B68019A1C1276
:1027500013406C4A9B009B580435FFF712F83B006E
:10276000083B1868FEF706FF3B1F06001868FEF7D7
:1027700001FF02000121A4003B1B1F003240520058
:102780000A431A605E4B04371B78002B01D0FFF719
:1027900016F82B68019A1C1213405A4A9B009B584A
:1027A0000435FEF7EEFF3B00083B1868FEF7E2FE3B
:1027B00006003B1F1868FEF7DDFE32000121A40071
:1027C0003B1B1F00024352000A431A604C4B043764
:1027D0001B78002B01D0FEF7F2FF2B68019A1C1228
:1027E0001340484A9B009B580435FEF7CAFF3B0044
:1027F000083B1868FEF7BEFE06003B1F1868FEF790
:10280000B9FE32000121A4003B1B1F0042405200D0
:102810000A431A603A4B04371B78002B01D0FEF7AD
:10282000CEFF2B68019A1C121340364A9B009B581E
:102830000435FEF7A6FF3B1F1868FEF79BFEC0435A
:102840000122A4003B1B1F004000104318602C4BCA
:1028500004371B78002B01D0FEF7B1FF2B68019ADB
:102860001C121340274A9B009B580435FEF789FF32
:102870003B00083B1868FEF77DFE06003B1F18680A
:10288000FEF778FE320082400121A4003B1B1F00AE
:1028900052000A431A601A4B04371B78002B01D0F0
:1028A000FEF78DFF2B68019A1C121340154A9B00FE
:1028B0009B580435FEF765FF3B00083B1868FEF7A0
:1028C00059FE06003B1F1868FEF754FE3200024115
:1028D0000121A4003B1B1F0052000A431A60084B51
:1028E00004371B78002B01D0FEF769FF2B68019A93
:1028F0001C121340034A9B009B580435FEF741FF0E
:10290000B00200203CDC00003B000C3B1868FEF7E6
:1029100031FE3B00083B06001868FEF72BFEF1175E
:102920000200C317300007F075FD3B1F04900591AE
:102930001868FEF71FFE02000498059907F01EFDB7
:102940000123A4003E1B370040001843E54B3060D4
:102950001B780437002B01D0FEF731FF2B68019A5A
:102960001C121340E04A9B009B580435FEF709FFF8
:10297000A300FE1A310020000493FEF757FB049BCE
:102980003060FF1AD74B04371B78002B01D0FEF7BD
:1029900016FF2B68019A1C121340D34A9B009B58C8
:1029A0000435FEF7EEFEA300FF1A39002000FEF703
:1029B00059FBCC4B1B78002B01D0FEF700FF2B6896
:1029C000019A1C121340C84A9B009B580435FEF71D
:1029D000D8FEA300FE1A310020000493FEF782FB0C
:1029E000049B3060FF1ABF4B04371B78002B01D0CB
:1029F000FEF7E5FE2B68019A1C121340BA4A9B00B1
:102A00009B580435FEF7BDFEA300FF1A39002000D5
:102A1000FEF706FCB34B1B78002B01D0FEF7CFFE70
:102A20002B68019A1C121340AF4A9B009B58043537
:102A3000FEF7A7FEA300FE1A310020000493FEF764
:102A400077FC049B3060FF1AA64B04371B78002BE1
:102A500001D0FEF7B4FE2B68019A1C121340A24A63
:102A60009B009B580435FEF78CFE3B1F186801F055
:102A70001DF93A000121083A12680300A4000A4235
:102A800029D1042A0CD910680F22104001380828D7
:102A90000FD807F0F3FA052026220E0E0E0E2400A2
:102AA000924918000AF042F8434258413B1B80000B
:102AB00018608C4B3F1B1B780437002B01D0FEF7AE
:102AC0007EFE2B68019A1C121340874A9B009B587C
:102AD0000435FEF756FE8649E3E78649E1E7864975
:102AE000DFE78649DDE7069B3E1DF31A7D4CD82BB8
:102AF00003DD1A232370FEF762FE00F067FE012259
:102B00003B0040001043186023783700002B01D0B1
:102B1000FEF755FE2B68019A1C121340724A9B0067
:102B20009B580435FEF72DFE069B3E1DF31A6D4C97
:102B3000D82B03DD1A232370FEF741FE00F03CFE84
:102B40006F4A4000104001223B0010431860237878
:102B50003700002B01D0FEF732FE2B68019A1C12C1
:102B60001340614A9B009B580435FEF70AFE069A03
:102B70003B1D9B1A5B4CD82B03DD1A232370FEF7F9
:102B80001EFE00F023FE5F4B1A68831A904201D2AA
:102B90005D4A9B1801213A005B000B4313602378C8
:102BA0000437002B01D0FEF70AFE2B68019A1C1295
:102BB00013404D4A9B009B580435FEF7E2FD00F0A0
:102BC00005FE504BA4001860464B3F1B1B78002BA2
:102BD00001D0FEF7F4FD2B68019A1C121340424A03
:102BE0009B009B580435FEF7CCFD00F0FDFDA300D3
:102BF000002810D1FF1A3B4B1B78002B01D0FEF7A9
:102C0000DEFD2B68019A1C121340374A9B009B582B
:102C10000435FEF7B6FD3E00FF1A012320001A001E
:102C20003900FEF7F5FC394C2068643003F010F9E8
:102C3000002803D1043D3700FEF7D4FD029B216834
:102C40005A78334803F01FFD0123029A137000F0F5
:102C5000B3FD304B22681B68063253431818FFF748
:102C6000F5F800F0C1FDA300002810D1FF1A1D4B9C
:102C70001B78002B01D0FEF7A2FD2B68019A1C12D5
:102C80001340194A9B009B580435FEF77AFD3E001D
:102C9000FF1A2000012300223900FEF7B9FC1B4C6B
:102CA0002068643003F0D4F80028C3D0184803F03B
:102CB0007BFAC9E7A4003E1BFEF72AFD3700094B4B
:102CC00030601B780437002B01D0FEF778FD2B68AD
:102CD000019A1C121340044A9B009B580435FEF7CE
:102CE00050FDC046B00200203CDC000078DE000051
:102CF00080DE000087DE00008EDE000093DE000034
:102D0000FEFFFF7FDC05002037894100D40500204D
:102D1000B102002004000020FB4BA4001B783F1BE5
:102D2000002B01D0FEF74BFD2B68019A1C121340BB
:102D3000F64A9B009B580435FEF723FDA4003E1B7A
:102D4000300000F07EFD3700EF4B30601B78043719
:102D5000002B01D0FEF733FD2B68019A1C121340A3
:102D6000EA4A9B009B580435FEF70BFDA4003E1B6E
:102D7000300000F068FD3700E34B30601B7804370B
:102D8000002B01D0FEF71BFD2B68019A1C1213408B
:102D9000DE4A9B009B580435FEF7F3FCA300FE1AA5
:102DA00031002000049300F0C1FC049B3060FF1A46
:102DB000D54B04371B78002B01D0FEF700FD2B68A4
:102DC000019A1C121340D14A9B009B580435FEF710
:102DD000D8FCA4003F1B380000F038FDCA4B1B781C
:102DE000002B01D0FEF7EBFC2B68019A1C1213405C
:102DF000C64A9B009B580435FEF7C3FCA300FE1A8D
:102E000031002000049300F0F5FB049B3060FF1AB2
:102E1000BD4B04371B78002B01D0FEF7D0FC2B688C
:102E2000019A1C121340B94A9B009B580435FEF7C7
:102E3000A8FCA4003F1B380000F04EFDB24B1B78ED
:102E4000002B01D0FEF7BBFC2B68019A1C1213402B
:102E5000AE4A9B009B580435FEF793FC01212000ED
:102E600000F022FDA84B1B78002B01D0FEF7A7FC39
:102E70002B68019A1C121340A44A9B009B580435EE
:102E8000FEF77FFC0021200000F00EFD9E4B1B781A
:102E9000002B01D0FEF793FC2B68019A1C12134003
:102EA0009A4A9B009B580435FEF76BFCA4003E1B1E
:102EB000300000F03FFD3700934B30601B78043743
:102EC000002B01D0FEF77BFC2B68019A1C121340EB
:102ED0008E4A9B009B580435FEF753FCA4003E1B12
:102EE000300000F03BFD3700874B30601B78043723
:102EF000002B01D0FEF763FC2B68019A1C121340D3
:102F0000824A9B009B580435FEF73BFCA4003F1B04
:102F1000380000F0F7FC7C4B1B78002B01D0FEF74B
:102F20004EFC2B68019A1C121340784A9B009B5858
:102F30000435FEF726FCA4003F1B380003F0ACFF6D
:102F4000714B1B78002B01D0FEF739FC2B68019ADE
:102F50001C1213406D4A9B009B580435FEF711FC70
:102F6000A4003E1B300004F071F83700664B30605F
:102F70001B780437002B01D0FEF721FC2B68019A47
:102F80001C121340614A9B009B580435FEF7F9FB65
:102F9000A4003F1B380003F0FBFE5B4B1B78002BAB
:102FA00001D0FEF70CFC2B68019A1C121340574A03
:102FB0009B009B580435FEF7E4FBA4003E1B300049
:102FC00003F000FF3700504B30601B780437002BB4
:102FD00001D0FEF7F4FB2B68019A1C1213404B4AF8
:102FE0009B009B580435FEF7CCFBA300FF1A390069
:102FF000200001F075FD444B1B78002B01D0FEF73B
:10300000DEFB2B68019A1C121340404A9B009B5820
:103010000435FEF7B6FBA300FF1A3900200001F0CB
:103020007FFB394B1B78002B01D0FEF7C8FB2B68C8
:10303000019A1C121340354A9B009B580435FEF739
:10304000A0FBA300FF1A3900200001F001FC2E4B69
:103050001B78002B01D0FEF7B2FB2B68019A1C12E3
:1030600013402A4A9B009B580435FEF78AFBA300B5
:10307000FF1A3900200001F013FC234B1B78002BB2
:1030800001D0FEF79CFB2B68019A1C1213401F4ACB
:103090009B009B580435FEF774FBA300FE1A310019
:1030A0002000049304F042F8049B3060FF1A164B92
:1030B00004371B78002B01D0FEF781FB2B68019AA7
:1030C0001C121340114A9B009B580435FEF759FB14
:1030D000A300FE1A31002000049304F02FF8049B93
:1030E0003060FF1A084B04371B78002B01D0FEF725
:1030F00066FB2B68019A1C121340044A9B009B58E4
:103100000435FEF73EFBC046B00200203CDC000068
:10311000A300FE1A31002000049304F017F8049B6A
:103120003060FF1AAA4B04371B78002B01D0FEF742
:1031300046FB2B68019A1C121340A64A9B009B5821
:103140000435FEF71EFBA300FE1A31002000049395
:1031500004F004F8049B3060FF1A9D4B04371B7881
:10316000002B01D0FEF72BFB2B68019A1C12134099
:10317000984A9B009B580435FEF703FBA300FF1AF7
:103180003900200001F02CFC914B1B78002B01D062
:10319000FEF715FB2B68019A1C1213408D4A9B0009
:1031A0009B580435FEF7EDFAA300FF1A3900200002
:1031B00001F09EFB864B1B78002B01D0FEF7FFFA37
:1031C0002B68019A1C121340824A9B009B580435BD
:1031D000FEF7D7FAA300FE1A31002000049301F095
:1031E00003FB049B3060FF1A794B04371B78002BDC
:1031F00001D0FEF7E4FA2B68019A1C121340754ABD
:103200009B009B580435FEF7BCFAA300FF1A390057
:10321000200001F0B1FA6E4B1B78002B01D0FEF7B5
:10322000CEFA2B68019A1C1213406A4A9B009B58E5
:103230000435FEF7A6FA002C79DD3B1F1E68012C31
:103240000CD1264207D1042E05D90F233268300055
:103250001340042B11D001235B4213E0022CFAD15E
:103260003B00083B186801231842F4D10428F2D926
:1032700002680E331340042BEDD100F017FDFEF76A
:103280001DF90300A200BF1A5A1C50D00020022CC6
:1032900011D101223240824223D1042E21D90F21A3
:1032A0003068014009291CD171684810C0B2810002
:1032B000914211D17F18FF2B1BD81C0204433A0006
:1032C000069B0C32D31AD82B01DCFEF7ADFC1A2278
:1032D0003F4B1A70FEF773FAB418A468BC5004325E
:1032E000E6E70B223A4B1A7000233B600437FEF7E7
:1032F00066FA069A0299BA1A86009210BE1B0A61F3
:10330000310098470022344B371D1A60304B306033
:103310001B78934201D0FEF752FA2B68019A1C12D7
:1033200013402C4A9B009B580435FEF72AFA0023D1
:103330003B60274B3A1D1B78002B02D01700FEF78D
:103340003EFA2B6801991C120B4022499B005B58E6
:1033500017000435FEF715FA069B029AFB1A9B101C
:103360001361A300FF1A3900200002F05BFF184B25
:103370001B78002B01D0FEF722FA2B68019A1C1251
:103380001340144A9B009B580435FEF7FAF9069B3C
:10339000029AFB1A9B101361A300FE1A3100200051
:1033A000049302F03FFF049B3060FF1A084B043780
:1033B0001B78002B01D0FEF702FA2B68019A1C1231
:1033C0001340044A9B009B580435FEF7DAF9C046C7
:1033D000B00200203CDC0000E40F00200023F7B521
:1033E0005A1E0192002B07DA01F090FB03F032F82D
:1033F00003F0A8F91923019300263000194B19682E
:10340000B14212DD184B1A6801328A420FDAF024F9
:103410001A601D68154F6C43E35D002B1FD0E41943
:10342000022B06D12000FEF78BF9019BD8E7002282
:10343000EDE7012B0DD1002801D100F0BDF9F022FC
:103440006A43BB185B680A49C31A8B4201D802233E
:10345000BB54F0235D43054BEB5C022BE2D00136FD
:10346000CCE7C046D805002000000020401C00200A
:103470003F420F0080220B4B52001A600121A8220C
:10348000A920094BD20019649A58C00005321A507D
:1034900006481A50C122C020920000039850044BE5
:1034A0001970704700E100E0008000404C0500000A
:1034B0000106002004207047F8B550C901232200FE
:1034C0001A40101E2DD03340181E2AD06410002040
:1034D0001A2C26D81D4B761035009E4200DD1D00AB
:1034E0001B4F3B5D012B05D00121200005F0B6F9F3
:1034F00001233B55174B1B78002B01D1FFF7BAFF77
:103500000023154A9E420DDCFF2514491448D65C61
:10351000B44202D15E007052D5540133042BF6D16F
:103520000420F8BDD15C8C4203D10C4A5B009D5253
:10353000F6E70133042BF5D10023D15CFF2901D13B
:10354000D454F2E70133042BF7D1E9E788130000E4
:10355000E4050020010600201C0000200E000020D1
:10356000DC05000070B530C9012322001A40101E8E
:103570001BD02B40181E18D064101A2C00D9192407
:10358000154E335D012B05D00121200005F066F9B1
:103590000123335569100800104A1038104B90422F
:1035A00004D9012252421A60042070BD1C600D48EB
:1035B00006F0F8FD0C4B040018800C4B1B78002B18
:1035C00001D1FFF757FF0122094B9A64A922D200CB
:1035D000995864189C50E7E7E405002090860100A4
:1035E0001800002020A107000C0000200106002088
:1035F0000080004070B501240D68254204D10D20E3
:10360000FEF780F8200070BD6D101A2D17D8002429
:10361000012804DD4C68043C63425C416400094EAF
:10362000735DA34204D02100280005F017F97455FA
:10363000280005F047F903000420012BE3D0002007
:10364000E1E7C046E4050020F8B501260D68340026
:10365000B04200DD4C682B003340181E0BD0230015
:103660003340181E07D06D10002D05DCA12300206B
:103670001E4ADB00D650F8BD641000201A2CFAD880
:103680001B4F3B5D012B04D00121200005F0E6F823
:103690003E552900174806F085FD0A21053006F041
:1036A00081FD154BA400E258144B12021343A222D1
:1036B0001349D2008B50134C0C4B9C50124C195197
:1036C000012412495C50124B196900219950114A8A
:1036D000904200DD1000A8228021D20098500122E3
:1036E00089005A5004201A60C5E7C04600F0014026
:1036F000E405002000B4C4045CF0000003000300F3
:103700000060004040A100401405000004050000D6
:1037100000A00040FFFF0000030010B50120002BB7
:1037200002DC1B30FDF7EEFF10BD0000F8B50124F0
:103730000B6806000D00234204D10D20FDF7E2FFC7
:103740002000F8BD5B1004D103F04EFB4000204385
:10375000F7E72000072BF4D80D4A9B009C580D4F2B
:103760003B5D002B05D00021200005F077F80023F9
:103770003B55012E06DD6B68042B03D1022120008E
:1037800005F06CF8200004F017FF01244000DEE78C
:1037900008DF0000E40500200420704710B5002871
:1037A00003DC1C20FDF7AEFF10BD0B680020DB071B
:1037B000FAD40D30F6E700000122034B1A64A82268
:1037C000D20098587047C046008000400122054B47
:1037D00010B51A64A822FA21D2009858890006F080
:1037E00057FC10BD00800040012070470048704722
:1037F00028DF00001B20704770B5054E0400335CC5
:103800000D008B4202D005F029F8355570BDC04639
:10381000E405002070B50024084D635D012B09D13B
:103820000021200005F038F80021200005F016F8EE
:103830000023635501341B2CEED170BDE40500203C
:10384000704711207047372070470000F8B50126F7
:103850000568354202D04468344203D10D20FDF79B
:1038600051FFF8BD6D101A2DFBD80A4F7B5D012B5F
:1038700004D03100280004F0F1FF7E5506496410A1
:103880008C4202DCE143C9172140280004F01AFFF2
:10389000E7E7C046E4050020FF03000010B508007C
:1038A000FFF7D4FF002010BD70B504000D001A28EA
:1038B0000ED8084E335C012B04D0012104F0CEFF5A
:1038C00001233355290020004D1EA94104F0E4FFD7
:1038D00070BDC046E4050020036810B5DA0703D4C4
:1038E0000D20FDF70FFF10BD4168581004394A4202
:1038F0005141FFF7D9FFF6E710B50800FFF7ECFFDD
:10390000002010BD37B569460A00064B30CB30C2E7
:1039100003680220042B02D100F09AFF37BD00F0AB
:10392000BFFFFBE7A0DE000010B50800FFF7EAFFCD
:10393000002010BD10B5084C237D002B05D00021C0
:10394000142004F08BFF00232375142004F0BAFF29
:1039500043425841800010BDE405002010B5084CDA
:10396000A37D002B05D00021162004F077FF002353
:10397000A375162004F0A6FF43425841800010BDF5
:10398000E4050020A02200230349D2008B50034904
:1039900010328B507047C04600F00140006000407C
:1039A000F7B52F4D2F4EEB6C002B14D0A92400231C
:1039B000E4003759EB642C4B186800280BDB2B4BC9
:1039C00019784A425141C9B2197004F065FF284B79
:1039D0001B88DF1937512B6D002B38D00021254B68
:1039E000254FF45829653A780193244D8A4206D030
:1039F0002B68032B03D8224AD05C04F04DFF2B68C0
:103A0000204A0133134004D50422013B52421343A0
:103A100001331B4900228C462B60042B18D06046D2
:103A2000C05C591CFF2802D10B000122F5E7002AD7
:103A300000D02B60012104F02FFF01233B702B6885
:103A4000114A5B009B5A0C34E418019BF450F7BDFB
:103A500001235B422B6000233B700C4BF4E7C04614
:103A6000FC8000400080004018000020000600207C
:103A70000C0000204C050000FF050020E0050020A0
:103A80001C000020030000800E0000205C460000A7
:103A9000084B094AFF201A805A809A80DA80002356
:103AA000064A07491370074A087048708870C87042
:103AB000136070470E000020DC050000FF050020A9
:103AC0001C000020E00500200122024B52421A6037
:103AD0007047C0461800002010B5034A0C21034867
:103AE00002F0EEF810BDC046A8DE00009EE7000020
:103AF000E12170B54902194804F0D4FA00240122EA
:103B00000320174B17491A615C5004315850801834
:103B1000083158501A60063004F048FDFF21124A5F
:103B2000A15401341B2CFBD1012200200F4B0100BA
:103B30001A6004230E4A0F4D1468002CFCD02C6828
:103B40000002013B20431160002BF5D101220A4BFA
:103B50001A6004F063FC01F025F970BDC81B002059
:103B60000080004004050000E405002000D0004073
:103B700000D1004008D5004004D00040F8B50B4EFD
:103B8000070030000D0004F0D5FA0400A84200DD63
:103B90002C003D00EB1B9C4205DD300004F0D4FA04
:103BA00028700135F6E72000F8BDC046C81B00208C
:103BB00010B50100014804F07DFA10BDC81B0020BB
:103BC00010B5054C200004F083FAE12120004902E1
:103BD00004F068FA10BDC046C81B0020C3070CD40F
:103BE000064B1B68834208D8054B1B68984204D8D3
:103BF000031F1B68002B00D0180070470C06002024
:103C0000080600200023012210B50A48990001335C
:103C10004250642BFAD1084C084B00211A60200056
:103C2000074A08F003FC074B074A6360074B1A601A
:103C300010BDC046982D002010060020080000206E
:103C4000D4090000302700001406002004060020DC
:103C500010B5044B044A1A60044B054A1A60FFF77A
:103C6000D1FF10BD0C060020100600200806002021
:103C7000E40F0020044B1B681868000980B202386A
:103C8000C343DB17184070470406002000B59BB003
:103C90000200054901A808F00DFF01A802F0A0FAF2
:103CA00002F050FDFCE7C046F1DF00000B4BC207FD
:103CB00004D4042804D80A4B00D00A4B18007047DB
:103CC0000F2203681A40031D042AF7D0064B092A65
:103CD000F4D0064B032AF1D0054BEFE7CBDF000011
:103CE000E0DA0000DADA0000D5DF0000E5DF0000EE
:103CF000DCDF00000020064A0649131F1860136825
:103D00001B099BB202339B00D2188A42F5D370473D
:103D100014060020E40F0020F7B50F240126314BD4
:103D2000314A1968314B324D186813681F0027401B
:103D3000072F26D813681B099BB202339B00D218A9
:103D4000AA42F2D300242B4EA500AD192868FFF734
:103D500045FF01342860642CF6D1274C2068FFF71A
:103D60003DFF2060254C2068002802D0FFF736FF79
:103D700020600025224B1B680093009B9D4214DBB2
:103D8000F7BD1B099BB29B00D3189A42D2D01F6883
:103D9000374208D1B94206D2B84204D3043F3F6843
:103DA000002F00D01F60043BEFE7F0236B43154A60
:103DB0009B181A78002A01D10135DEE71F693C23E0
:103DC00000266B43DB199B0001930136BB1BF3D428
:103DD000019BB4001C1B0B4B1C19A069FFF7FEFED6
:103DE000A061F2E70C06002014060020080600205F
:103DF000E40F0020982D002008000020E40F002090
:103E0000D8050020401C0020F7B50124204246D1EF
:103E1000234B1B689C46984241D3224B1B6801935D
:103E200098423CD8031F1B68002B38D1020003685E
:103E300000941B099BB2002B0FD10099131F19602E
:103E400090422CD015682B1F1B68990069180C68CC
:103E5000013B14600A602A00EDE79D0055192968AE
:103E6000009C214219D18C4517D8019C8C4214D357
:103E70000E1F3468002C10D10F680F343C40072C03
:103E800008D92F60151F2B600B680A601B099BB2B5
:103E90000A00D0E700993160CDE7013BCBE7F7BDE1
:103EA0000C060020080600200D4970B50A000D4DD3
:103EB0001368141F1B0926689BB2981C002E0BD098
:103EC00000238A4200D00B0023608300C9188000C1
:103ED0001218AA42ECD370BD1B011360F7E7C0466D
:103EE00014060020E40F0020F8B5124C27000F2222
:103EF0003B681D09ADB213420DD06E1CB600A7423F
:103F000004D032003900200008F07DFA0022A31905
:103F10000436A4191A600235AD00074B7F199F4281
:103F2000E5D31B1B9B10013B1B012360034B1C6053
:103F3000F8BDC04614060020E40F0020040600204F
:103F4000F0B59BB0FFF738FC00240700214AA3001E
:103F5000D0580134FFF758FF642CF7D11E4B186876
:103F6000FFF752FF1D4B1868002801D0FFF74CFFE8
:103F700000261B4B1B689E4217DBFFF795FFFFF7E0
:103F8000CBFEFFF7B1FFFFF717FC164BC21B1B68F8
:103F900015491B6801A81B099BB2023B08F08AFD6A
:103FA00001A802F01DF91BB0F0BDF02575430F4BC1
:103FB000ED182B78002B01D10136DAE72B695C1E56
:103FC000002CF9DBA300EB189869FFF71DFF013CFB
:103FD000F6E7C046982D002008000020E40F0020DE
:103FE000D805002004060020ABDF0000401C0020A4
:103FF000F7B5174D4F1C2B6806001B680C001B09FA
:104000009BB201929F420BDBFFF79AFF2B681B6864
:104010001B099BB29F4203DB0A20FDF773FBFEBD29
:104020002868A71CBA00DB1B81181B010B602960E4
:104030000021031F19600F231E40030024012643A3
:1040400040C3083A9A189A42E9D9019902C3FAE79B
:1040500004060020F7B503000122134004000D0000
:104060000193002B2BD1174B1B68834227D8164B8B
:104070001B68834223D90F23144F3860006818400F
:10408000FFF7B6FF019B3C68061E3B6017D0236814
:1040900004301B099BB29D4200DD1D00AA00211DBA
:1040A000251F08F0A7F9FFF725FE2E60FFF734FE65
:1040B00000232B602268064B13402360340020004D
:1040C000FEBDC0460C06002008060020E40F0020BC
:1040D000F0FF0F000323043010B5C1171940091871
:1040E000891000220420FFF783FF10BD70B5050082
:1040F00008000C00FFF7EEFF0023002804D170BD7C
:10410000E95CC21811710133A342F9DBE343DB1709
:104110001C40002304192371F1E7F0B50C009BB09B
:10412000022804DC1C20FDF7EDFA1BB0F0BD0123D2
:104130000868184206D1042804D90F2601683140C6
:10414000042901D00E20EEE761680D001D40F9D171
:104150000429F7D90A683240042AF3D1A2681A4226
:1041600001D10D20DFE7FFF7A1FD06006068FFF732
:104170009DFDA768010001AC7F103000257003F0A1
:10418000BBFB39006423220003F01BFC200008F075
:10419000D7FC01002000FFF7A9FFC6E710B51C4CB3
:1041A000A544041E02D1FFF795FF0BE003F0BCFA13
:1041B0000138062828D805F061FF090911182904DB
:1041C000240000208023DB009D4410BD200003F06C
:1041D00027FB011B2000FFF789FFF3E7200003F016
:1041E000CDFA430001201843ECE780226946D20053
:1041F000200003F0DAFA684608F0A2FC01006846E5
:10420000E9E704210348E6E70020CCE70420D9E7EA
:1042100000FCFFFF38E0000070B50C00022803DC52
:104220001C20FDF76FFA70BD01230868184206D103
:10423000042804D90F2501682940042901D00E2043
:10424000EFE761681942FAD10429F8D90A682A40CF
:10425000042AF4D1A2681A4201D10D20E1E7FFF748
:1042600025FD05006068FFF721FDA46801006410CA
:10427000280003F041FB210003F07EFBFFF78EFFD7
:10428000D1E770B50D00012803DC1C20FDF73AFAD8
:1042900070BD01240868204206D1042804D90F21EA
:1042A00002680A40042A01D00E20EFE76A68224221
:1042B000FAD1042AF8D913680B40042BF4D1FFF784
:1042C000F5FC06006868FFF7F1FC0100300003F020
:1042D00013FB03F095FB40002043D9E7F8B5070036
:1042E0000C001C20012F0BDD01250868284206D197
:1042F000042804D90F2102680A40042A03D00E20A2
:10430000FDF700FAF8BD62682A42F8D1042AF6D90E
:1043100013680B40042BF2D1FFF7C8FC060060685D
:10432000FFF7C4FC0100022F14D0A4682C4211D066
:104330006410300003F0E0FA050003F0F5F90128FD
:1043400011D1002C02DD0135012C06D12800FFF728
:1043500025FFD7E701246442EBE7280003F06DFA5C
:10436000013C0500F0E70228F0D1002CEEDD01351C
:10437000012CEBD000222800110003F090FA03F08A
:104380005CFA013C0500F3E710B50124086804401D
:1043900016D04410200006F099F9154906F064F88B
:1043A00007F04AFF04F09CFB0022124B07F0FEF8D6
:1043B00004F03EFB07F0D0FE43000120184310BD7F
:1043C000042810D90F2302681340042B07D1FFF7EC
:1043D0006DFC21000A2208F07BFC0400DAE7032BC5
:1043E00001D10430F5E70D20FDF78CF9D2E7C04686
:1043F000D30237390000D040086870B501240500A9
:10440000254006D1042804D90F2302681340042B49
:1044100003D00E20FDF776F970BDFFF747FC037857
:104420002900233B5A4253411022C01808F050FC87
:1044300080239B05C218044B9A4201D91420E9E756
:1044400040002043E8E7C046FFFFFF3F10B5034AA6
:104450000621034801F034FC10BDC04608E000000E
:1044600002E000000020704710B51E20FDF74AF959
:1044700010BD10B51E20FDF745F910BD10B51E206A
:10448000FDF740F910BD10B51E20FDF73BF910BD3A
:1044900010B51E20FDF736F910BD10B51E20FDF732
:1044A00031F910BD10B51E20FDF72CF910BD10B567
:1044B0001E20FDF727F910BD10B51E20FDF722F9CB
:1044C00010BD10B51E20FDF71DF910BD10B51E2042
:1044D000FDF718F910BD10B51E20FDF713F910BD3A
:1044E00010B51E20FDF70EF910BD10B51E20FDF70A
:1044F00009F910BD10B51E20FDF704F910BD10B567
:104500001E20FDF7FFF810BD10B51E20FDF7FAF8CC
:1045100010BD10B51E20FDF7F5F810BD10B51E201A
:10452000FDF7F0F810BD10B51E20FDF7EBF810BD3B
:1045300010B51E20FDF7E6F810BD10B51E20FDF7E2
:10454000E1F810BD10B51E20FDF7DCF810BD00002D
:1045500010B5034A1821034801F0B2FB10BDC04654
:1045600074E0000034E100000120034B1860034BAD
:104570001B6883401843704700100020E80F00209C
:10458000F0B5EFF310810123194083F31088134A2B
:10459000A1261268124D013A9340A022114FD20574
:1045A000F600002B17D02C68945103420BD0C04664
:1045B000C046C046C046C046C046C046C0462C683D
:1045C000D4515B08EDE7D451C046C046C046C04652
:1045D000C046C046F5E781F31088F0BD20000020FA
:1045E000F40F00200C05000030B585B001AD0C22A1
:1045F0000649280007F0FEFE0024285D0121013451
:10460000FFF7FAF80C2CF8D105B030BD70E20000CD
:10461000F7B56A463B4B01AE1380062393703A4BC5
:1046200033800F23B370FFF7C7F8384B384DC018ED
:104630002B68984201D200232B602C68002C41D1BA
:10464000375D01213800FFF7D7F801340021380029
:1046500004F022F9032CF3D1002401276B461E5DE0
:1046600039003000FFF7C8F801343900300004F099
:1046700013F9032CF2D1C8200138C046C046C04609
:10468000C046C046C046C046C046C046C046C046FA
:10469000C046F1D16B4600211878FFF7ADF86B46A4
:1046A00000215878FFF7A8F86B4600219878FFF7AB
:1046B000A3F8FFF781F8FA2300241B01C018286033
:1046C0002000FEBDFFF778F82B6800249842F7D34E
:1046D000042003F071FF0600052003F06DFF36187B
:1046E000062003F069FF0B4B9B1B181A0A4BA042D4
:1046F00006DB18600023094A2B6013600124DFE702
:104700001C60F7E7040500000D0E000010270000F4
:10471000F80F002043030000E80F002000100020E5
:104720000022054B10B51A60044B1B68934201D060
:1047300002F09AFF002010BDFC0F0020EC1A0020B0
:1047400010B5041E0CDA1A24084BA400E2581F23EB
:104750001A401E3B9340064A1360064A136010BD80
:10476000FFF748F8A042EEDDEEE7C0465CF000003F
:10477000F40F0020180500500200086810B5C307A8
:104780000FD540101823012A03DD4A68042A00D1FE
:104790000833054A1360FFF753F8FFF7D1FF0020F5
:1047A00010BD01204042EDE72000002010B501249B
:1047B000044002D04410200010BD042810D90F235B
:1047C00002681340042B07D1FFF770FA21000A2278
:1047D00008F07EFA0400EEE7032B01D10430F5E780
:1047E0000D20FCF78FFFE6E70868F8B5C3071AD578
:1047F000FFF7DCFF0300203B5E2B25D80520434359
:1048000001221D180020114E9D4219D005211024AF
:10481000F75C3C4200D08018013952006410002936
:10482000F7D10133F0E704280ED90F2203681A40AC
:10483000042A09D11B099BB2002B05D00379DAE7C2
:10484000012340001843F8BD0120FCE77CE2000092
:1048500070B508680D00FFF7A9FF04006868FFF74E
:10486000A5FF621E0100042A14D8451E042D11D88C
:1048700005236B439B18012215009D402B00064821
:1048800005682B430360054B1B68002B02D02000FA
:1048900002F0EBFE002070BDFC0F0020EC1A00209F
:1048A00070B508680D00FFF781FF04006868FFF726
:1048B0007DFF621E0100042A13D8451E042D10D866
:1048C00005236B439B1801229A40074803689343D2
:1048D0000360064B1B68002B03D00022200002F06F
:1048E000C4FE002070BDC046FC0F0020EC1A002062
:1048F000F0B5050089B008680C00FFF757FF069077
:10490000022D36DD6068FFF751FF0190A068FFF7C8
:104910004DFF04000127231D661E0793731C02939D
:10492000079B9E4235D0052373430593019B019D50
:1049300005330493049BAB421ED0042E16D86B1E85
:10494000042B13D80122059B2349013B5B199A4094
:104950009446224A0B681068069A3A4003920DD09A
:1049600062461A430A60012200280DD17F000135FA
:10497000E0E701240194CDE7029ECFE7624693432E
:104980000B600028F2D0039A0299280002F06DFE15
:10499000ECE7019B1E1D042E1AD8012C18D100250E
:1049A00005273B0021006B439B1999400B000A4AE5
:1049B000013511689943094B11601B68002B05D024
:1049C000019B0022581D290002F04FFE052DE8D161
:1049D000002009B0F0BDC046FC0F0020EC1A0020FA
:1049E000F0B53B4B85B01B680C00002B03D10120B8
:1049F0004042FFF7A5FE012627683E403CD1042F28
:104A00003AD90F233A681340092B35D17B685B10E4
:104A10000293029B9E4258DAB300FB189868FFF796
:104A2000C5FEFF2305000414001218401C4029494C
:104A30002B404043019305F0B5FB030420002549BA
:104A40006043039305F0AEFB039C0002044301980E
:104A50002049404305F0A6FB1F4B20431B68202B39
:104A600006D1AD00AD0E1D4BAD00EC580002204349
:104A7000FFF786FD0136CCE73800FFF797FEFF26EB
:104A800005000714001230401249404305F08AFB2C
:104A90003740040438000F49784305F083FB2E406B
:104AA0000002044330000B49704305F07BFB0A4BC6
:104AB00020431B68202B06D1AB009B0E074A9B00AE
:104AC0009B5800021843FFF75BFD002005B0F0BDC6
:104AD000F40F0020590600002000002058E40000D8
:104AE000086810B5C30703D5FFF760FE054B1860D3
:104AF000054B1B68002B03D0024B186802F0B6FD73
:104B0000002010BDFC0F0020EC1A00207FB5A04C47
:104B10002368002B0AD19F4A1268002A06D19E4BB7
:104B20001B68002B01D0FFF773FD7FBD9B4D2A68EA
:104B3000002A26D1984A1268002A1BD0FFF768FD88
:104B40000028F2D0FFF750FD924B24681A681C60D1
:104B5000002A16D0002C14D101AD0C229049280057
:104B600007F048FC285D00210134FEF745FE0C2CBF
:104B7000F8D1DAE7874A1268002AE5D1002BE3D0A2
:104B8000E0E700210D2003F087FE00210E2003F056
:104B900083FE00210F2003F07FFE2E68012E5DD0E2
:104BA000022E00D1A2E0002E51D101363100794C05
:104BB00004202368994303F06FFE04212368052035
:104BC00019404B42594103F067FE1021236806202B
:104BD00019404B42594103F05FFE802123680901CF
:104BE00019404B4259410C2003F056FE80212368A6
:104BF000090219404B4259410B2003F04DFE802120
:104C00002368490219404B4259410A2003F044FEEF
:104C100080212368890219404B425941092003F041
:104C20003BFE80212368C90219404B4259410820AC
:104C300003F032FE802321681B0319404B42594187
:104C4000072003F029FE31000D2003F025FE2B681C
:104C50000321581C05F08CFB296066E702214D4CAE
:104C60000720236819404B42594103F015FE0820E4
:104C7000216801404B42594103F00EFE8021236818
:104C8000C90019404B425941052003F005FE80211F
:104C90002368490119404B425941062003F0FCFDAD
:104CA00080212368C90119404B425941042003F077
:104CB000F3FD80212368890319404B4259410A20A2
:104CC00003F0EAFD802321681B0419404B4259413F
:104CD000092003F0E1FD31000C2003F0DDFD31007F
:104CE0000B2003F0D9FD31000E20AEE72021294C26
:104CF0000720236819404B42594103F0CDFD402164
:104D00002368082019404B42594103F0C5FD80211A
:104D10002368092019404B42594103F0BDFD802111
:104D20002368490019404B4259410A2003F0B4FD61
:104D300080212368890019404B4259410B2003F020
:104D4000ABFD80212368890119404B4259410C2059
:104D500003F0A2FD80212368490319404B425941C9
:104D6000062003F099FD80212368C90319404B42B6
:104D70005941042003F090FD802321685B04194011
:104D80004B425941052003F087FD01210F205CE7CC
:104D9000FC0F0020F00F002000100020EC0F00207E
:104DA00070E20000012010B54042FFF7C9FC00206E
:104DB000FFF7E6FB10BD000010B5034A09210348C8
:104DC00000F07EFF10BDC04658E50000A0E50000E1
:104DD0008023F0B502255B051A690A4C0A4BA1260F
:104DE0001D5103278025F600ED00BA43884202D307
:104DF00000221A51F0BD5F59002FFCD09851801845
:104E0000F4E7C0460405000000E0014010B50028AA
:104E100006D1C020B02140028902FFF7D9FF10BDA2
:104E2000B02080218002C902F7E7000043425841C8
:104E3000064B40421840B0239B02C0180368002074
:104E40001A0E532A01D11B02180A704700C0FEFF38
:104E500030B501248025054B054AED009C505C5976
:104E6000002CFCD001600021995030BD00E00140D1
:104E70000405000043425841074B40421840B0230C
:104E80009B02C018A62310B50902DB05090A1943C5
:104E9000FFF7DEFF10BDC04600C0FEFFF0B50124E5
:104EA00080260D4B0D4DF6005C51002902DC0022DE
:104EB0005A51F0BD577814783F0227439478240460
:104EC0002743D478043224063C439F59002FFCD05A
:104ED00010C00139E9E7C04600E0014004050000C8
:104EE00070B505004B680A009C1C2100A400FFF768
:104EF000D5FF281970BD0000134B1B68002B0CD088
:104F00008022B023D2029B0200280BD11A1D5B68BD
:104F10001B0E522B00D110007047B022C02392020A
:104F20005B02F1E782420DD903681B0E522B09D1B7
:104F3000436802339B00C018824203D903681B0EEA
:104F4000522BE9D00020E7E704110020F0B5002043
:104F5000B7B00024FFF7D0FF270005002600002D82
:104F60002ED1284D2868FFF761FF32003B000190E9
:104F70000094254904A807F09DFD04A801F030F92C
:104F8000224B64201C682B68A0215A425341204ABE
:104F90005B421340B02292029B18E41A604349021C
:104FA00005F000F9A02252020300009219492200E4
:104FB00004A807F07FFD04A801F012F937B0F0BD96
:104FC000FF226B6829689C460233FF180B120136DA
:104FD00013409C4200DA1C00FF200A140240039296
:104FE0006246014001920091039A0B4904A807F020
:104FF00061FD04A801F0F4F82800FFF77DFF05002B
:10500000ADE7C04604110020AAE600000811002008
:1050100000C0FEFF54E6000096E6000070B50020D8
:10502000FFF704FF04000120FFF700FF844200DACD
:1050300004000A4B1D686A42554128001D60FFF7B5
:10504000E5FEA0226B4252021340054A28009B183D
:10505000044A611C1360FFF70DFF70BD04110020AE
:105060000480010008110020F8B50020FFF7DEFEE3
:1050700007000120FFF7DAFE3E00204D0643204CDA
:105080000DD18021C020C9024002FFF7A1FE0121FD
:105090003000FFF7EFFE1B4B2E6023601DE08742C0
:1050A00009DD0023B0212B60164B890223602368A1
:1050B0000020012517E0012380212B60124BC9023B
:1050C0002360F4E7120E522A08D0002800D0236093
:1050D0000E4801F085F8FFF7A1FFF8BD28005A68D7
:1050E000023292009B188B4205D21A68561CE9D1F5
:1050F0000028F2D0D1E72160EFE7C046041100207C
:10510000081100200480010004C002006FE60000C6
:1051100070B50020FFF7F0FEFF260500002801D142
:10512000280070BD03681C143440FFF7E5FEDA2C3C
:10513000F4D10500F2E70000FF2270B5134CD20055
:105140000021200007F072F9FF25FFF7E1FF00269C
:10515000002800D170BD03681A142A400A2A0AD117
:105160001A122A40FF2A03D0D200A1180B71A050B6
:10517000FFF7C2FEECE7132AFAD11B122B40FF2BDC
:10518000F6D0DB00E2181671E650F1E7A02500200A
:1051900010B59AB0FFF768FFFFF7CEFF00231A00A3
:1051A0000A48D900415801334C1EA1415218FF2B27
:1051B000F7D1074901A807F07DFC01A801F010F81C
:1051C000044801F00DF81AB010BDC046A02500201B
:1051D000DFE60000F3E600008022F0B55200A1B047
:1051E0000021684807F022F9802200215200664819
:1051F00007F01CF9654BFF271B681A000493534204
:105200005A4110000592FFF701FE049C0020631E26
:105210009C415F4B64421C405E4BE418FFF778FFF3
:105220000600002E2FD10498FFF700FE411C0598C0
:10523000FFF720FE059A554B574D1A602C60FFF77B
:105240007BFFFEF7BDFC514B64201B68A0215A4236
:1052500053414F4A5B421340B0222C6892029B1884
:10526000E41A6043490204F09DFFA02252020300A9
:1052700000924A49220007A807F01CFC07A800F08A
:10528000AFFF21B0F0BD3268131412123A403B4018
:1052900003921A000A3A092A49D83A4B039A995CB0
:1052A000002931D110223E4807F0C0F835002B68A4
:1052B00003991A123A40914209D11A143A400B2A22
:1052C00027D0132A2DD00A2A01D1354B1D60280082
:1052D000FFF712FE051EEAD1314B196800290FD0E5
:1052E0002000FFF7FDFD04002D4B5B1959680029D4
:1052F00003D02000FFF7F4FD040004350C2DF3D19A
:10530000204B0121039A99543000FFF7F5FD060068
:1053100087E73B40022BDADC214A9B00D3185D6013
:10532000D5E7102200211E4807F080F8CFE71A00C9
:10533000153A082AE8D8144A0399525C002AE3D1A6
:105340003500152B00D01500300003681A143A40C0
:10535000152A0FD01D2A00D10025FFF7CDFD00280A
:10536000F3D1002D04D020002900FFF7B9FD04007F
:10537000054BC6E7039A1B123B409A42EDD105004C
:10538000EBE7C046041000200C110020041100209F
:1053900000C0FEFF04C002000811002039E6000032
:1053A000282F002010B5FFF717FF10BDF0B585B00E
:1053B000039203220333DC17294D1440E4182B68B1
:1053C000284F5A42534180225B42D202A4103B40F4
:1053D0009B18A21C0291244E91000091019031680B
:1053E00000980A18934215D2FFF7F6FE2B685A422E
:1053F000534180225B421F40D202BF183368009A9B
:105400009B189F4206D2194800F0EAFE00252800AA
:1054100005B0F0BD029B356819066B461A7BA423C4
:10542000DB051343FF222F00090C1943019B1204D3
:105430001B04134019432800FFF70AFD0837281DF5
:1054400021003760FFF704FD002C04D00A9A2100E8
:105450003800FFF723FD009B083BFF183760D6E7B5
:105460000411002000C0FEFF0811002013E6000018
:105470000021094B094A59600131516059680029DE
:10548000FCD000211961012393600222044B813179
:10549000FF315A501A607047FC1000400010004065
:1054A00000E100E00222064B0121DA670022054BF1
:1054B0005A61054A11615A69002AFCD07047C046FA
:1054C00004E100E0FC1000400010004010B5044C66
:1054D0002378002B01D0FFF7E5FF0020207010BDDE
:1054E0000D120020802301205B055B6E5B001843DA
:1054F000704700000120024B1B685B001843704797
:10550000901200200120024B1B685B00184370477B
:10551000240000200120024B1B685B0018437047E9
:105520009412002070B504000D001600FEF74EF92D
:10553000802301215B055A6E26700026530061709E
:10554000E1706272010A5A0A6071A171A272010CC3
:105550005A0C000E5B0EA6702571E1712072E2728A
:10556000237370BD10B5044C200007F0E9FA010068
:105570002000FEF7BBFD10BD991200200E4B10B5A8
:105580001B680E4C5A1C0FD00D4C002B0CD00D4C30
:10559000012B09D00C4C022B06D0094C042B03D054
:1055A0000A4C052B00D1074C200007F0C9FA010076
:1055B0002000FEF79BFD10BD2800002084E70000BE
:1055C00080DE00008FE7000087DE000089E7000032
:1055D00070B5214C2278002A3DD1204B01215A6020
:1055E0008022D20511605A68002AFCD000220720D0
:1055F0001B4B1C4901255A500439585008315A5048
:1056000019481A4958501A491A485A501A495A50B2
:10561000A622D2009D50082218495A5004315850F1
:10562000022017495850174917485850174804394D
:105630005850182016495850C12189005A50053930
:10564000FF395858921802435A501249124A995039
:10565000FFF70EFF257070BD0D120020FC0000400A
:10566000001000400C050000746962751C05000004
:1056700024050000200004022C0500001405000091
:10568000340500003C050000FFFF00002110010070
:10569000540500000E1200200405000070B50E4BEA
:1056A00006001B78002B01D1FFF792FF00200B4D65
:1056B0002C7884420ED00A4B202219780323091B30
:1056C0001940084B4901C918300006F093FE01202B
:1056D000013C2C7070BDC0460D12002098120020B5
:1056E0000C1200200E120020002370B588B09842E2
:1056F00035DD0D6801262C0034409C422FD123005B
:10570000042D2CD90F222B681A402300092A26D1F8
:105710006A683F2A23DD6846FFF7C0FF23000028A0
:105720001DD06B4619783300A14203DB6B461B5D2D
:105730005B003343A200AA1801349360202CF2D1FD
:10574000092169444A780B7812021A438B781B04AA
:105750001A43CB781B061343024A13600423180034
:1057600008B070BD9412002070B5454B8AB01B780C
:10577000002B01D1FFF72CFF02AC2000FFF78EFFBA
:10578000002802D100200AB070BD23780B2BF9D974
:105790006378012BF6D1E378012BF3D1002311209C
:1057A000384E394D33602B7068442379374A41783D
:1057B0001360027809021143827812041143C278FF
:1057C00012060A4332490A60002B0ED115216944A2
:1057D0004A780B7812021A438B781B041A43CB7851
:1057E0001B0613433360002318E0012B1AD1152147
:1057F00069444A780B7812021A438B781B041A43C7
:10580000CB781A211B06134333600E23627C694454
:10581000934200DD130000229A422CD10022042082
:10582000EA54B0E7022B03D1627B10331621EEE776
:10583000042B0DD1152108226944684606F0DAFDD3
:105840000098019903F064F806F086FC3060CAE71E
:10585000052BC8D1152108226944684606F0CAFD07
:105860000098019903F054F806F076FC3060627DF0
:105870000A231E21CBE7885CA8540132CCE7C0463E
:105880000D12002090120020991200202800002004
:105890009412002010B5134B04001B78002B01D18B
:1058A000FFF796FEFFF7FEFD00200F4A0F49104B51
:1058B000545058600130106058680028FCD0002017
:1058C00018610130906018690028FCD0094B0A4823
:1058D0001B785B011B185350FFF7E4FDFFF7C8FD71
:1058E00010BDC0460D12002000100040040500004D
:1058F000FC1000400C1200200E12002010B588B0E1
:1059000000281DDD0A68012113000B4018D1042A6C
:1059100016D90F2014682040092811D150683F285B
:105920000EDD9800101880680024084201D0401055
:10593000C4B26846C4540133202BF2D1FFF7AAFF4A
:10594000002008B010BD000010B5002813DD0C6861
:10595000E30710D56410532C0DD8084B1B78002B8F
:1059600001D1FFF735FEFFF79DFDA123044ADB00BF
:10597000D450FFF77DFD002010BDC0460D12002061
:105980000010004010B500280EDD0C68E3070BD5B1
:105990006410FF2C08D8054B1B78002B01D1FFF7B2
:1059A00017FE034A034BD450002010BD0D120020F7
:1059B000001000402405000013B5002814DD0C6819
:1059C000E30711D5094B64100093094B0193072C91
:1059D0000AD8084B1B78002B01D1FFF7F9FD6B4665
:1059E000054A1957054BD150002016BDE2ECF0F4E2
:1059F000F8FC00040D120020001000400C0500000F
:105A000070B588B0002820DD0124086804401CD14E
:105A100004281AD90F2302681340042B15D1FEF76E
:105A200045F9060007F08CF80500122800D9122568
:105A30002A0002210D326846FFF774FD6B465D7344
:105A4000A54205DC6846FFF725FF002008B070BDC1
:105A50002300325D6B449A730134F1E7F0B50D0019
:105A60008BB0012832DD08680122040014402DD1DA
:105A700004282BD90F2301680B40042B26D16B6817
:105A8000134223D0FEF712F96E68070073100193DA
:105A900007F056F805000E2800D90E252A0001212E
:105AA000113202A8FFF73EFD6A46127902AB5A7323
:105AB00002AA73129373019B76141B0ED673137490
:105AC0005574A54205DC02A8FFF7E4FE00200BB0E8
:105AD000F0BD3A5D02A963189A740134F1E730B55C
:105AE00089B0002814DD0C68E30711D51022684640
:105AF0000021FFF717FD6B466A4665105D73684627
:105B000063122D0E64149373D4731574FFF7C2FEE1
:105B1000002009B030BD0000174B184A5968002911
:105B200003D00021596001319160196900291FD00B
:105B3000002018618023DB00D3581149012B18D1B4
:105B4000A923DB00D3585B420B600E490B78032B73
:105B500001D801330B7003200B490B78013303404C
:105B60000B700A495B015B1809495350012393608C
:105B700070470860FAE7C046FC1000400010004083
:105B800024000020981200200C1200200E12002089
:105B90000405000010B5034A1021034800F090F8F6
:105BA00010BDC04604E70000FBE60000044A0549BA
:105BB0001368C85401339B059B0D13607047C046A2
:105BC000C8160020C812002070B5114C114A236875
:105BD000834202DC0023236016E0155C411C2E008A
:105BE000FA3E012E05D899420FDA555C013D1F2D72
:105BF00001D90800ECE70100151A565C6E5401311A
:105C00008B42FADC181A206070BD1570FAE7C046A6
:105C1000D41A0020D416002010B5FDF7CDFD064B98
:105C20001A68824201D900221A601B68C31A03480D
:105C300098428041404210BDC4120020204E000016
:105C400010B5094C094A23681268934200D110BD6F
:105C5000074AD05CFDF7ACFF0028F8D02368013379
:105C60009B059B0D2360ECE7CC160020C816002096
:105C7000C812002010B50400064B074A1B681268C2
:105C80009B1ADB439B059B0DA34200DB10BDFFF776
:105C9000D7FFF1E7C8160020CC16002070B5FFF73B
:105CA00037FAFF250400002801D1200070BD0368E9
:105CB0001B142B401D2B00D10400FFF71DF9F2E748
:105CC00070B5074E33680B2B08DC0C255D43054C83
:105CD0000133285164196160A260336070BDC04611
:105CE000D0160020382F0020F0B5B7B0040006F021
:105CF00027FF012802D8002037B0F0BD23785B2BA6
:105D0000F9D1013825182B785D2BF4D101343A21D3
:105D1000200006F0FDFE061EEDD0071B002FEADD79
:105D2000210000243A0004A806F022FF04AB711CF5
:105D3000DC556F1AA742DEDD1DAD3A00280006F0E3
:105D400017FF134BEC551B6803950193019BA3426E
:105D5000D1DD0C2666430F4B04A9F618306806F017
:105D6000E5FE051E05D17368B6680293029B9D424D
:105D700001DB0134EAE73068039906F0D7FE37000B
:105D80000836002801D17868B6E70135EEE7C0464D
:105D9000D0160020382F002010B5FBF7EDFAFFF7E2
:105DA0000BF8FBF711FBFDF797FEFEF74FFBFEF735
:105DB000CFFBFFF7EFFE01F043F801F02BFC01F001
:105DC00057FC01F0A1FE10BD962210B51201002172
:105DD000034806F02BFB0022024B1A6010BDC046A0
:105DE000401C0020D805002070B514007F22174BFE
:105DF000C000C0580D00836813401C2B01D0002048
:105E000070BDC368190011400429F8D101690A4026
:105E1000192AF4D11B0A01339B000C30C018FDF77E
:105E200045FF037806000120002BE9D0300006F082
:105E300087FE0023A042E2D1A34201DB0120DFE77D
:105E4000F15CEA5C9142DAD10133F5E7A02500204C
:105E5000064B074A1B6812689B1ADB439B059B0D88
:105E60000122834200DC002210007047C816002087
:105E7000CC160020F8B505000C0016001F1E0ED130
:105E80000320FFF7E5FF002808D0FA20FFF78EFE79
:105E9000E8B2FFF78BFEE0B2FFF788FEF8BD501DB9
:105EA000FFF7D6FF0028F9D0FB20FFF77FFEE8B20E
:105EB000FFF77CFEE0B2FFF779FEF0B2FFF776FE67
:105EC0003012C0B2FFF772FE3C00E31B9E42E5DDDC
:105ED0002078FFF76BFE0134F7E7000070B500246F
:105EE000F0250B4B1B68A34202DCFFF76DFF70BD72
:105EF0002B006343074A9B181A78002A05D059786B
:105F0000002311201A00FFF7B5FF0134E9E7C0466E
:105F1000D8050020401C0020F8B507000024F0251B
:105F20002B0063430C4A01349E18B74211D03178DC
:105F300000290BD00133D15C002311201A00FFF798
:105F400099FF2A000021300006F070FA0A2CE7D1F0
:105F5000F8BD024B1C60F9E7401C0020D80500206A
:105F6000F0B5150001222F007A4C1740A54401908E
:105F70000291002F11D005AB1A706A105A70120EE0
:105F80001A710522691299706D140299DD70FFF77C
:105F900071FFCF239B009D44F0BD042D2AD90F240F
:105FA00028680440042C32D1022304AA280013716B
:105FB000FDF77CFE050006F0C3FDC82302009B0030
:105FC000984200DD1A007C1C97420DD1984206D9F8
:105FD000614804AB03226149C01806F00BFA2200A5
:105FE00005AB02990198D2E72700611E695C05ACF8
:105FF000E155E8E7042D00D0A7E0032304AA043DFF
:1060000013716B425D4105AB55710222E9E7092C22
:106010007ED1042205AB1A706A685110009169465E
:10602000521209789A70009A59701F2A01DD2022B5
:1060300000926A46127806ACDA70009BBB4202DC22
:1060400005ABE21ACDE70126BB00EB1898680640C5
:1060500006D1042837D90F210368194002290CD131
:10606000012323704310637042121B0E4014A27070
:10607000E070237105340137DFE7042921D10223C1
:106080002370FDF713FE039006F05AFDA31C0C28A5
:1060900009D86070864201D19C19ECE7039A925DA1
:1060A0009A550136F6E70C226270039A925D9A5572
:1060B0000136092EF9D12E23E372237363730E3454
:1060C000D9E7012907D103230438237043425841FB
:1060D00060700234CFE7092909D104232370436893
:1060E0005A1062705B12A370E6700434C3E7032990
:1060F0000BD1052323700068020992B2430F92006E
:106100000B40D31A63701B12EDE726700134B2E71F
:10611000032C00D03DE7052205AB01091A7089B2B6
:10612000420F890022408A1A11125A709970642A0B
:1061300000DD64220421DA70081F824201DC04328F
:106140004FE7685C58540131F6E7002D00D020E796
:1061500053E7C046C4FCFFFF22030000EADA000058
:1061600070B502000024F0210D4E08006043801934
:106170004578954203D001340A2CF6D170BDF02247
:10618000002106F053F9074A1368013BA34200D1EE
:106190001460002329001A001120FFF76BFEEDE7C1
:1061A000401C0020D805002010B5B2B002236A467A
:1061B0000400137006F0C4FCC72800D9C7200023D0
:1061C000984207DC421C6B46FE211420FFF752FE6A
:1061D00032B010BD694601335A1EA25CCA54EFE7C3
:1061E00030B5B3B002236A460500137006F0A8FC70
:1061F0000400C72800D9C72400239C420BDC2000E0
:106200003230FFF737FD621C6B46FF211420FFF789
:1062100031FE33B030BD694601335A1EAA5CCA5400
:10622000EBE70000F0B5BDB005900C00012803DCE1
:106230001B20FBF767FA55E02C4B08680393C30754
:1062400009D4042807D90F2302681340042B02D174
:10625000FDF72CFD0390254B60680493C30709D418
:10626000042807D90F2302681340042B02D1FDF73D
:106270001DFD049000261E4B1B680893089BB3422B
:106280000BDC049B1B4A0093C821039B0AA806F061
:10629000DFFB0AA8FFF7A4FFCAE70C257543164BDE
:1062A0000399ED18286806F041FC071E05D16B68BC
:1062B000AD680993099B9F4201DB0136DEE7286840
:1062C0000499079506F032FC0835069000280BD19A
:1062D00021000598079B08315B6802389847074BF7
:1062E000069A1A603DB0F0BD0137E3E701E0000017
:1062F000D016002060E80000382F0020E40F0020B6
:10630000F7B5234B06001B68F02100930023009A89
:106310009A4211DC0024F0231A0062430192019991
:106320001C4A55182F78002F12D001340A2CF3D1B3
:106330001948FFF755FF29E00A005A43154882180B
:106340005078B04202D11278002A1FD10133DEE723
:10635000F0223900280006F069F802230D4A01995D
:10636000EB6053540D4AF1008A58009B6E70AE707A
:10637000AA602F616F61A34202DC054B01341C60EF
:10638000002331001A001020FFF774FDF7BDC0464E
:10639000D8050020401C0020A9EC0000A02500200A
:1063A00010B5FFF79BFDFF24084AE3005B429B18F2
:1063B000074AD35C043B012B03D8E043C0B2FFF78C
:1063C0009FFF013C002CEFD110BDC046FC07000030
:1063D000A0250020F8B505000E00FDF787FEFF247C
:1063E0000D4B18600D4AE3005B429B180C4AD35CCE
:1063F000062B01D0032B0BD1E743FFB2320029005B
:106400003800FFF7F1FC002802D03800FFF778FFD2
:10641000013C002CE6D1F8BD08000020FC0700007C
:10642000A025002070B50500FF24084AE3005B4268
:106430009B18074AD35CAB4203D1E043C0B2FFF7DD
:106440005FFF013C002CF0D170BDC046FC0700008E
:10645000A0250020F7B5FDF7AFF9574B1A68824227
:1064600001D900221A601A685449821A8A420DD949
:10647000FF2253491860D3005248CB1A1B181B78CF
:10648000073B022B0CD9013A002AF4D1F7BD0720B3
:10649000FFF7C8FF4C4B27E00820FFF7C3FF38E0A9
:1064A000FDF794F9071E00D101270020FDF742FAFD
:1064B00001900020FDF752FA019B0090434C444D9F
:1064C000002B12D02368002B6ED12B682760002B85
:1064D0006ED0404B01261B78002BD8D10920FFF746
:1064E000A1FF394B1E703B4B1E70009B002B12D03E
:1064F0002B68002B0FD123682F60002B1ED0324B4E
:1065000001261B78002BC7D10920FFF78BFF2E4BEC
:106510001E70304B1E702368002B0FD02A4E32782D
:10652000002A0BD19F4200D227602368FB1A312B2F
:1065300004D90720FFF776FF012333702B68002B67
:106540000FD0244E3278002A0BD1BB4200D92F60E5
:106550002B68FF1A312F04D90820FFF763FF0123AE
:1065600033702368002B0CD0019B002B09D1164EF1
:106570003378002B02D10720FFF754FF002323605C
:1065800033702B68002B00D180E7009B002B00D0DC
:106590007CE7104C2378002B02D10820FFF742FF44
:1065A00000232B60237071E7009A002AA0D1B5E781
:1065B000009B002B9FD1AEE7C01200200F270000E8
:1065C000A0250020FC070000B4120020B01200201B
:1065D000B8120020BC12002037B500240500FFF7D8
:1065E0007DFC01A80194FDF78DF921002000FEF744
:1065F00097F8FEF78BFAFDF7C5F9FDF749FAFDF7B5
:1066000063FAFEF7CFFBFDF705F9A54204D0FDF7CD
:10661000F9FA0248FFF7E4FD37BDC0469AEC0000E6
:10662000002310B501001A001120FFF723FC10BD54
:1066300007B56B46197069465A7013128B701314A4
:10664000120ECB700A716B46010005221320FFF772
:1066500011FC07BD10B50A0001001220FFF780FCF5
:1066600010BD70B505000C00FDF7BEF8002809D07C
:1066700020003230FFF7FEFA2B00220000211B2001
:10668000FFF7F8FB70BD10B50C00030011001420DB
:106690002200FFF7EFFB10BD012370B5FF24084A6D
:1066A00041185B42884201D3D84370BD06781D0A69
:1066B000234073409B009B5801306B40F2E7C0467B
:1066C0007CE8000013B50400FE2813D80A4BC20072
:1066D000D05800280ED0436808309900FFF7DCFF3F
:1066E00001900920FFF7C6FA01AB04222100172010
:1066F000FFF7C0FB13BDC046A0250020F7B50190F1
:10670000FFF7CCFA01250400FF276D42002C01D1D0
:106710002800FEBD266833143B40152B0DD1210007
:106720000198083106F002FA002801D135123D40E7
:106730002000FEF7E1FB0400E8E71D2BF8D101255E
:106740006D42F5E7F0B58027A1B0FFF779FAB84CB4
:10675000B84D2068FF00391A4019FDF70FFA236879
:106760000600C3182360002B0ED121B0F0BD2068B5
:10677000391A2818FDF702FA236806001B1823604F
:10678000FDF71AF8AC4B1860002EF0DC2B78FA2BD2
:1067900000D014E12368022B07DCFFF73DFA002844
:1067A000E3D00120FFF710FADFE76B78AC78981E92
:1067B000182800D9F8E003F061FC0D2024282B34C0
:1067C000F73E707A7E94D3E4F7F7F7F7F7F7F7F729
:1067D000F7F7F200FF2C0ED02000FFF7C1FC0022DB
:1067E000964BE100CA505B181A7121000092130009
:1067F0001320FEF7DBFD0320D4E72000FFF780FD28
:10680000F9E72000FFF7ACFCF5E7FFF7C9FDF2E779
:10681000FFF764FB0020FFF7DFFE8948FFF7E0FC8D
:10682000E9E7632CE7D8874BA200D2582100152056
:10683000FFF796FBDFE7FFF731FAFF270400002C94
:10684000D9D025682B143B40152B04D02000FEF72F
:1068500053FB0400F3E72000083006F071F906004E
:106860000530FFF707FAFB20FFF7A0F92D121D20D6
:10687000FFF79CF9E8B2FFF799F9F0B2FFF796F944
:106880003012C0B2FFF792F925002B1B9E42DDDDCE
:10689000287AFFF78BF90135F7E700211D200091D9
:1068A0000B000A00FEF782FDFDF7ACF9A3E720001C
:1068B000FFF708FF9FE7FCF799FF07AC624A6421E6
:1068C0000090624B200006F0C3F8022320002370E2
:1068D00006F036F92300020000211620FFF7CAFA5D
:1068E00089E75B4BFA21186803F05CFC00260490F2
:1068F000524AF3009B181C68002C28D01B79059382
:10690000636808349F00B81D0393FFF7B3F9FB20B9
:10691000FFF74CF901207D1CFFF748F9F0B2FFF7B3
:1069200045F9E8B22D12FFF741F9E8B2FFF73EF959
:106930000598FFF73BF9E719A7420CD8FFF780F954
:10694000049B0398584301F087FDFFF779F901365E
:10695000FF2ECDD14FE72078FFF728F90134EBE780
:106960000024FFF7BBFA2200210000942300DA2064
:10697000FEF71CFDFF222100D200304805F056FD35
:1069800092E7012C02D1FEF7E1FA34E7022C02D1A2
:10699000FEF708FD2FE70120FFF71EFE2BE700237F
:1069A00021001A001A2099E71A00C83A052A00D9CE
:1069B00021E7002218001100FAF712FD1BE7FB2B5C
:1069C00000D0EEE62268042A00DCE6E62E79E878BC
:1069D000204B360206439E4200DDE2E6331D9A421A
:1069E00000DCDAE6EB5CFE2B00D0DAE66878AC7807
:1069F000771E1B2800D17FE030D8072865D00828F3
:106A00003AD001282FD1FF2C10D02000FFF7A8FB8F
:106A10006D79114AB31E009221002A000A20FEF768
:106A2000C5FC064BE400E0501B191D71701DB9E652
:106A3000D41A0020D4160020C4120020A025002063
:106A40007CEC0000982D002093EC00008EEC000000
:106A500004000020F6030000DA1600201D285DD097
:106A60004FD31E2871D00300C83B052BDED8404A07
:106A70003900FAF7B5FCD9E7632CD7D86A79022A2E
:106A800013D0032A1BD0012AD0D1E979AB790902AE
:106A900019432B7AA4001B0419436B7A1B060B4382
:106AA0005B001343334AA350C0E7002FBEDDB11E85
:106AB0003148FDF71BFB2F4BA400E050B6E7AB7944
:106AC000A4005A1E93419B00ECE7632FAEDC07AD98
:106AD0003A002749280005F08DFC00232800EB55DB
:106AE000FFF70CFE0028A1DB224B8000C2582100DA
:106AF0001520FFF735FA99E739001D48FFF76AFCC2
:106B000094E7FF2C92D06A79022A8FD81A490B2079
:106B100000912100B31EFEF749FC87E7632F00DDDB
:106B20006327002307A99F420ADCFB430022DB17EF
:106B30003B40CB181A70152000917B1C2100EAE71E
:106B4000EA185279CA540133EDE7012C00D06DE701
:106B5000002F00DC6AE76B79002B03D01C00322B7E
:106B600000DD322464235C43044B1C605EE7C046B6
:106B7000D9160020982D0020DA16002004000020ED
:106B80000120704710B5064C200001F0D1F80549EE
:106B9000200001F001F90122034B1A6010BDC0462C
:106BA000101B0020801A0600D81A00201FB50021F3
:106BB0001020FCF721FE01211120FCF71DFE012110
:106BC0001620FCF719FE1C4C200001F00FF81B4B9F
:106BD0001B4A1B6812681B49D2B28B420BD8802318
:106BE0009B04019301AB1A710199029A00232000C2
:106BF00001F018F81FBD14498B4202D88023DB0432
:106C0000EFE712498B4202D880231B05E9E71049C0
:106C10008B4202D880235B05E3E70E498B4202D802
:106C200080239B05DDE70C498B4202D88023DB05DE
:106C3000D7E780231B06D4E7F01A0020300000209D
:106C40002C00002048E8010090D0030020A107009C
:106C500040420F0080841E0000093D0010B500284E
:106C600015DD01240B68234211D023410C4A136027
:106C70000C4AA04209D04B68234206D02341022B84
:106C800009D0032B09D0A34203D0022313600020B4
:106C900010BD0023FAE70323F8E71460F7E7C046C6
:106CA000300000202C000020F8B50125086828429B
:106CB00003D10D20FAF726FDF8BD4010FCF7C0FD0A
:106CC000041E2DDBFCF796FDA04229DB00212000ED
:106CD000FCF792FDFA222900D200200001F0EEFB21
:106CE00000281DD0002500270726FA220121920046
:106CF000200001F0E3FB002812D0282802DD012348
:106D0000B3401F43013EF0D20D4EAF550135052D66
:106D1000E9D1012206210920FDF76AF9002801D1F5
:106D20000020C9E70B23012443600023F25C990093
:106D300052004118224301338A60052BF6D1BBE78C
:106D4000DC1A002070B500281EDD0D68EB071BD48F
:106D5000042D19D90F242B681C40032C14D11A09B7
:106D600092B25B0F92001C40141B2E00FFF71EFF17
:106D7000731B06489C4205DD317900F059FF01364E
:106D8000F070F5E700F053FF002070BDF01A00200E
:106D900010B504680D20E30703D56410FF2C03D958
:106DA0001720FAF7AFFC10BDFFF700FFE1B2044C6B
:106DB000200000F03DFF200000F039FF0020F2E746
:106DC000F01A002070B5FFF7F1FE064D00212800F3
:106DD00000F02EFF0400280000F029FF01206400CD
:106DE000204370BDF01A0020A02101220B4BC900E6
:106DF0005A500B480B4958500B491A604A68002AF0
:106E0000FCD000224A60A121C900585801215960D4
:106E1000A021C9005A50054BC018704700700040AF
:106E20006A10000004050000FC700040FBFDFFFF3D
:106E300010B5FFF7D9FF43000120184310BD000033
:106E400010B5034A0E210348FEF73AFF10BDC046B5
:106E5000C0EC000030ED00000D4B70B51B68040065
:106E60000E001500002B01D1FFF78CFEE1B2094C9A
:106E7000200001F028F8F1B2200000F025FFE9B26F
:106E8000200000F021FF200001F088F870BDC0460E
:106E9000D81A0020101B002010B5012403682342DB
:106EA00005D04168214202D08268224203D10D20E0
:106EB000FAF728FC10BD5810802801D91520F7E7F3
:106EC0004910FF2901D91620F2E75210FF2A01D9F3
:106ED0001720EDE7FFF7C0FF0020EBE710B5002813
:106EE00003DC1C20FAF70EFC10BD0B68DA0701D496
:106EF0000D20F7E75B100322012B06DD0522022B94
:106F000003D00C22042B00DC08220F211820FFF7ED
:106F1000A3FF022001F0A0FA0020E5E7F7B5012267
:106F20001400904226DD0D682A4223D02D4B1541D6
:106F30001B684C68002B01D1FFF724FE2A4EE9B2F2
:106F4000300000F0C0FF27000122174014D0144188
:106F5000FF2C02D91720FAF7D5FBE1B2300000F080
:106F6000B3FE300001F01AF80024A04202D0232022
:106F7000FAF7C8FB2000FEBD042CF2D90F252368C8
:106F80001D40092D1CD1636801925B100093009B8A
:106F9000BB42E6DDBB00E3189D68019B1D420BD0A0
:106FA0006D10FF2D02D91720FAF7ACFBE9B23000C3
:106FB00000F08AFE0137EAE71720FAF7A3FBF9E7AA
:106FC000032DCED127001A0992B25B0F92001D400B
:106FD000551B3B1B9D42C4DD3979300000F074FE27
:106FE0000137F6E7D81A0020101B0020154B70B5AA
:106FF0001B6805000E00002B01D1FFF7C3FD124CEA
:10700000EDB22900200000F05EFFF1B2200000F098
:107010005BFE0021200000F061FF002801D040420B
:1070200070BD72B601222900200000F047FF62B651
:10703000200000F03AFE0028F2D0200000F03AFED6
:10704000EEE7C046D81A0020101B002010B501241E
:107050000368234202D04168214203D10D20FAF790
:1070600051FB10BD5810802801D91520F7E74910B1
:10707000FF2901D91620F2E7FFF7B8FF40002043AF
:10708000EFE7000070B5284D04002B68002B08D1F5
:1070900005211820FFF7AAFF022001F0DDF90123E6
:1070A0002B60012C14D105211820FFF79FFF7F28AA
:1070B0002BDC03007F3301DA7F204042C8235B4290
:1070C00058437F2103F06EF8052C00D1404270BD7B
:1070D000032C11D121001820FFF788FF7F2814DC32
:1070E00003007F3301DA7F204042C8235B425843CC
:1070F0007F2103F057F8EAE70020052CF5D107219E
:107100001830FFF773FF7F2802DD0138FF38D0E722
:1071100003007F3301DA7F204042C8235B4258439B
:107120007F2103F03FF8D1E7E41A002010B50120D9
:10713000FFF7A8FF43000120184310BD10B503203E
:10714000FFF7A0FF43000120184310BD10B5052034
:10715000FFF798FF43000120184310BD10B5082128
:107160001820FFF743FF0300C00FC0180123401091
:1071700015304000184310BD414B70B51B68050029
:10718000002B01D1FFF7FEFC3E4C23787F2B00D86B
:1071900072E007210E20FFF729FFC42833D1012216
:1071A0000E26394B10211A70384B30001A70267099
:1071B000FFF752FE802211213000FFF74DFE002123
:1071C000615600291EDB324EC9B2300000F07BFE52
:1071D0002D4B3000197800F077FD300000F0DEFE16
:1071E00021780622300000F069FEAC1D300000F06E
:1071F0005CFD002806D0300000F05CFD28700135F1
:10720000A542F3D170BD0F211920FFF7EFFE3328FF
:107210000FD168221C4B1E261A7000221B4B6021C6
:107220001A7030000C322670FFF716FE0222612120
:10723000C2E700211820FFF7D9FEFA28BFD1422269
:10724000114B10261A700022104B4B211A7030007F
:1072500001322670FFF700FE042001F0FDF838220D
:107260004C213000FFF7F8FD0F2251213000FFF7CD
:10727000F3FD1B2252219FE700216156A3E7C04680
:10728000D81A0020340000203600002035000020ED
:10729000101B002073B5002606220021684605F069
:1072A000C5F86846FFF768FFFFF74CFA1A4B6A46C5
:1072B0009E576C466B4691781878D5785B78127932
:1072C0006479002E1FD000020902034329431BB238
:1072D00009B2120211482243007812B240B21028BB
:1072E00002D15210DB10C910D8171B184340C81721
:1072F0000918414001205918D317D2185A408A184A
:107300005200104376BD1B022D02034329431BB2DA
:1073100009B22402DEE7C046350000203400002018
:10732000F8B501231C0098422BDD0F683B4228D0A2
:107330004E6835001D4024D1042E22D90F22316819
:107340000A40092A1DD173685C10202C00DD20241E
:10735000144B1B68002B01D1FFF714FC72B67F1091
:10736000F9B2114F2200380000F0A8FD62B6A54224
:1073700014DA380000F099FC002804D101246D00D3
:107380002C432000F8BD380000F094FC0122AB0033
:107390004000F31810439860AD18E8E76400012539
:1073A000EEE7C046D81A0020101B002070B52B4B0A
:1073B00086B01B68002B02D10120FFF763FE01ADF0
:1073C00014220021280005F031F8254E1821300044
:1073D00000F079FD0321300000F076FC0021300040
:1073E00000F07CFD041E13D172B605221821300076
:1073F00000F064FD62B6300000F057FC002802D0B7
:10740000300000F057FCA3000134E850052CF2D105
:10741000019B7F2B01DD013BFF3BAA687F2A01DD39
:10742000013AFF3A29697F2901DD0139FF39C82076
:10743000434342434843DB11D2115243C0115B43E3
:1074400040439B18181804F0BDFE01F091FB04F0B6
:1074500083FE43000120184306B070BDE41A0020EB
:10746000101B002010B5054C2368002B02D01B20F8
:10747000FAF748F90020206010BDC046E81A002045
:1074800010B5002803DC1C20FAF73CF910BD0B688E
:10749000DA0706D4042B04D90F221B681340032BF0
:1074A00001D02420F0E7034B25201B68002BEBD0F4
:1074B0001B20E9E7E81A002010B5002803DC1C2097
:1074C000FAF720F910BD0B68DB0701D40D20F7E7B0
:1074D0001B20FAF717F90020F4E700001D4B70B5E8
:1074E0001B680C00002B03D12520FAF70BF970BDA7
:1074F000012801DC1C20F8E708680121084207D1B7
:10750000042805D90F2302681340DD1E8D4201D9DE
:107510002420EAE765680D4201D11120E5E7042B3C
:107520000BD1FCF7C3FB05F00BFB63685B10013B61
:1075300001D4834208DB1220D7E7100980B2520041
:107540008000920F801AF0E71B20FAF7DBF8012089
:10755000CDE7C046E81A002010B50400802803DDFE
:107560002620FAF7CFF810BD002CFCDD1B20FAF71F
:10757000C9F8FEF76FFFFFF7E5F8012000F06CFF98
:10758000F2E7000010B5002805DC1C20FAF7BAF875
:107590000400200010BD184B1B68002B01D12520D2
:1075A000F4E70124086804400FD04010FF2801D9F7
:1075B0002820EBE71B20FAF7A5F8FEF74BFFFFF7B3
:1075C000C1F8012000F048FFF4E70428E1D90F21B9
:1075D00002681140042906D1FCF768FB05F0B0FAF7
:1075E000FFF7BAFFD5E70329D3D1100980B2520FB4
:1075F00080000A40801AF3E7E81A0020044B10B517
:107600001B682520002B00D01B20FAF77BF810BD4B
:10761000E81A002010B5034A06210348FEF750FB84
:1076200010BDC046CCED0000FCED0000002070470E
:1076300001207047002070470020704700207047ED
:1076400001207047002070470020704700207047DD
:1076500000207047002070470020704700207047CE
:107660000020704700207047704770477047000047
:1076700010B5034A0F210348FEF722FB10BDC04698
:1076800024EE00009CEE00000378013B1F2B00D984
:1076900070470130F8E710B5FFF7F6FF0378002BCD
:1076A0000BD00130222B11D10378002B03D0421CC8
:1076B000222B03D11000FFF7E7FF10BD5C2B03D195
:1076C0004378002B00D0821C1000EDE73A2BF2D05B
:1076D0002C2BF0D07B2B0BD1FFF7D6FF0378002BA0
:1076E000E9D07D2B01D10130E5E7FFF7D4FFF5E7C5
:1076F00020225B2B14D1FFF7C7FF0378002BDAD0D1
:107700005D2BF0D0FFF7C7FFF7E7202BD3DD2C2B45
:10771000D3D0190091435D29CFD0222BCDD0013099
:107720000378002BF1D1C6E7002210B5904216D0A5
:10773000FFF7AAFF03780422222B10D0023A7B2BFA
:107740000DD0013A5B2B0AD01900303902320929D9
:1077500005D92D2B05D14178303909290AD81000D7
:1077600010BD0522742BFAD00132662BF7D00132FE
:107770006E2BF4D0581E83415A42F0E770B5FFF7E4
:1077800083FF037801222D2B01D18018023A0023B8
:107790000A2502E06B430130CB1801783039CCB2B6
:1077A000092CF7D95A43100070BDF8B50C0015002C
:1077B000FFF76AFF0378222B02D000232370F8BD65
:1077C0000D236A1E210008250C260A279C4601303D
:1077D0000378222B02D100230B70F0E7002BFAD0A4
:1077E000441C5C2B0BD14378841C622B0ED0662B7F
:1077F0000ED06E2B0ED0722B0ED0742B0ED0002A12
:10780000E9DD0B70013A01312000E1E72B00F6E7DA
:107810003300F4E73B00F2E76346F0E70923EEE7C5
:1078200010B50400FFF737FFA04203D90378013BEE
:107830001F2B00D910BD0138F6E710B5002815D070
:107840000378002B13D0FFF71FFF202103780200DD
:107850008B4300205D2B09D01000FFF71CFF03783D
:107860002C3B5A425341C018FFF70EFF10BD1800C1
:10787000FCE70300002070B50C0081420EDD1A7891
:107880005B2A0BD1581CFFF7FFFE0125AC4205D047
:10789000FFF7D3FF002801D00135F7E770BD70B5C1
:1078A0000C001500002901D000230B70002820D007
:1078B0000378002B1ED0FFF7E7FE037806002C2B81
:1078C00003D10130FFF7E0FE0600337800207D2B66
:1078D0000FD0844204D02A0021003000FFF765FF5A
:1078E0003000FFF7D8FE03783A2B02D10130FFF7C2
:1078F000CBFE70BD1800FCE7F0B50D0004009DB094
:107900002E78002E35D02E21280005F001F9071E13
:1079100014D0431B0193303E092E14D82800FFF7E2
:107920002DFF01002000FFF7A4FF0400002C20D051
:10793000002F1ED0019B0133ED18E1E7280005F070
:10794000FFF80190E7E723787B2B11D1601C6422BC
:1079500003A9FFF7A4FF041E0BD0019A290003A876
:1079600005F0F5F80028E1D02000FFF794FEEEE7DF
:10797000002420001DB0F0BD70B5050000200C00F3
:1079800081421DDD2800FFF7CFFE0300681C012B9C
:1079900014D00020022B13D10022681C1100FFF725
:1079A0007EFF012C0CD0FFF748FF00221100FFF7EB
:1079B00076FF013CF5E7FFF740FF013C012CFAD1CF
:1079C00070BDF8B5050000200C0016001F008142B4
:1079D0000DDD2800FFF7A8FE03000020022B06D1D2
:1079E000681C3A003100FFF75AFF012C00D1F8BDA6
:1079F000FFF723FF3A003100FFF751FF013CF4E7A6
:107A000010B50024A04218D0FFF73EFE03787B2B70
:107A10000AD1013000221100FFF741FF00280CD0ED
:107A2000FFF739FE0134F5E75B2B06D10130FFF794
:107A300004FF002801D00134F9E7200010BDF8B59B
:107A4000002816DD0D68EB0713D56D10013D0124EC
:107A5000FDF75EFB0026FF27644200280CD1002EB4
:107A600021D0300005F06CF801003000FCF73EFB3F
:107A7000F8BD01256D42EAE703681A143A40152A59
:107A80000BD11B123B409C4200DA1C009D4201D1ED
:107A900006000836FDF730FADFE71D2AFAD1012487
:107AA00000266442F6E70120013464002043DFE74A
:107AB00010B508680C00FCF7F9F8FEF71FFE002867
:107AC00003DB6268024B8000C250002010BDC0463C
:107AD000982D002010B50868FCF7E8F8FEF70EFEB8
:107AE0000123002802DB024B8000C358180010BDA0
:107AF000982D002010B50868FCF7D8F8FEF7FEFDB9
:107B0000C043C00F800010BD10B5034A04210348D4
:107B1000FEF7D6F810BDC04638EF000032EF000087
:107B200010B5FBF7E5FFFCF793F8FEF735F90448CD
:107B3000FEF756FBFDF72CFBFEF732FC10BDC046EE
:107B400087EF000010B5FBF749FC10BD70B50025AC
:107B500004AC24780573A94205D10A4B0A4A2521B1
:107B60000A4804F0D9FB01600949920052589B0071
:107B700002715B58A40083716358856043710223CE
:107B8000C37170BD9FEF0000FEEF0000ADEF00007D
:107B90005CF00000037B002B04D14373837303610B
:107BA00001330373704700001FB50191A021002429
:107BB0000068C900D2B24450012A10D0A24209D0B4
:107BC000032A0AD0074A8350074B019AC250012367
:107BD00043501FBD02221343F4E70422FBE70622B1
:107BE000F9E7C046540500002405000010B5040064
:107BF000FFF7D0FFA1222368A179D20099506179C3
:107C0000064A20009950217904329950044B196892
:107C10005A689B68FFF7C8FF10BDC0460C050000FE
:107C2000041B00201FB5FFF7BFFF05B000BD704764
:107C30000368074A99501A00FC32D1680029FCD029
:107C4000A321C90058580023C0B2D3607047C04672
:107C50001C05000007B58022074BD2051A600022E0
:107C60009A6002321A7111230E32009303490533D0
:107C70000348FFF76BFF07BD041B002000300040E6
:107C8000F01A0020F8B505000E0017000024BC42D1
:107C900008D02B68315D1B6828009847002801D068
:107CA0000134F4E72000F8BD704710B51C3000F037
:107CB000AFF910BD10B51C3000F09CF910BD10B527
:107CC0001C3000F0ABF910BD70B5437E0D00002BE9
:107CD00001D1002070BD6430040000F0A8F9002834
:107CE000F7D12000290000F076F90120F2E700002A
:107CF000F7B50193FA23002504009B0083600B4B2A
:107D00004560083303601C300F00160000F058F97E
:107D10002000643000F054F96B461B7927616675CA
:107D20006576A5762000A375FEBDC0463CF0000038
:107D3000012330B5A024C375837D13499B005A5895
:107D4000437DC132114DFF32E40592009B005B5828
:107D50001551CC22C133FF339B001D5104690C4BDC
:107D60005204E25005220469243BE250837D0469F9
:107D70009B005A58A123DB00E250437D02699B001F
:107D80005958044BD15030BD5CF000000C06000087
:107D9000240500000C050000A022002310B5046992
:107DA000D200A3500A4CA1420FD90A4C8C425B412D
:107DB00009495B420B40CD21C9045B18046907499E
:107DC000635005210369995010BDCC235B04F5E78E
:107DD000A086010090D00300000098FD240500005B
:107DE000F7B5040000200D000193824265D0160013
:107DF000402A00D9402627001C37380000F0F6F84A
:107E0000B1232269DB00D550802201232169920031
:107E10008B50A27E002A03D122691362226913606B
:107E20000025731EAB4207D1019B002B04D080229A
:107E30000221236992009950012223691A62236961
:107E4000FC33DA68002A02D19A6A002AF9D09A6AC9
:107E5000002A0BD1DA60A3232269DB00D158380055
:107E6000C9B2013500F0B7F8B542DAD3019B2269F7
:107E7000002B0FD11300FC339B6A002B0AD1013376
:107E8000A376D3612369FC33DA6C002AFCD000228C
:107E9000DA640AE000230121A37651611A00236904
:107EA000FC3399680029FCD09A602369FC339A6AF4
:107EB000002A01D000229A62E8B2FEBD10B501236B
:107EC000FFF78EFF10BD0300AC3310B5040019702E
:107ED000643000F08BF80123637610BD00230200AC
:107EE00070B5AC3243760D001178B1220400006900
:107EF000D20081508022216992008B502269013387
:107F000013622269936026006436300000F080F826
:107F1000002812D0300000F06DF81E4B2269D050BE
:107F20002369FC331A6A002A02D19A6A002AF9D01E
:107F30009A6A002A01D11A62E5E723690122002D1D
:107F40000DD11900FC31896A002908D1DA61236951
:107F5000FC33DA6C002AFCD00022DA6407E05A61B4
:107F60002369FC339A68002AFCD000229A60002022
:107F70002369FC339A6A82420BD098622169064ACF
:107F80008B588B501800022B03D0181F431E9841AA
:107F9000033070BD1C050000C404000010B50121B1
:107FA000FFF79CFF10BD000010B5132312220249F9
:107FB0000248FFF79DFE10BD00400040101B00204E
:107FC00010B540220021040004F030FA0023200004
:107FD0002364636410BD10B53F24026C531C23401E
:107FE000446C9C4201D08154036410BD002303649F
:107FF00043647047436C026C934206D03F21C25CDD
:1080000001330B4043641000704701204042FBE7FE
:10801000036C406C181A00D540307047436C026CFA
:10802000934201D0C05C704701204042FBE73F22F1
:10803000036C406C01331340181A43425841C0B2DC
:108040007047000003210A4802680A430260094899
:1080500002680A4302600849084A094B9B1A03DD7B
:10806000043BC858D050FBDC00F012F8F8F74CF88D
:108070002405004054050040A0F500000000002049
:1080800070020020FEE7FEE7FEE7FEE7FEE7FEE700
:10809000014B024A1A607047380000200024F400A7
:1080A0000120704710B503681322DB69984710BDA3
:1080B00070470000054B0269D1500369FC331A6A0E
:1080C000002AFCD0002201201A6270471C05000023
:1080D000030010B55C331A781F231A401E3B1900A9
:1080E0009140114AD167C222042104699200A15033
:1080F000026953600269D360A02300220169DB009A
:10810000CA5001230169094A5B428B500169084A40
:108110008B5001690C3A8B50016908328B50143036
:10812000FFF764FF10BDC04604E100E00C0500004D
:108130001405000010B51430FFF76AFF10BD10B52C
:108140001430FFF76BFF10BD10B51430FFF752FF6E
:1081500010BD0000030070B55E331A780469724BDD
:10816000E25003005D331A780469704BE25003005B
:1081700061331C7802696E4B012C00D09EE0050033
:108180005F352E78A225ED00565102006032157839
:10819000A1220669D200B5500269D4509623DB00B3
:1081A000994200D88CE096231B01994200D88AE0BE
:1081B00096235B01994200D888E096239B0199425F
:1081C00000D885E0E1239B01994200D882E0962304
:1081D000DB01994200D880E0E123DB01994200D81D
:1081E0007DE096231B02994200D87AE0E1231B022E
:1081F000994200D877E096235B02994200D874E058
:10820000E1235B02994200D871E0E1239B0299428D
:1082100000D86EE0474B994200D86CE0E123DB02C6
:10822000994200D86AE0E122002312038A425B41AE
:10823000414A5B421340802252059B1801693F4A24
:108240008B50A02304220169DB00CA50002103697E
:10825000FC33D9600369FC331962012301690B60A7
:1082600001698B60C1210469890062501F215C3063
:1082700002780A4093406231314AFF315350002165
:10828000415600293CDA0F230B40083B2D4C9B083C
:108290009B001B1903242140A140FC348C40DD6964
:1082A000A5432C00C0258D4029002143D9611F23FF
:1082B000017819401E3B8B40136070BD00246CE7B1
:1082C0009E23DB02BAE79D231B03B7E71E4BB5E7EE
:1082D0001E4BB3E7EC239B03B0E71D4BAEE71D4BF2
:1082E000ACE71D4BAAE71D4BA8E71D4BA6E71D4BAE
:1082F000A4E71D4BA2E78023DB049FE71B4B9DE710
:108300008C080F4BA400E41803230B40FF21C02569
:10831000DB009940AD0066598E433100C0269E4077
:1083200033000B436351C2E70C0500001405000045
:108330006C05000090D0030000D0BEFE24050000B4
:1083400000E100E000ED00E000B013000050270065
:1083500000A04E0000F0750000509D0000F0EB0002
:1083600000903A0100E0D70100B0AF0300705F0752
:10837000F7B5009308AB1B7800250193FA2304009E
:108380009B0083600E4B45600833036014300F0080
:108390001600FFF715FE23005C3327611E70009B5B
:1083A000084A9B00995823005D331970019B2000F7
:1083B0009B009A5823005E33DD701A70FEBDC046E4
:1083C000D8F000005CF00000036910B51A00FC3220
:1083D000D2680400002A0AD0A322D200995814308F
:1083E000C9B2FFF7F8FD00222369FC33DA6010BD43
:1083F00010B50248FFF7E8FF10BDC046C81B0020BB
:108400001D2307B502220093024901330248FFF7FA
:10841000AFFF07BD00200040C81B002010B500289A
:1084200001D004F0BFFA10BD0849094A094B10B544
:108430001B688858FA22190A1B0618439200002369
:1084400001F0E8FF4904C00B084310BD00100140D3
:10845000040500002C1C002070B5041E09D0FFF795
:10846000E3FF050000F014F8FFF7DEFF401BA04219
:10847000F8D370BD0022044B9A60044A136801339C
:10848000DBB213607047C046FC1001402C1C00207A
:108490007047704710B500F05FF8FFF7FAFF012052
:1084A000FFF7DAFFFFF73CFBFFF74CFB024B002B1B
:1084B000FAD000E000BFF7E700000000F8B54C1E5E
:1084C000A1410125104B114F8000C3584C42386820
:1084D0000F499D40160001F0DBFD0A21704301F0B9
:1084E000D7FD2C400300220029000A4800F016F8AE
:1084F000FA21094C89004443386801F0C9FD0100A4
:10850000200001F0C5FDF8BD5CF00000380000203F
:1085100040420F00100500501027000030B50468DD
:108520000C40944206D1013B002BF8D112E0013BF4
:10853000002B0FD004680C409442F8D10024056849
:108540000D40954204D101349C42F8D1002002E054
:10855000201C00E0181C30BDC420114B80001A58AC
:1085600010491140C02212020A431A50C021802231
:10857000490092025A501A608023A3220021DB0591
:10858000D20099500122F9309A60074BFF30195000
:10859000C120023180001950403019501A607047D4
:1085A00000E100E0FF00FFFF00100140014B1860F8
:1085B0007047C04684000020F7B500231E285AD813
:1085C000384B8000C258042A5BD007D8022A54D006
:1085D00055D80423012A09D000234CE0062A54D0A0
:1085E00051D31A2A53D002231B2AF5D12E4A1168DF
:1085F00008294ED909294FD00A240226A020012596
:108600002A4AC00015502A482A4D07681C20BF007E
:1086100007402948019700685759009027481B02D6
:1086200007401F43C02300989B020340FF2057517F
:108630005759000207401F43019B1F43009B5801ED
:108640006023184007433E43565101251C4B1560DB
:1086500058680028FCD000205860A1230125DB00C9
:10866000D3585560A025ED0050511BB2A14202D055
:1086700015D2611ACB401800FEBD0823B6E71023BF
:10868000B4E72023B2E74023B0E78023AEE701231D
:10869000ACE708240026B1E70C000126AEE7091B71
:1086A0008B40E8E75CF00000800000200070004094
:1086B0003C0000200405000040000020FF00FFFFF8
:1086C000FC700040F0B51E285BD8364B8000C258C5
:1086D000354B1E68002E30D1C227344BBF00D8590D
:1086E000334C03250440C02000022043D851C0244D
:1086F00080206400800018512E4F18602E4B803C63
:10870000D859FF3CA043D8510437D859A843204337
:10871000D8510837D8590C35A843844607206546F8
:108720002843D851A820C0001E50C12080268000B8
:1087300076021E501C601C4B1C60142500202B0070
:108740001E4C2E0046433659771C1BD14343E25042
:10875000A0230325C132FF329200DB05D550184B10
:108760001A68082A14D114234343E3189A6812485C
:108770005132FF32920059601150DA68C1239B00D8
:10878000C250F0BD9642E1D001300328D9D1F8E7BC
:10879000082A02D9083AD140E5E708239A1A9140FD
:1087A000E1E7C0465CF00000301C002000E100E082
:1087B000FF00FFFF0405000000900040440000207F
:1087C000840000202149F0B54A6C2148002A14D0C9
:1087D000A025A12600230124ED05F600C258571C50
:1087E00006D0C7187F68002F02D027009740AF51EE
:1087F00014333C2BF2D100234B64A0230121DB0571
:1088000000260F009C4614234B43C3181A1F1268FE
:10881000104C0E4D920014195219526C002A10D0AF
:108820001A00143A1268551C09D0103B1B68FF2B24
:1088300005D03B00934065461A00074BEA50FC34D4
:10884000666401310429DED1F0BDC046FC900040D1
:1088500044000020009000400C05000000B51E28D8
:1088600010D80C4A8000835803290BD8A022080096
:10887000C133FF33D2059B0001F000FC020905075C
:108880000021D15000BD0C21FBE70421F9E70321B1
:10889000F7E7C0465CF000001E280AD8074B8000AE
:1088A000C25801239340A022D205002902D10449D5
:1088B00053507047A121C900FAE7C0465CF00000A0
:1088C0000C050000030000201E2B0AD8A021A222C4
:1088D000C905D2008858034A9B009B58D840012301
:1088E000184070475CF00000F7B506000D000C0062
:1088F0008B180193019B671B9C4207D0336821783A
:108900001B683000984701340028F3D13800FEBDC1
:10891000F0B5C64600B5CB0F9846404A4B005B0DFC
:108920009A1882B00D000400132A2FDC002A49DBBC
:108930003B4F17413E000E40064323D07F083900CD
:1089400029400C430AD03749BD438C4663445C42FE
:108950005C418023DB021341E4071D434146CE0006
:1089600031492B008E1922003468756820002900D7
:1089700001F0F6FE009001910098019922002B0071
:1089800003F086F802B004BC9046F0BD332A08DD3F
:108990008023DB009A42F5D102000B0001F0E0FEDB
:1089A000F0E7224A9446012263445242DA400242EE
:1089B000E8D052080242D1D094438022D2051A4115
:1089C0001443CBE74B005B080343DBD00B031B0BCB
:1089D0001C436342234380244D0C24031B0B234080
:1089E0006D042B4319004346DA000F4B9B181C689B
:1089F0005D6802000B002000290001F0B1FE00902C
:108A000001910098019922002B0003F041F84246A1
:108A10004B005B08D60733431900B3E701FCFFFFA7
:108A2000FFFF0F00EEFBFFFF08F10000EDFBFFFF73
:108A3000F8B5274A4B005B0D9A180C000700132A63
:108A400010DC002A36DB234B13410B423AD0802442
:108A500024031441002064189C43060025003000C4
:108A60002900F8BD332A0EDD80230600DB000D004F
:108A70009A42F4D102000B003800210001F070FE90
:108A800006000D00EBE7144D0600AC4601256344DB
:108A90006D42DD40AC4663460D000342DFD0332318
:108AA0009A1A323B93401818874200D94C1C6346EF
:108AB0009843D2E7C90FCC070020531CCDD1074BF8
:108AC0001C43CAE706000D000028C0D1C7E7C04616
:108AD00001FCFFFFFFFF0F00EDFBFFFF0000F03F79
:108AE00030B5214A4B0087B05B0893421EDD1F4A18
:108AF000934205DD02000B0002F0CAFF07B030BD53
:108B000002AA00F095F803231840049A059B012857
:108B100013D002281DD0002814D00298039900F029
:108B20006FFB80231B069C466144E7E7002300227D
:108B30000093002301F0DEF8E0E70298039900F0CB
:108B40005FFBDBE7012402980399009401F0D2F85F
:108B5000D4E7012402980399009401F0CBF8802314
:108B60001B069C466144C9E7FB21E93FFFFFEF7FFD
:108B7000F0B54746CE4680B58DB004000D0000F03C
:108B800067FA294B06001B780F005BB29846013349
:108B900010D022002B002000290003F0C1FA8146EA
:108BA000002807D1002200232000290001F00AFC40
:108BB000002806D1300039000DB00CBC9046994613
:108BC000F0BD01230293194B0694079503934B467E
:108BD0000A93434604940595002B15D000230022E8
:108BE0001900100002F0D8F8434608900991022BB2
:108BF0000ED103F0AFFB212303600A9B0193002BEE
:108C00000CD1089E099FD5E70023002408930994FE
:108C100002A801F0C1F90028EFD1EAE703F09AFBBE
:108C20000A9B01930360ECE78800002018F1000024
:108C3000F0B54E464546DE465746E0B5E14B4C00A2
:108C40008FB09046894664089C4200DC87E0DE4B8A
:108C50009C4222DCDD4A002900DC92E0DC4B02F081
:108C600017FFDB4B06000F009C4200D17EE1D94A82
:108C7000D94B02F00DFF02000B00414630000A60A4
:108C80004B60390002F004FFD34BD24A02F000FFE0
:108C9000434601259860D9606BE0D04B9C4200DCD4
:108CA0008FE0CF4B9C4200DD55E1CE4A2315924622
:108CB0009A4451460905631A19001D00040003F087
:108CC0004BFA03F07FFA02000B0020002900089203
:108CD000099302F0DDFE0022C34B02F067FC0F0097
:108CE000060003F039FA03F06DFA04000D000200EB
:108CF0000B00300039000A940B9502F0C9FE0022E7
:108D0000B94B02F053FC002200230C900D9101F0AE
:108D100053FB002800D192E100230022200029000B
:108D200001F04AFB434243410133B04A41460192BC
:108D3000022208A80092524600F07CFB4B46050038
:108D4000002B16DA802243461206944642465B68A0
:108D5000454263445360D3686344D36009E00B0029
:108D6000020041460A604B600022002300258A6011
:108D7000CB6028000FB03CBC90469946A246AB465B
:108D8000F0BD934B01F0ECFC914B06000F009C42B0
:108D900000D13DE18F4A904B01F0E2FC02000B0054
:108DA000414630000A604B60390002F071FE894A8A
:108DB000894B01F0D5FC012543466D429860D9608E
:108DC000D7E701F049F88A4A8A4B06000F0002F003
:108DD000EDFB0022884B01F0C3FC03F0BDF9050058
:108DE00003F0F0F9794A7A4B0490059102F0DEFB2A
:108DF00002000B003000390002F04AFE754A0600FE
:108E00000F0004980599744B02F0D0FB0290039177
:108E10001F2D00DCC7E0029A039B3000390002F0EE
:108E200037FE83468A4653465B0024155B0DE31AE2
:108E3000102B6CDD04980599D322674B520502F084
:108E4000B5FB02000B00300039000292039302F0E0
:108E50001FFE0A000100130006910792020039006C
:108E6000300002F015FE029A039B02F011FE06008C
:108E70000F0004980599614A614B02F097FB32009C
:108E80003B0002F005FE069E079F0B000200390022
:108E900030000292039302F0FBFD4B005B0D834612
:108EA0008A46E41A312C32DD04980599B822544BD5
:108EB000920502F07BFB03000C0002000293039476
:108EC0000B000698079902F0E3FD02000B00060074
:108ED0000F000698079902F0DBFD029A039B02F04F
:108EE000D7FD484A0290039104980599464B02F039
:108EF0005DFB029A039B02F0CBFD02000B003000E9
:108F000039000292039302F0C3FD83468A465A4613
:108F10005346414630000A604B60390002F0B8FD0C
:108F2000029A039B02F0B4FD44460B000200A260CB
:108F3000E3604B46002B00DB1BE75B46236080238E
:108F40001B065344636080231B069C466144A0605B
:108F5000E1606D420DE70B00020002F099FD43460F
:108F600000259860D9601860596002E7D3221A4B37
:108F7000520502F08DFD214A214B0D00040002F044
:108F800087FD02000B00414620000A604B6029006B
:108F900002F07EFD1A4B194A02F07AFD4346012584
:108FA0009860D960E5E602000B003000390002F05D
:108FB0006FFD6B1E154A9B009B5883468A46A34251
:108FC000A5D130E7FB21E93F7BD9024000004054A6
:108FD000FB21F93F3163621A61B4D03DFB21394175
:108FE000FFFFEF7FEAFBFFFF00007041A0F10000F0
:108FF00083C8C96D305FE43F0000E03F7370032E0B
:109000008A19A33BC14920259A837B3920F10000AE
:10901000D3220C4B520501F0A3FB0B4A0B4B04006F
:109020000D0001F09DFB02000B00414620000A608C
:109030004B60290002F02CFD034A044BB9E60323E0
:1090400073E6C04661B4D03D7370032E8A19A33B0A
:10905000F8B54746CE46674B80B50A000F001900A9
:1090600005003940994200D19BE004000100002F27
:1090700069DD3F1500D1B4E05F4B12039C468023AD
:10908000120B5B0313435B00CA0F67449B184A0033
:10909000F80703D5D20F5B009B188A0079108C4625
:1090A000002180201624894680030D189D4202DC91
:1090B00029185B1B8144D50F5B00013C5B195200F2
:1090C0004008002CF1D10020804680202025002778
:1090D000000609E08B425CD0D40F5B00013DE31831
:1090E00052004008002D16D0C4198B42F2DD27181B
:1090F0000E00002C49DB5B1AA242894149425B1AEF
:10910000121BD40F5B00013D80443100E318520074
:109110004008002DE8D113434ED143465B08374940
:109120004A468846494652104244C90702D5802122
:1091300009060B4361460F05BD18180029000CBC39
:1091400090469946F8BD7B005B0803433900002B2D
:10915000F5D0002F3CD1E30A153A6405002BFAD074
:109160008020400303423FD1002700E00F005B0056
:10917000791C0342FAD0250020208D40401A290096
:10918000D71B2200C2401A4376E7FE43F60F8E1922
:10919000B1E79442A0D82718002CF6DB1E0000236C
:1091A000AEE702003B002800390002F0FFF92A0078
:1091B0003B0001F0D5FAC2E74346013303D04346F2
:1091C00001335B08ABE7012398460023C144A6E7BF
:1091D0003B00020002F05CFC02000B0001F0DCFD31
:1091E000ADE713000022BBE70127210020207F42CA
:1091F000C6E7C0460000F07F01FCFFFF0000E03F33
:10920000F0B54746CE4680B587B000920193754BC6
:109210004F00814688467F089F4263DC02F09CFF36
:10922000002800D1D4E04A4643464846414602F071
:10923000BDF904000D006C4A6C4B02F0B7F96C4AA2
:109240006C4B01F08DFA22002B0002F0AFF96A4A54
:109250006A4B02F01DFC22002B0002F0A7F9684ABD
:10926000684B01F07DFA22002B0002F09FF9664A5C
:10927000664B02F00DFC22002B0002F097F9644AC5
:10928000644B01F06DFA22002B0002F08FF902907E
:1092900003910022604B2000290002F087F9029A16
:1092A000039B06000F002000290002F07FF9009ABE
:1092B000019B04000D004846414602F077F9020088
:1092C0000B002000290002F0E3FB02000B0030003D
:1092D000390002F0DDFB02000B0000204F4902F0D4
:1092E000D7FB70E002000B0002F060F904000D00F3
:1092F0003D4A3E4B02F05AF93D4A3E4B01F030FAEE
:1093000022002B0002F052F93B4A3C4B02F0C0FB1A
:1093100022002B0002F04AF9394A3A4B01F020FAB8
:1093200022002B0002F042F9374A384B02F0B0FB22
:1093300022002B0002F03AF9354A364B01F010FAC0
:109340002B00220002F032F9354B029003919F422C
:109350009FDD344B00229F423DDC334900207B18C7
:109360002E4916001F0002F093FB04900591002285
:10937000294B2000290002F019F932003B0002F0CD
:1093800087FB029A039B06000F002000290002F0D1
:109390000DF9009A019B04000D004846414602F079
:1093A00005F902000B002000290002F071FB020009
:1093B0000B003000390002F06BFB02000B00049838
:1093C000059902F065FB07B00CBC90469946F0BDCC
:1093D00000201249F7E7154B002604920593144F1D
:1093E000C5E7C046FFFF3F3ED43888BEE9FAA8BDB6
:1093F000C4B1B4BD9EEE213EAD529C804F7E923EE4
:109400009015CB19A001FA3E7751C1166CC1563F99
:109410004C5555555555A53F0000E03F0000F03F25
:109420003233D33F0000E93F0000E0FF0000E73F98
:109430000000D23FF0B5DE464E4645465746E0B501
:10944000DC4CA5440D9114001900A49A0993DA4B41
:109450009200D6584D1E03901821E01E06960295E4
:1094600000F0A0FEC3430100DB1719404B1C9A001B
:109470009B1ADB001B190B9105934C1B771918D411
:10948000A59BA5009C463F1922AE6544013707E025
:10949000286802F097FE013403C60435BC4208D0A8
:1094A000002CF5DA00200021013403C60435BC424B
:1094B000F6D1069B002B01DA00F0FDFB069B039919
:1094C0000133DB009A46099BDA00944600920022A1
:1094D000914672AA0492B94A6144934688469AAB6F
:1094E00063449B44029B002B00DABCE15D460026EE
:1094F0000027039C4D442A686B6803CC02F056F8A1
:1095000002000B003000390001F02AF9083D060086
:109510000F004445EFD1049B4B441E605F6008235D
:109520009C46E144D145DDD10EA804218446494240
:1095300061448C46069A93009C44614684460A9195
:109540000399083B63448C460C93009B0092634450
:109550009B46009A0498D10003008C46634408910E
:109560001E685F68002A33DD954980468C46624458
:10957000D300984470AB9A460EAB99460022914BAB
:109580003000390002F012F802F0E6FD02F01AFE97
:1095900000228D4B04000D0002F008F802000B00C1
:1095A0003000390002F074FA02F0D6FD4B4601C3D8
:1095B0009946434620001A685B68290001F0D0F8FC
:1095C00008235B429C46E04406000F00D045D5D1FD
:1095D000059B30001A003900984600F0DFFCFF239D
:1095E00000229B0504000D0001F0E0FF00F038FCB4
:1095F0000022764B01F0DAFF02000B002000290068
:1096000002F046FA0D00040002F0A6FD814602F0C9
:10961000D9FD02000B002000290002F039FA0600F3
:1096200040460F00002800DCEEE0009B18215A1E87
:1096300092000EAB9B58091A1D000D41A9448D40A4
:109640005D1B0EAB9D5017231B1A1D41002D2DDDF8
:1096500001239C46009BE144002B00DC1CE20E9C95
:109660000123002C00D0B5E0009A012A09D099000E
:109670000EAA54580133002C00D0ACE0009A9A4254
:10968000F5D1059B002B0EDD012B00D1A8E1022BAB
:1096900009D1009B0EA95A1E92000EAB9B5807934E
:1096A0009B029B0A8B50022D00D1C1E000230022B7
:1096B0003000390000F080FE009B002800D194E2C9
:1096C000069A591E8A4210DC414A0A9894460EAA0C
:1096D0006344944600229B0063441C68043B22437D
:1096E0008342FAD1002A00D0C0E0069B0EAA013BBB
:1096F0009B00D358002B00D0B3E001220C9B043B0D
:10970000596801320029FAD0009B9C46624411003E
:1097100007921A0001338B4246DC0B986346804661
:10972000A59C4344A046099C9B00A1464A449844FA
:10973000D30022AA9146049A99449446089BA59A7C
:1097400063448446614494469A468B006344009384
:109750004346586802F036FD4B4618605960029B3C
:10976000002B24DB4D46039C0026002701E02868DF
:1097700069680CCC01F01AFF02000B0030003900C0
:1097800000F0EEFF083D06000F005C45EFD15346A8
:109790009E60DF6004239C460433E0449C46009BAB
:1097A000E144E2449845D3D1079B0093D1E60026DB
:1097B0000027ECE794FDFFFFE8F2000018FEFFFF32
:1097C000FFFFFF1F0000703E0000704100002040BE
:1097D000FFFFFF3F002180225204141B0EAA5450A9
:1097E000009999420EDD0EA884469B000EAA8900BE
:1097F000D25861446344CF4800E01A68821A04C317
:109800008B42FAD101243CE7059B002B06D1009B3B
:109810000EAA013B9B00D558ED1517E70022C64B59
:10982000300000F0EDFD002800D024E100253DE7E8
:1098300032003B000020C14902F02AF906000F0067
:10984000002C00D132E7059A0020BC4900F0A6FBAD
:1098500002000B003000390002F01AF906000F0078
:1098600024E7012250E70026002754E64B46059ADC
:10987000079388468B000EA9CB58183A0895059295
:10988000002B0DD18C464146AD4B43449B006344B5
:10989000043B58680139183A0028F9D088460592E7
:1098A000059A0020A54900F079FB434604000D000D
:1098B000002B00DA05E29E000EAB9C464346DB001F
:1098C00066449C46059370AB9946049F6744009795
:1098D000306802F077FC22002B0001F067FE0022C6
:1098E00038607960974B2000290001F05FFE083F47
:1098F00004000D00043EB945EAD14AAB03939B46F0
:1099000000239A46069B42469946434601320292FC
:1099100004934B46002B00DAAAE080208A4B009D7E
:109920009846C005894900260027002408E008233E
:109930009C460835E044544511DC43461868596894
:109940002A686B6801F032FE02000B00300039001B
:1099500000F006FF013406000F00A145E7DA5B4680
:10996000C0C39B4601239C46009BE244083B0093F6
:10997000029B9A45CDD1049B9846A49B022B00DD07
:109980008EE0002B37DC1FD1059B00271D00039BB9
:1099900000249C461E006544083E2A686B68380017
:1099A000210000F0DDFE083D07000C00AE42F4D1BE
:1099B000089B002B03D080231B069C4664443A007E
:1099C00023000D990A604B600720079B18409B23DA
:1099D0009B009D443CBC90469946A246AB46F0BDD8
:1099E000009B0EA95A1E92000EAB9B5807935B0278
:1099F0005B0A8B5057E64346002B00DA70E10020EB
:109A00000021DB004AAAD61848AF32687368083EC6
:109A100000F0A6FEB742F8D1089B002B00D025E14C
:109A20000B0002004A984B990D9C2260636002F083
:109A30002FF8434607000C00002B13DD01254CAE28
:109A4000B14638002E0021004C4601360CCC00F007
:109A500087FEA146B045F7DA089B07000C00002BF3
:109A600000D015E13A0023000D998A60CB60ABE786
:109A70000026002773E701239C46009BE144022552
:109A8000002B00DDEBE532003B0000202B4901F00C
:109A9000FFFF06000F0009E60024F2E54AAB03933E
:109AA000A49B032B00D08FE74346002B00DC14E17E
:109AB000039ADB009B46130091465B441E685F6877
:109AC000234B43440293DB00994448AB9A464B46F0
:109AD0005C681B681800210032003B000090019177
:109AE00000F03EFE04000D0002000B0000980199FA
:109AF00001F0CEFF3B00320000F032FE4B46986092
:109B0000D9601C605D6008235B429C46E1442600EE
:109B10002F00CA45DBD14346012B00DCE3E0039A6A
:109B200013005B441E685F68029BDB0099464A4451
:109B3000904610E0FFFFFF000000E03F0000F03F14
:109B4000FFFFFF3F0000703EA8F20000FB21F93F3D
:109B5000FFFFFF1F984643465C681B681800210002
:109B600032003B000090019100F0FAFD04000D006E
:109B700002000B000098019901F08AFF32003B00BF
:109B800000F0EEFD4346039A9860D9601C605D606A
:109B9000083B26002F009A42DCD14D469446002611
:109BA00000244746083565442A686B683000210068
:109BB00000F0D6FD083D06000C00AF42F4D1039B37
:109BC0004A9F5D689968D868089B002B65D0802201
:109BD000120694460D9B6544604464441F605D60BA
:109BE0009960D8601E615C61EEE69A464B46079329
:109BF000059B30005A423900089500F0CFF9002249
:109C00003A4B06000F0000F0FBFB002824D0384B35
:109C100000223000390001F0C9FC02F09DFA5246E2
:109C20000400950002F0CEFA0022304B01F0BEFC99
:109C300002000B003000390001F02AFF02F08CFA1C
:109C40000EAA50510122059B5244183390460593A9
:109C500093000EAAD45023E65346300039009C00EE
:109C600002F07AFA0EAB1851D04619E680230D9A0D
:109C70001B06CB18106053600B0002004A984B99EA
:109C800001F006FF434607000C00002B00DDD5E67F
:109C900080231B069C466444E4E62B003A000D9D9D
:109CA0002A606B600A000300AA60EB6032002300A8
:109CB0002A616B6188E6099BDB00009372AB049319
:109CC00032E4A49B022B00DDE8E6002B00DD92E6E7
:109CD00000D079E6002700246AE6002600246EE71B
:109CE0000020002198E60026340068E7000070415B
:109CF0000000703EF0B5CE46474680B587B0009272
:109D00000193474A4B00814688465B08934207DC33
:109D10004146484602F020FA4146031E484666D0B6
:109D20004A4643464846414601F040FC04000D00C7
:109D300002000B004846414601F038FC394A3A4BD4
:109D400006000F002000290001F030FC374A384B94
:109D500001F09EFE22002B0001F028FC354A364B14
:109D600000F0FEFC22002B0001F020FC334A344BB3
:109D700001F08EFE22002B0001F018FC314B324A1C
:109D800000F0EEFC0E9B02900391002B34D0009863
:109D9000019900222D4B01F009FC029A039B0490CB
:109DA00005913000390001F001FC02000B0004981D
:109DB000059901F06DFE22002B0001F0F7FB009ADF
:109DC000019B01F065FE224A04000D00214B30008A
:109DD000390001F0EBFB02000B002000290000F02D
:109DE000BFFC02000B004846414601F051FE07B09F
:109DF0000CBC90469946F0BD02000B0020002900E3
:109E000001F0D4FB124A134B01F042FE32003B003A
:109E100001F0CCFB4A46434600F0A2FCE7E7C0460F
:109E2000FFFF3F3E7CD5CF5A3AD9E53DEB9C2B8ACC
:109E3000E6E55A3E7DFEB157E31DC73ED561C11927
:109E4000A0012A3F1111813FA6F810110000E03F48
:109E5000495555555555C53F49004B0819007047A0
:109E6000474AF0B54F4691464B005B0D9944464634
:109E7000D6464A46C0B505000C000E0088460700CD
:109E8000132A27DC002A4BDB3E4B13419A460B007A
:109E900052461340034318D03B4A3C4B2800210054
:109EA00000F05EFC0022002300F0A0FA002847D05A
:109EB000002C04DA80234A465B031341984446464B
:109EC000534600279E43380031001CBC90469946FB
:109ED000A246F0BD332A08DD8023DB009945F4D18A
:109EE00002000B0000F03CFCEFE7294A94460122F7
:109EF00063445242DA4092460242E6D0224A234B61
:109F00002800210000F02CFC0022002300F06EFA53
:109F1000002815D0002C1EDB534646469F430FE019
:109F2000194A1A4B2800210000F01AFC00220023D5
:109F300000F05CFA002803D0002C04DB0027002688
:109F400038003100C1E76400640825430027002D74
:109F5000F6D0104EF4E74B46142B0BD03422D21A15
:109F6000012393405D19BD4208D201239C462F0076
:109F7000E044D1E7133B9C46E044CDE72F00CBE71C
:109F800001FCFFFFFFFF0F009C7500883CE4377E5B
:109F9000EDFBFFFF0000F0BF002070474B0070B5E5
:109FA0005B0D14000A00002B1AD14B005B08034321
:109FB00015D0234B002201F0F9FA224B9C422DDBF5
:109FC0000A004B005B0D363B1F4DE318AB422ADC09
:109FD000002B0DDD1D4C1B0522401A43110070BDE6
:109FE0001B4DAB42F0D102000B0000F0B9FBF6E7CD
:109FF0001D00353519DA174B02009C4209DD0B00B4
:10A000001548164900F032F8134A144B01F0CEFA05
:10A01000E5E70B001248134900F028F8104A114BED
:10A0200001F0C4FADBE70200E9E7084C36332240CE
:10A030001B051343190000220B4B01F0B7FACEE7C2
:10A0400000005043B03CFFFFFE070000FFFF0F8001
:10A05000FF07000050C300009C7500883CE4377E79
:10A0600059F3F8C21F6EA5010000903C30B54A00BC
:10A07000DB0FDB0752081A43110030BD02B47146F2
:10A0800049084900095C49008E4402BC7047C0463B
:10A09000002243088B4274D303098B425FD3030A27
:10A0A0008B4244D3030B8B4228D3030C8B420DD33A
:10A0B000FF22090212BA030C8B4202D312120902C8
:10A0C00065D0030B8B4219D300E0090AC30B8B4206
:10A0D00001D3CB03C01A5241830B8B4201D38B03B4
:10A0E000C01A5241430B8B4201D34B03C01A524159
:10A0F000030B8B4201D30B03C01A5241C30A8B429C
:10A1000001D3CB02C01A5241830A8B4201D38B0286
:10A11000C01A5241430A8B4201D34B02C01A52412A
:10A12000030A8B4201D30B02C01A5241CDD2C3099C
:10A130008B4201D3CB01C01A524183098B4201D318
:10A140008B01C01A524143098B4201D34B01C01A03
:10A15000524103098B4201D30B01C01A5241C3087B
:10A160008B4201D3CB00C01A524183088B4201D3EA
:10A170008B00C01A524143088B4201D34B00C01AD6
:10A180005241411A00D20146524110467047FFE742
:10A1900001B5002000F0F0F802BDC0460029F7D05C
:10A1A00076E7704703460B437FD4002243088B4277
:10A1B00074D303098B425FD3030A8B4244D3030B4E
:10A1C0008B4228D3030C8B420DD3FF22090212BA13
:10A1D000030C8B4202D31212090265D0030B8B428F
:10A1E00019D300E0090AC30B8B4201D3CB03C01A79
:10A1F0005241830B8B4201D38B03C01A5241430B54
:10A200008B4201D34B03C01A5241030B8B4201D343
:10A210000B03C01A5241C30A8B4201D3CB02C01AAE
:10A220005241830A8B4201D38B02C01A5241430A26
:10A230008B4201D34B02C01A5241030A8B4201D315
:10A240000B02C01A5241CDD2C3098B4201D3CB01BC
:10A25000C01A524183098B4201D38B01C01A52416B
:10A2600043098B4201D34B01C01A524103098B426F
:10A2700001D30B01C01A5241C3088B4201D3CB005A
:10A28000C01A524183088B4201D38B00C01A52413D
:10A2900043088B4201D34B00C01A5241411A00D2ED
:10A2A00001465241104670475DE0CA0F00D0494256
:10A2B000031000D34042534000229C4603098B42C6
:10A2C0002DD3030A8B4212D3FC22890112BA030A4E
:10A2D0008B420CD3890192118B4208D389019211D0
:10A2E0008B4204D389013AD0921100E08909C30955
:10A2F0008B4201D3CB01C01A524183098B4201D357
:10A300008B01C01A524143098B4201D34B01C01A41
:10A31000524103098B4201D30B01C01A5241C308B9
:10A320008B4201D3CB00C01A524183088B4201D328
:10A330008B00C01A5241D9D243088B4201D34B0043
:10A34000C01A5241411A00D20146634652415B1085
:10A35000104601D34042002B00D549427047634666
:10A360005B1000D3404201B5002000F005F802BDAB
:10A370000029F8D016E770477047C046D0400B1C44
:10A380001141203A03D49C4613411843634652427C
:10A39000934018437047C0468446101C62468C4662
:10A3A000191C634600E0C0461FB501F097F800286D
:10A3B00001D40021C8421FBD10B500F0EFFF40429C
:10A3C000013010BD10B501F089F8002801DB002034
:10A3D00010BD012010BDC04610B501F07FF8002867
:10A3E00001DD002010BD012010BDC04610B501F0F8
:10A3F00011F8002801DC002010BD012010BDC0466E
:10A4000010B501F007F8002801DA002010BD012086
:10A4100010BDC046F0B5CE46474615042D0C2E00A3
:10A4200080B50704140C3F0C9946030C7E435D4332
:10A43000674363437F19340CE4199C46A54203D952
:10A4400080235B029846C4444B4643435143250C4A
:10A4500036046544360C2404A4195B1959182000ED
:10A460000CBC90469946F0BDF0B54E465746454661
:10A47000DE46E0B543025B0A450083B00F1C9946F7
:10A480002D0EC60F002D57D0FF2D24D08020DB00CD
:10A49000C0041843002381469A469B467F3D7C02B8
:10A4A0007A00FB0F640A120E984623D0FF2A4BD085
:10A4B000E30080240020E4047F3A1C43AD186B1CA9
:10A4C00047460193534677403A000F2B48D87D49C1
:10A4D0009B00CB589F46002B00D085E008339A465E
:10A4E000063B9B467C027A00FB0FFF25640A120E96
:10A4F0009846DBD1002C00D090E0524601231A434D
:10A5000092460120DBE74C4658461700022824D02B
:10A51000032800D1CFE00022002301284DD15802AA
:10A52000D205400AFF071043384303B03CBC9046B5
:10A530009946A246AB46F0BD002B5BD104239A4658
:10A54000033B00259B46AAE7FF35002C60D152460D
:10A5500002231A4392460220B1E7FF220023DEE7DE
:10A560004B461B0C9C464B462604360C1804614691
:10A570003300220C6446000C43434E435043544383
:10A5800080191A0C1218964203D9802149028C4670
:10A5900064441B041B0C1004C01883015E1EB341ED
:10A5A000800E1843130C1B199B0103431C0023014D
:10A5B00079D5012362081C401443019A7F32002A96
:10A5C0004DDD630704D00F232340042B00D0043457
:10A5D000230103D53C4B019A1C408032FE2ABCDC8F
:10A5E000A3015B0AD2B29AE70C239A46093BFF25E6
:10A5F0009B4654E7180001F071FE4A46431F76253A
:10A600009A4000236D4291462D1A9A469B4646E792
:10A61000524603231A439246032050E7200001F0DC
:10A620005DFE431F2D1A9C40763D002047E78023A6
:10A630000027DB03FF2272E7424666E74C46320002
:10A64000584662E780234A46DB031A4222D01C4266
:10A6500020D123435B025B0A4746FF225FE70123C9
:10A660009A1A1B2A21DC23000199D3409E318C4089
:10A670001A0023005C1EA34113435A0704D00F2283
:10A680001A40042A00D004335A0111D49B015B0AFA
:10A69000002244E780234A46DB0313435B025B0A44
:10A6A0003700FF223BE7019587E70022002336E7CA
:10A6B0000122002333E78023DB0323435B025B0A91
:10A6C000FF222CE7F8F20000FFFFFFF770B500282B
:10A6D0003DD0C317C5185D40C40F280001F0FEFD32
:10A6E0009E22121A962A07DCD2B2082833DD0838D7
:10A6F00085406802400A23E0992A0BDD05232900E2
:10A700001B1AD94003001B339D402B005D1EAB413B
:10A7100019430D00052801DD431F9D402B000F4903
:10A720000B406E0709D00F263540042D05D00433A9
:10A730005D0102D59F220B40121A9B01580AD2B22A
:10A740004002D205400AE4071043204370BD0024B4
:10A7500000220020F4E76802400AF1E7FFFFFFFB58
:10A76000F0B54F464646D6460C000903C0B5490A27
:10A77000470F5E0039431F03DB0F9C4665007B0AD1
:10A78000570F1F436D0DE40F760DA146C000B8466C
:10A79000D200AB1B64457BD0002B5FDD002E00D0C8
:10A7A000A4E03E00164300D112E15E1E002E00D050
:10A7B0009EE1871A4346B84280410125C91A4042AA
:10A7C000091A0B0200D431E149024E0A002E00D1D1
:10A7D0006EE1300001F082FD0300083B1F2B00DD1D
:10A7E00061E120223900D21A9E40D1409F400E43A1
:10A7F0009D4200DD51E15D1B6B1C1F2B00DD7CE1E8
:10A800002021C91A3D0030008F408840DD40791E6C
:10A810008F41310007222843D940002507433A40A1
:10A82000002A09D00F233B40042B05D03B1DBB421F
:10A83000BF417F42C9191F000B0200D426E26A1CE7
:10A84000C64B55056D0D9A4200D106E1C44AFF087A
:10A850000A40530752023B43120B8EE0002B00D0FC
:10A86000B8E06B1C5B055B0D012B00DC30E1871A47
:10A870004346B842B641CB1A76429E1B330200D5FE
:10A880004CE13B003343A1D100220024002570E0BD
:10A89000002B00DCE5E0002E00D183E0AF4EB54296
:10A8A00060D0802636043743B846382B00DC3EE1C2
:10A8B000434613431F007A1E97413F188742804149
:10A8C000404209180B0200D4B0E0A44B01359D4270
:10A8D00000D1C3E0A24A7B080A4001210F401F4378
:10A8E0005108D30707221F433A4099E79B4EB542D0
:10A8F00038D0802636043743B846382B00DDDCE0FC
:10A900001F2B00DC30E11E004746203EF740BC46CE
:10A91000202B04D04026F31A46469E4032431700AF
:10A9200063467A1E97411F43CCE0002B00D104E21E
:10A930004346134300D159E14B07C0081843802315
:10A94000C9081B03194208D04546ED081D4204D131
:10A950004346D008590708432900420FC9007F4DDC
:10A960001143C0004B07CA087C49C00803438D420D
:10A9700068D012036D05120B6D0D00211203180033
:10A98000130B0A0D12051A43764B2D0513402B436A
:10A990005B00E4075B08234319001CBC9046994602
:10A9A000A246F0BD3E00164312D05E1E002E00D01F
:10A9B00000E187188742804141444042091801253F
:10A9C0000B0233D5022585E764463300414610006B
:10A9D0001D00C7E7002D00D0DAE00C000443F3D0DF
:10A9E0005C1C00D19FE15D4CA64200D12FE1DB430E
:10A9F000382B00DD66E11F2B00DD83E120240500FC
:10AA0000E41A0F00DD40D940A0404346A7405B1A3E
:10AA1000441EA04198462F433843171ABA42924128
:10AA200043465242991A64463500CAE607223A4024
:10AA3000002A00D0F6E64B07CA084849FF083B4306
:10AA40008D4296D11900114300D19EE18021090366
:10AA50000A431203120B414D8FE715000022002319
:10AA60008BE7002B00D0C7E06B1C5F057F0D012F2B
:10AA700000DCF1E0394DAB4200D1B9E085180A00A5
:10AA8000854289414244494251180722CF076D0847
:10AA90002F4349083A401D00C2E607223049ED1A0B
:10AAA00031403A40BCE63E002838864000279FE609
:10AAB000380001F013FC20308EE6434613431F009C
:10AAC0007A1E9741C71BB84280414042091A78E676
:10AAD0000E003B0006431343002D61D1002E00D031
:10AAE000F4E0002B00D11BE164463900100039E787
:10AAF0001A4FBB427AD03300FFE630001F3DE840DA
:10AB0000202B03D04021CB1A9E4037437B1E9F4110
:10AB1000072207433A400021002589E7171A4346D8
:10AB2000BA42B641591A76428E1B64464EE61F2B36
:10AB300000DDADE020264746F61AB740B9461700BB
:10AB4000B246DF404E463E4337005646B240561EA0
:10AB5000B24117434246DA408918AEE6FF070000CB
:10AB6000FFFF7FFFFFFF0F8020264746F61AB74002
:10AB7000B9461700B246DF404E463E4337005646C0
:10AB8000B240561EB24117434246DA40891A99E74D
:10AB90007F4CA6425BD0802424045B42214327E7FC
:10ABA000002E0CD1002B00D1CBE064463900100000
:10ABB000774DD7E6764FBB4218D0330075E6002BB1
:10ABC00014D04B07C00818438023C9081B0319423F
:10ABD00007D0FC081C4204D17907D0080843E1469D
:10ABE00021004C46420FC9001143C000684DB9E630
:10ABF0001D0000220023C0E6002D5BD10D0005439F
:10AC000000D1E2E65D1C00D1B0E0614DAE421FD044
:10AC1000DB43382B71DC1F2B00DD96E020250F0075
:10AC2000ED1AAF40B9460700AA46DF404D463D4306
:10AC30002F005546A840D940451EA84188440743E7
:10AC4000BF18974292415142414435003AE664466A
:10AC500035004146100085E60B000343002D00D06F
:10AC600063E6002BF5D04346134300D17AE68718FC
:10AC70008742804107224144404209183A400B0272
:10AC800000D4D5E6434B01351940C9E5380069E6E3
:10AC90001E004746203EF740BC46202B04D04026ED
:10ACA000F31A46469E403243170063467A1E974188
:10ACB0001F4302E6364DAE42CAD080252D045B42CA
:10ACC0002943A6E70843411E8841A6E6002B00D190
:10ACD00048E6871A4346B842B641CB1A76429E1BD5
:10ACE00033024BD5171A4346BA429241591A52427F
:10ACF000891A072264463A4092E501430F00791E03
:10AD00008F419DE71C000F00203CE740202B03D023
:10AD10004024E31A99400843411E884138437CE6A9
:10AD20000022002425E6171A4346BA429241591AD6
:10AD30005242891A6446350043E541461000144DDD
:10AD400010E680220024120380E61D000F00203D43
:10AD5000EF40BC46202B03D04025EB1A9940084316
:10AD600007006346781E87411F4369E787189742AB
:10AD70009B4141445B42C9183500A3E53B00334386
:10AD8000CED0072231003A4052E600231A00F4E503
:10AD9000FF070000FFFF7FFFF0B55746DE464E4637
:10ADA0004546E0B5834607000E03480085B092464D
:10ADB0001C00360B400DCD0F002800D19DE0954BB7
:10ADC000984239D08023F6001B041E43924A7B0F21
:10ADD00033439946944603006344009300230026BE
:10ADE000FF00029323031B0B98466300E40F5246B7
:10ADF0005B0D019400D1B3E086498B4200D19EE007
:10AE00004246D100802212040A435146490F1143A1
:10AE10008B46814952468C4600996344CB1A0021E7
:10AE2000D20000932B0063409A460F2E00D905E113
:10AE30007A4BB6009B599F465B463343994600D0F8
:10AE4000B8E002230826002700900293CAE7CB4609
:10AE50003A0002990195019B9A46022927D00329BD
:10AE600000D180E2012944D06D49009B8C466344A7
:10AE70001C00002C38DD530700D013E2D2085B46DB
:10AE8000DB0109D55946674B19408B468021C90023
:10AE90008C46009B63441C00634B9C4207DC5B4672
:10AEA00064055F075B0217431B0B620D02E0002382
:10AEB0000027584A00211B031C0B0B0D1B052343C5
:10AEC00014055A4A380013401C4353466400DB07FC
:10AED00064081C43210005B03CBC90469946A2463C
:10AEE000AB46F0BD0122524201231B1B382B00DC74
:10AEF000ADE1002200230027DCE75B46334399469F
:10AF00005ED0002E00D18AE1300001F0E7F90300A5
:10AF10000B3B1C2B00DD7BE11D22D31A5A4601009E
:10AF2000DA4008398E4013005F46334399468F401C
:10AF30003F4B00261B1A00930023029352E7414621
:10AF400053460B433B499B468C46009B634400930E
:10AF50005B46002B3BD1022300221E43022161E706
:10AF6000434613439B4637D04346002B00D162E152
:10AF7000404601F0B3F903000B3B1C2B00DD53E10D
:10AF800002004146083A914088461D21CB1A51469D
:10AF9000D9400B0041460B439B46534693401A0051
:10AFA000009B25499C46604403008C466344009303
:10AFB000002137E70323B14600900C26029311E7E6
:10AFC0000023009301330426002702930AE703239A
:10AFD000C3461E43032125E701331E4300220121FE
:10AFE00020E700239A46802300271B03094A61E7D4
:10AFF000802349461B03194200D1E2E05946194219
:10B0000000D0DEE00B431B0317001B0BA246014AD6
:10B0100050E7C046FF07000001FCFFFF38F30000C7
:10B02000FF030000FFFFFFFEFE070000FFFF0F8091
:10B030000DFCFFFF01F8FFFFF3030000D94500D925
:10B04000CBE000D1C6E03C0048460027009B013B16
:10B0500000935B46160E1B021E43130298463304F0
:10B060001B0C9946310C0191FFF798F84A46424370
:10B070000B04210C050019438A4207D98919013DA7
:10B080008E4203D88A4201D9851E8919881A0199EE
:10B09000FFF784F809048C464A462104644642437B
:10B0A000090C030021438A4204D98919013B8E42CD
:10B0B00000D8F1E02D041D43AB464346891A4246B1
:10B0C000280C12041D0C5B46140C22001B041B0CE4
:10B0D0005A4303946B434443029568431B19150C70
:10B0E000EB189C4203D980246402A44660441C0CE3
:10B0F00015041B042D0C20185D19814277D373D0E1
:10B100000C1AA24A7D1BAF42BF419446009B7F426E
:10B110006344E01B1C00864200D1DBE00199FFF78D
:10B120003DF84A4642430B04290C070019438A4262
:10B1300007D98919013F8E4203D88A4201D9871E57
:10B140008919881A0199FFF729F809044A4689469E
:10B1500029044D464243090C030029438A4207D97A
:10B160008919013B8E4203D88A4201D9831E89196D
:10B170003F04891A3A00039F1A43380013041B0C3A
:10B18000584381460298150C6F4343434543484654
:10B19000000C8446DB1963449F4203D9802040029F
:10B1A0008446654448461F0C00041B04000C7D19AE
:10B1B0001818A94200D284E000D17FE001231A438D
:10B1C00057E680234A461B0313431B031B0BAA4667
:10B1D0006F4A6FE6BA4200D935E74B46DC0758089C
:10B1E0007B081C43FF0734E70024AF4289D2474461
:10B1F0004745A4415B466442A4196418013BA6423A
:10B200001ED2A0426DD800D1B6E0241A9B4678E742
:10B2100003005A46283B9A400027914688E6584644
:10B2200001F05CF8203072E603005246283B9A4059
:10B2300093460022B4E6504601F050F820309AE6DA
:10B24000A642E2D1B845DCD9341A9B4659E71F2BF8
:10B2500065DC504C0099A4465C46614408008C4073
:10B2600011008240D940501E82410C4314435A467B
:10B27000DA401300620709D00F222240042A05D0C9
:10B280002200141D9442894149425B181A0262D57A
:10B290000122002300270DE68A4200D80AE7831E18
:10B2A000891907E70F231340042B00D1E6E5171D8A
:10B2B0009742924153429B44FA08E0E5002800D1AE
:10B2C000D7E57118531EB14227D3A94215D358D0E0
:10B2D0001A0073E7002B00DC04E6012300229B44E4
:10B2E000CDE502234744474589415B429C4649429C
:10B2F00089190C19E344241A03E743465F004745C4
:10B300009B41B8465B429E19023A8919A94200D076
:10B3100054E7404500D051E7ABE51A00F6E71F219E
:10B320005F4649420C1BE740202B07D01A49009B7F
:10B330008C46634418005B4683401A43501E82418A
:10B340003A4307270023174009D00F21002311405B
:10B350001400042995D122005F075B021B0BD20861
:10B3600017430022A6E5802359461B030B431B030A
:10B3700017001B0B064A9DE5BD42B2D89B46002430
:10B38000BFE68045B9D31A00C3E7C046FF030000FB
:10B39000FF0700001E0400003E040000F0B54F4609
:10B3A0004646D6468446C0B58046194E18030F035C
:10B3B0004D00000B5C0082463F0B6D0DC90F91469E
:10B3C000640DDB0F0120B5420AD0B44203D0A54280
:10B3D00001D157450CD01CBC90469946A246F0BD01
:10B3E00066463E43F7D1AC42F5D154461443F2D100
:10B3F0000120C845EFD1994207D0002DEBD163461B
:10B400001F433800471EB841E5E70020E3E7C04688
:10B41000FF070000F0B54F464646D6464D00C0B582
:10B420000E03C90F8A462C491F035C008046360B69
:10B430006D0D91463F0B640DDB0F8D421ED08C428B
:10B4400016D0002D1ED130438446002C01D13A4342
:10B4500023D06246002A1AD09A4529D051460220AC
:10B460000139084001381CBC90469946A246F0BDFF
:10B4700039001143E5D002204042F4E73043FAD1CD
:10B48000AC420FD0002C0FD13A43E7D00CE00122A0
:10B49000013B934318000130E5E763460020002B91
:10B4A000E1D0DBE73A43E6D19A45D7D1A542D5DCD6
:10B4B000A54205DBBE42D1D808D00020BE42D2D280
:10B4C00050460123013898430130CCE7C845C5D820
:10B4D0000020C845F4D3C6E7FF070000F0B54F468B
:10B4E0004646D6464D00C0B50E03C90F8A462E49C2
:10B4F0001F035C008046360B6D0D91463F0B640DBB
:10B50000DB0F8D4218D08C4211D0002D18D1304362
:10B510008446002C1ED13A431CD163460020002BE8
:10B5200030D0514602200139084001382AE0390064
:10B530001143EAD0022025E03043FBD1AC4226D0B3
:10B54000002C26D13A4324D151460220013908402B
:10B55000013817E06246002A0FD09A45E1D1A54292
:10B5600005DBBE42DDD819D00020BE420AD25046CB
:10B57000012301389843013004E00122013B934349
:10B58000180001301CBC90469946A246F0BD3A43D3
:10B59000D0D19A45C5D1A542C3DCE0E7C845C0D8A3
:10B5A0000020C845E3D3EDE7FF070000F0B557469C
:10B5B000DE464E464546E0B5834606000F0348008A
:10B5C00087B092461D003F0B400DCC0F002800D1E4
:10B5D0006FE0DE4B984238D08023FF001B041F43EE
:10B5E000730F3B430193DA4B0027994600239B4698
:10B5F000F60081442B0369001B0B52469846490D07
:10B60000ED0F002900D185E0D04B994200D173E0C5
:10B610004346DA0080231B0413435246CC48520FA2
:10B6200084461343524600206144D20089442100DD
:10B63000694000918C46012149448A460F2F00D968
:10B6400090E0C449BF00CF59BF465B463B430193DE
:10B6500000D06AE102230827002681469B46C9E7FD
:10B6600032005846019B61460091022800D175E0E6
:10B67000032800D1FEE1012800D02CE1002300279F
:10B68000002600253F032A0D3F0BB34812053A431D
:10B6900002401B051343009A5B00D1075B080B4374
:10B6A0003000190007B03CBC90469946A246AB4614
:10B6B000F0BD5B463B43019300D12FE1002F00D149
:10B6C000A5E1380000F00AFE03000B3B1C2B00DD57
:10B6D00096E11D22D31A5A460100DA405E46083927
:10B6E0008F4013008E403B4301939C4B00271B1A55
:10B6F000994600239B467DE7414653460B439349B9
:10B700008C46E144002B00D01AE1022202201743AC
:10B7100000228CE7134300D10DE14346002B00D1FA
:10B7200081E1404600F0DAFD02000B3A1C2A00DD00
:10B7300072E10100434608398B4098461D239A1A4E
:10B740005346D3401A004346134352468A40494663
:10B75000081A824989468144002068E77B4B00270C
:10B7600000268EE7140C1204120C1100370C36045C
:10B77000350C794328008C462E0060436044834694
:10B7800056432100300C804658467943404402918C
:10B79000844506D98846802149028C46E0444146CA
:10B7A00002913604010C360C00048B4681191E0CE4
:10B7B0001B041B0C0391190079438C462800754328
:10B7C0006544A8465843050C45447743A94203D92C
:10B7D000802149028C466744290C8C4639000004BC
:10B7E000000C2D042D186144AB4405915946049179
:10B7F00001990F043F0C080C390051434243904615
:10B8000002008C46090C8B4662437C4344445C44F2
:10B81000A04503D98021490288464244210C88462C
:10B8200061460904090C8C4639005943434370436F
:10B830007E430F0CF6182404BE19644442448C461F
:10B84000B34203D980235B0298464044029B614681
:10B850009846049B370443449B46AB45AD416B423D
:10B860000D0405992D0C8C467F196744FD18A846D8
:10B870005D462D19A542A44193466442A446C344A3
:10B88000DC448F42BF4198459B4193459241A4457A
:10B89000A4415B427F421F43360C52426442BF19AF
:10B8A0002243BF18624638184302D20D039913434E
:10B8B0006A020A43501E82416146ED0D2A434E0240
:10B8C0003243D90100D4B3E001265008324002438C
:10B8D000DE0732435B08224C5444002C62DD5107E2
:10B8E00009D00F201040042805D0101D904292412D
:10B8F00052429B180200D90104D580241948E40063
:10B90000034054441848844200DD27E75E075B0289
:10B91000D2081F0B630516435B0DB2E60023994660
:10B920000133042700269B4664E6032301978146E2
:10B930000C279B465EE6012201201743002276E693
:10B94000032303201F43434671E6C046FF07000060
:10B9500001FCFFFF78F30000FFFF0F800DFCFFFFED
:10B96000FF030000FFFFFFFEFE070000002380270B
:10B9700000933F030026434B83E6019B3200A4461D
:10B98000584670E6AC466EE6802701993F0339427F
:10B990002DD03B422BD11F433F033F0B0095160098
:10B9A000384B6EE601252D1B382D00DD66E61F2D78
:10B9B00040DC35481C005044160082408440EE4074
:10B9C000501E824134431443EB40620709D00F22DA
:10B9D0002240042A05D02200141D94428041404296
:10B9E0001B181A023ED501230027002649E68027AE
:10B9F000019B3F031F433F033F0B0094214B40E655
:10BA000003005A46283B9A40002601926DE65846AC
:10BA100000F064FC203057E603005246283B9A4071
:10BA20001300002293E6504600F058FC20307BE6DD
:10BA3000CA4650E71F201E004042041BE640202D4E
:10BA400003D0124C5444A3401A43501E8241324347
:10BA500007260027164009D00F20002310401400AD
:10BA60000428B9D122005E075B021F0BD2081643DF
:10BA7000002306E680273F031F433F033F0B1600CA
:10BA8000004BFEE5FF0700001E0400003E0400001E
:10BA9000F8B557464E464546DE460C000903E0B56C
:10BAA000490A460F5F0031431E03DB0F760A9B46AF
:10BAB000530F3343C84E6500C000E40FD2006D0D34
:10BAC000A24681467F0D9C469046B74200D1B9E020
:10BAD0005B46012673409B46EE1BA34500D183E0E5
:10BAE000002E63DD002F00D0B1E06346134300D188
:10BAF00023E1731E002B00D0BAE1861A6346B042E0
:10BB000080410125C91A4042091A0B0200D447E1BD
:10BB100049024B0A98464346002B00D189E1404632
:10BB200000F0DCFB0300083B1F2B00DD7CE1202242
:10BB30003000D21A4146D040994002009E400A434C
:10BB40009D4200DD6AE15D1B6B1C1F2B00DD94E153
:10BB5000202110003500C91A8E40DA408840DD40AF
:10BB6000711E8E41110007222843002506433240F2
:10BB7000002A09D00F233340042B05D0331DB342D4
:10BB8000B641764289191E000B0200D43DE26A1CC0
:10BB9000914B55056D0D9A4200D119E18F4AF60877
:10BBA0000A40570752023743120B9BE0002E00D089
:10BBB000C5E06E1C7605760D012E00DC48E1674677
:10BBC000861ACB1BB042BF417F42B8461F00434696
:10BBD000FF1A3B00B8461B0200D55FE137439AD1FC
:10BBE00000220024002579E0002E00DCFAE0002F7E
:10BBF00000D18DE0784B9D4267D0802367461B04BF
:10BC00001F43BC46382E00DC52E1634613435A1EE4
:10BC100093411E1886428041404209180B0200D40D
:10BC2000BEE06D4B01359D4200D1D2E06B4A7308F6
:10BC30000A4001210E401E435108D30707221E432C
:10BC4000324095E71E00164300D045E740E7624BBF
:10BC50009D423AD0802367461B041F43BC46382EC2
:10BC600000DDEBE01F2E00DC3AE133006746203BAD
:10BC7000DF403B00202E05D04027BF1B6646BE405C
:10BC8000324390464646721E96413343DAE0002B1B
:10BC900000D114E26346134300D168E180234E07CC
:10BCA000C008C9081B030643194208D06046C008F3
:10BCB000184204D163460100D2085E071643F30020
:10BCC0009946C900720F444D11434B46DE08424B62
:10BCD0004F073743CA089D4200D16EE012036D053D
:10BCE000120B6D0D00211203130B0A0D12051A43DE
:10BCF0003B4B2D0513402B435B00E4075B082343BC
:10BD0000380019003CBC90469946A246AB46F8BDA7
:10BD10006346134311D0731E002B00D007E1861831
:10BD20008642804161444042091801250B0237D503
:10BD300002257BE73E00614691463500C5E75C463B
:10BD4000002D00D0E1E00B000343F3D0731C00D1C1
:10BD5000ACE1214B9F4200D13AE1F343382B00DDA7
:10BD60006FE11F2B00DD8CE120250E00ED1AAE40A7
:10BD7000B0460600AA46DE40454635432E005546ED
:10BD8000D940A8406346451EA8415B1A9C463043F3
:10BD9000161AB242924163465242991A3D00B4E6E5
:10BDA00007223240002A00D0E4E60B4BF6084F078A
:10BDB0003743CA089D4200D090E73B00134300D1AF
:10BDC000A6E180231B031A431203120B024D89E7DD
:10BDD00015000022002785E7FF070000FFFF7FFF17
:10BDE000FFFF0F80002E00D0C7E06B1C5E05760DB4
:10BDF000012E00DCF0E0C84DAB4200D1B9E085185F
:10BE00000A00854289416244494251180722CE07FF
:10BE10006D082E43490832401D00A9E6BF49ED1ABE
:10BE2000114007223240A3E6320028388240002623
:10BE300086E6300000F052FA203073E66346134382
:10BE40005A1E9341C61AB04280414042091A5CE62C
:10BE50000E00674606431743002D5ED1002E00D02A
:10BE6000F3E0002F00D11EE15C46614691462CE7CD
:10BE7000A94FBE427BD01E00F1E610001F3DE840F6
:10BE8000202B03D04021CB1A9A401643731E9E41AB
:10BE90000722064332400021002583E7161A634635
:10BEA000B2428041591A40420B1A98465C4632E62B
:10BEB0001F2E00DDABE02027BB1B9A46634657468A
:10BEC000BB40994613004F46F3401F433B00574683
:10BED000BA40571EBA4113436246F240891898E6A9
:10BEE0002027BB1B9A4663465746BB409946130022
:10BEF0004F46F3401F433B005746BA40571EBA41D6
:10BF000013436246F240891A9CE7834B9F425FD0FD
:10BF100080252D047342294320E7002E0CD1002FE9
:10BF200000D1D0E05C46614691467B4DCDE67A4F2C
:10BF3000BE421CD01E0065E6002F18D0C0084E0778
:10BF400006438020C9080003014208D06346DC088C
:10BF5000044204D12100DA46D2085E071643F300FA
:10BF6000994601245346C900720F11431C406A4D83
:10BF7000ABE61D0000220027B4E6002D59D10B00CE
:10BF8000034300D1D6E6731C00D1B2E0624B9F425E
:10BF90001ED0F343382B6FDC1F2B00DD97E02025EC
:10BFA0000E00ED1AAE40B0460600AA46DE404546F9
:10BFB00035432E005546A840D940451EA8418C4423
:10BFC0000643B61896429241514261443D0025E62F
:10BFD0003D006146914678E60B000343002D00D0FA
:10BFE00055E6002BF5D06346134300D16DE6861865
:10BFF0008642804161444042091800220B0200D46D
:10C00000D0E6464B01351940B2E5B1465DE6330056
:10C010006746203BDF403B00202E05D04027BF1B5A
:10C020006646BE40324390464646721E96413343B2
:10C03000EFE5394B9F42CBD080252D047342294335
:10C04000A8E70843411E8841A2E6002F00D13CE644
:10C050006346861ACF1AB0429B415B42FB1A984650
:10C060001B024ED5161A6346B2429241591A5242E9
:10C07000891A5C4600227BE501430E00711E8E4149
:10C080009FE71D000E00203DEE40B046202B04D05F
:10C090004025EB1A99400843814648464346411ED5
:10C0A0008841184374E60022002417E6161A6346F6
:10C0B000B2429241591A5242891A3D0025E5614621
:10C0C0009146154D01E680220024120379E61D00F9
:10C0D0000E00203DEE40B046202B04D04025EB1A48
:10C0E0009940084381464E464346711E8E411E4389
:10C0F00067E7861896429B4161445B42C9183D0040
:10C100008CE547463743CED007224146324049E6C8
:10C1100000273A00E6E5C046FF070000FFFF7FFF6B
:10C1200070B50C4E0D031C0349005B002D0B490D2F
:10C13000240B5B0DB14208D0064900208B4203D18D
:10C1400014432000441EA04170BD05430120002D72
:10C15000FAD1F1E7FF07000030B5144D0A034B0098
:10C16000120B5B0DC90F0024AB4211DD104CA34232
:10C1700010DC8024640322430E4CE41A1F2C0CDDD7
:10C180000D48C31ADA4013005C42002900D11C009C
:10C19000200030BD094BCC18FAE7094DE040AC4611
:10C1A00063449A4013000343EEE7C046FE030000D9
:10C1B0001D0400003304000013040000FFFFFF7F94
:10C1C000EDFBFFFF70B500282DD0C317C5185D40EB
:10C1D000C40F280000F082F8154B1B1A5B055B0D9D
:10C1E0000A2815DD0B38854000222D032D0B002178
:10C1F00010002D030A0D2D0B12052A430D4D1B05B2
:10C200002A4013435B00E4075B082343190070BD19
:10C2100002002900153291400A000B21081AC5407E
:10C220002D032D0BE3E70024002300250022DEE789
:10C230001E040000FFFF0F804100090E4B1C70B56B
:10C24000DBB24602750AC40F012B14DDE0239B000C
:10C250006D07360BCB1800210A0D280012051C4D66
:10C2600032435B052A405B0813435B00E4075B082D
:10C270002343190070BD002914D1002D1ED02800C1
:10C2800000F02CF80A281CDC0B232A001B1ADA40C9
:10C29000030015339D400F4B12031B1A5B05160B51
:10C2A0005B0DD8E7002D06D0320B802636036D07D4
:10C2B0001643094BCFE7084B0026CCE700230026A6
:10C2C000C9E703002A000B3B9A400025E3E7C0467C
:10C2D000FFFF0F8089030000FF0700001C210123DE
:10C2E0001B04984201D3000C10391B0A984201D359
:10C2F000000A08391B09984201D30009043902A237
:10C30000105C40187047C04604030202010101019D
:10C31000000000000000000030B51C00094B0500C3
:10C320001B6885B0D868084B002A01D1074B1A005A
:10C330000292019300912B002200054900F026F89B
:10C3400000F0A6FD8C000020B8F3000001E0000022
:10C35000C5F30000014B18687047C0468C000020F0
:10C36000084B10B50400002B02D0002100E000BFF4
:10C37000054B1868836A002B00D09847200001F015
:10C380005DFBC04600000000F4F300000EB403B5EE
:10C39000010003AB044804CB0068019300F076F879
:10C3A00002B008BC03B018478C00002070B500260E
:10C3B0000C4D0D4C641BA410A64209D1002601F0BF
:10C3C0003FFB0A4D0A4C641BA410A64205D170BD68
:10C3D000B300EB5898470136EEE7B300EB589847A7
:10C3E0000136F2E75C0200205C0200205C020020C3
:10C3F0006C020020002310B59A4200D110BDCC5C25
:10C40000C4540133F8E710B5884202D98B1898421A
:10C4100003D3002307E08B5C8354013AFBD210BDA9
:10C42000CC5CC45401339A42FAD1F8E703001218E5
:10C43000934200D1704719700133F9E7936810B542
:10C44000013B9360002B04DA9469A34207DB0A29BD
:10C4500005D01368581C10601970080010BD00F05A
:10C460004BFC0100F9E7F8B506000F001400D518E1
:10C47000AC4201D1002007E021783A003000FFF7FC
:10C48000DDFF0134431CF3D1F8BD0000F0B59FB0CF
:10C4900002900F0016000593002805D083690493CD
:10C4A000002B01D100F0F4FD7B4B9F425BD1029B3E
:10C4B0005F68BB891B0762D53B69002B5FD00023F7
:10C4C00006AC6361203363761033A37635002B7896
:10C4D000002B01D0252B5CD1AB1B04930CD0320078
:10C4E00039000298FFF7BFFF431C00D1C4E0626926
:10C4F000049B9446634463612B78002B00D1BBE01E
:10C50000012200235242626002A9543252186E1C6A
:10C510002360E360A3601370A365317805225F4850
:10C5200000F0D4FE751C002835D12268D30604D54E
:10C53000532302A95B1820211970130704D5532334
:10C5400002A95B182B21197033782A2B2CD03500C7
:10C5500000210A20E3682A786E1C303A092A64D93F
:10C5600000292ED026E04E4B9F4202D1029B9F68AD
:10C570009FE74C4B9F429CD1029BDF6899E73900B3
:10C58000029800F00FFC002899D0012040421FB013
:10C59000F0BD01359BE7414B2268C01A012383405F
:10C5A000134323602E00B8E7059B191D1B680591F6
:10C5B000002B01DB099304E05B42E3600223134399
:10C5C00023602B782E2B0AD16B782A2B35D1059B33
:10C5D00002351A1D1B680592002B2BDB0793324E88
:10C5E00029780322300000F071FE002806D0402395
:10C5F000801B83402268013513432360297806227B
:10C600002A486E1C217600F061FE00283AD0284BA3
:10C61000002B25D10722059B07339343083305934D
:10C620006369039A9B18636150E7434301219B1898
:10C63000350090E701235B42D0E700230A201A006F
:10C640000135636029786E1C3039092903D9002B24
:10C65000C5D00792C3E74243012352183500F1E7E2
:10C6600005AB00933A00134B2100029800E000BF95
:10C670000390039B0133D3D1BB895B0600D584E7CC
:10C680000B9884E705AB00933A000A4B210002980F
:10C6900000F080F8ECE7C0464CF40000F8F300002E
:10C6A0006CF400002CF40000FEF3000002F4000023
:10C6B0000000000067C40000F7B5150001938A6808
:10C6C0000B6900900C00934200DA130022002B60EB
:10C6D00043321278002A01D001332B6023689B0675
:10C6E00002D52B6802332B60062723681F4027D012
:10C6F000230043331B785A1E93412268920630D49C
:10C700002200019943320098089EB047431C25D06F
:10C71000062320682A68E16803400025042B03D122
:10C720008D1AEB43DB171D40A3682269934201DD9C
:10C730009B1AED180027BD4220D1002010E00137E0
:10C74000E3682A689B1ABB42D2DD2200012319321A
:10C7500001990098089EB047431CF0D10120404247
:10C76000FEBD3020E1184331087021005A1C4531CC
:10C770000978A218433202331170C1E72200012365
:10C780001A3201990098089EB047431CE6D0013741
:10C79000D1E70000F0B589B004920A004332059356
:10C7A000039002920A7E0C000E9B6E2A00D186E056
:10C7B0001FD8632A33D008D8002A00D18CE0582A29
:10C7C0004DD0250042352A7030E0642A01D0692A14
:10C7D000F7D1196825680A1D280629D508681A6046
:10C7E000002803DA2D23029A404213706B4E0A2769
:10C7F0004FE0732A74D008D86F2A1FD0702AE0D176
:10C80000202209680A43226003E0752A16D0782A9C
:10C81000D7D12200782145321170614E22E02500E7
:10C820001A684235111D196013682B70012365E0E9
:10C8300008681A606906D3D500B2D1E7196825687F
:10C84000081D186008682E0605D5544E08276F2A63
:10C850001BD00A2719E06D06F7D580B2F5E7453100
:10C860004E4E0A7018682268011D0068196015068E
:10C8700021D5D30702D520231A4322601027002890
:10C8800003D1202322689A432260230000224333ED
:10C890001A706368A360002B58DB0422216891435F
:10C8A0002160002854D1029D002B5AD025003378F6
:10C8B00042352B7055E05506DBD580B2D9E71A68B2
:10C8C0000D68101D4969186013682E0601D519609E
:10C8D00002E06D06FBD519800023029D23614FE025
:10C8E0001A68111D1960156800216268280000F09F
:10C8F000EDFC002801D0401B6060636823610023C9
:10C90000029A13703CE023692A0004990398059D5C
:10C91000A847431C3ED023689B0715D4079BE068BB
:10C92000984239DA180037E02200012319320499BD
:10C930000398059EB047431C2CD00135E368079A45
:10C940009B1AAB42F0DCE9E70025F7E70028ADD001
:10C95000029D3900FDF722FC735C013D2B7000281D
:10C96000F7D1082F09D12368DB0706D56368226950
:10C97000934202DC3023013D2B70029B5B1B236141
:10C98000059B07AA00932100049B0398FFF794FEE0
:10C99000431CB8D10120404209B0F0BD09F40000A9
:10C9A0001AF400000D4B70B51C680500A36B002B3A
:10C9B0000FD1182000F06EFC094BA0630360094BF7
:10C9C00001224360084B83600B23838100230261B3
:10C9D00043610022A36B1D615A6170BD8C00002071
:10C9E0000E33CDAB34126DE6ECDE0500124B10B504
:10C9F0001C68A36B002B0FD1182000F04BFC0F4BD1
:10CA0000A06303600E4B012243600E4B83600B2337
:10CA10008381002302614361A46B0B4A2069616931
:10CA20000A4BFDF7F7FC01220023801859412061D1
:10CA300061614800400810BD8C0000200E33CDAB72
:10CA400034126DE6ECDE05002D7F954C2DF4515827
:10CA50000CB430B5164B9DB00C1E1D6808DA8B2344
:10CA600001202B6040421DB030BC08BC02B018470A
:10CA7000822302A99B008B810023029008619C42C3
:10CA800000D0631E8B604B6101235B42CB81209AF7
:10CA900021AB2800019300F055FD431C01DA8B23E4
:10CAA0002B60002CDFD00023029A1370DBE7C04616
:10CAB0008C0000200EB400B50B499CB01DAB029059
:10CAC0000690079104910948094904CB0591006833
:10CAD00002A9019300F036FD0023029A13701CB0E6
:10CAE00008BC03B01847C046FFFFFF7F8C00002042
:10CAF0000802FFFF020010B51378541C002B05D16B
:10CB0000CC5CD4540133002CFAD110BD2200F3E7E1
:10CB1000C9B20378002B04D08B4200D1704701309A
:10CB2000F7E74B42594149420840F7E702780B7852
:10CB3000002A03D0013001319A42F7D0D01A704751
:10CB40000023C25C0133002AFBD1581E704700232A
:10CB500030B59A420AD0013AC45CCD5CAC4204D1F3
:10CB6000934202D00133002CF6D1631B180030BD74
:10CB700030B50500002A00D130BD0C78013A6B1C9D
:10CB80002C700131002C05D19A189A42F4D01C70F7
:10CB90000133FAE71D00EDE710B50378002B0FD144
:10CBA0000B785A4253415B42184010BD0023CA5CC7
:10CBB000002AFAD0C45C944201D10133F7E7013076
:10CBC0000378002BF2D11800EFE70000F0B51F004A
:10CBD0000E0087B00590019102920C98347800F015
:10CBE000EAFA082200194378751C134036D12D2C1F
:10CBF00036D1B51C74780126002F62D0102F09D1D0
:10CC0000302C07D120222B789343582B54D1102756
:10CC10006C7802352D4B3900F31818000393FDF79B
:10CC2000BDFA049101210023494202008C461800FC
:10CC30002100303909291AD80C00A74223DD591CDC
:10CC400009D06346824206D302D10499A14202DB95
:10CC50000123784320182C780135E9E72E00BCE742
:10CC60002B2C01D01E00C7E7B51C7478FAE7210011
:10CC70004139192901D8373CDFE7210061391929E9
:10CC800001D8573CD9E75A1C08D1059A23331360C1
:10CC9000029B0398002B09D107B0F0BD002E00D0F5
:10CCA0004042029A002AF7D0002B01D06B1E01935C
:10CCB000029B019A1A60EFE73024002FAAD10827BF
:10CCC000A8E7302C9ED00A27A4E7C046FFFFFF7FCD
:10CCD00037B51300064A05001068046A002C00D11D
:10CCE000044C0A0000942900FFF770FF3EBDC046C7
:10CCF0008C000020F0000020F8B505000E001400A4
:10CD0000002804D08369002B01D100F0C1F9224B27
:10CD10009C422DD16C68A369A360A3891B0731D500
:10CD20002369002B2ED023682269F7B2981A636911
:10CD3000F6B2834205DC2100280000F03BF9002810
:10CD400026D1A3680130013BA36023685A1C2260EE
:10CD50001F706369834204D0A389DB071AD50A2EAA
:10CD600018D12100280000F025F9002812D00FE08A
:10CD70000A4B9C4201D1AC68CDE7094B9C42CAD119
:10CD8000EC68C8E72100280000F00CF80028CAD0A1
:10CD9000012676423000F8BD4CF400006CF400002F
:10CDA0002CF40000364B70B51D6806000C00002DF9
:10CDB00005D0AB69002B02D1280000F069F9314B96
:10CDC0009C420FD16C680C23E25E93B219072DD4FC
:10CDD000D90611D409230120336037331343A381CB
:10CDE000404270BD284B9C4201D1AC68EBE7274B19
:10CDF0009C42E8D1EC68E6E75B0713D5616B00293C
:10CE000008D023004433994202D0300000F06AFA7F
:10CE1000002363632422A3899343A38100236360D7
:10CE2000236923600823A2891343A3812369002B6C
:10CE30000BD1A0218022A389890092000B4093424C
:10CE400003D02100300000F0E1F90123A289134052
:10CE500011D00023A36063695B42A36100202369B2
:10CE60008342BED10C23E25E1306BAD5402313439E
:10CE7000A3810138B5E7920700D46369A360EDE7A9
:10CE80008C0000204CF400006CF400002CF4000036
:10CE900010B5062000F090FC012000F0CFFD00004E
:10CEA000F7B58A8905000C00130760D44B68002B86
:10CEB00004DC0B6C002B01DC0020FEBDE76A002FB8
:10CEC000FAD000232E682B6080235B01216A1A4070
:10CED00034D0606DA3895B0706D56368C01A636BA5
:10CEE000002B01D0236CC01A0200216A0023280005
:10CEF000E76AB847A189431C06D12B681D2B30D89F
:10CF00002B4ADA40D3072CD50023636023692360C2
:10CF1000CB0405D5431C02D12B68002B00D16065E2
:10CF2000616B2E600029C7D023004433994202D0A0
:10CF3000280000F0D7F900206063BEE70123280035
:10CF4000B847431CC6D12B68002BC3D01D2B01D082
:10CF5000162B01D12E60AFE74023A2891343A38192
:10CF6000ABE740230B430120A3814042A5E70F69B3
:10CF7000002FA1D00B680F60DB1B019300239207E9
:10CF800000D14B69A360019B002B00DC94E7019B5F
:10CF90003A00216A2800A66AB047002803DC402333
:10CFA000A2891343DFE7019B3F181B1A0193EAE7AD
:10CFB000010040200B6970B505000C00002B01D169
:10CFC000002070BD002804D08369002B01D100F03F
:10CFD0005FF80B4B9C4209D16C680C22A35E002BBE
:10CFE000EED021002800FFF75BFFEAE7054B9C42EB
:10CFF00001D1AC68F1E7044B9C42EED1EC68ECE760
:10D000004CF400006CF400002CF40000002310B578
:10D01000040003604360836081814366C2810361D1
:10D0200043618361190008225C30FFF7FFF9054B6B
:10D0300024626362044BA362044BE362044B2363E8
:10D0400010BDC046F9D7000021D8000059D8000013
:10D0500085D8000010B5024900F08CF810BDC0461C
:10D06000B5CF000070B568254A1E55430E00290053
:10D07000743100F081F9041E08D000212A000160FB
:10D0800046600C30A0606832FFF7D0F9200070BD18
:10D09000836913B50400002B28D18364C36403653E
:10D0A000134B144A1B6882620193984201D10123F9
:10D0B0008361200000F020F86060200000F01CF880
:10D0C000A060200000F018F80022E06004216068F1
:10D0D000FFF79CFF01220921A068FFF797FF0222BA
:10D0E0001221E068FFF792FF0123A36113BDC04640
:10D0F000F4F3000055D00000F8B51C4B07001E6883
:10D10000B369002B02D13000FFF7C2FF4836B46884
:10D110007368013B04D53368002B07D03668F6E707
:10D120000C22A55E002D0DD06834F2E704213800F2
:10D13000FFF798FF30600028F0D10C2304003B601B
:10D140002000F8BD20000A4B656625606560A5607B
:10D15000E36025616561A561082229005C30FFF765
:10D1600065F96563A563A564E564E9E7F4F3000088
:10D170000100FFFFF7B504000700002601914834C5
:10D18000002C01D13000FEBD6368A5680093009BB0
:10D19000013B009301D52468F2E7AB89012B08D944
:10D1A0000E22AB5E013304D029003800019B984762
:10D1B00006436835EBE7EC300068704770B50E0049
:10D1C0001D000E23C95E96B01400002907DA002363
:10D1D0002B60B3891B0611D48023DB000FE06A4665
:10D1E00000F088FB0028F2DBF022019B12021340C2
:10D1F000054A9B185A4253412B60EDE7402300201B
:10D20000236016B070BDC04600E0FFFFF7B50226F0
:10D210008B8905000C00334206D02300473323607E
:10D22000236101236361F7BD01AB6A46FFF7C6FFC7
:10D2300000990700280000F09FF8002808D10C2270
:10D24000A35E9A05EFD4032293431E43A681E4E72D
:10D250000F4BAB628023A28920601343A381009B04
:10D2600020616361019B002B0DD00E23E15E28003D
:10D2700000F052FB002806D00322A38993431A0032
:10D2800001231343A381A0893843A081CBE7C04683
:10D2900055D0000010B5034B0100186800F06CF881
:10D2A00010BDC0468C00002082B0002900D101A929
:10D2B000101E06D0002B06D013780B601078431E8A
:10D2C000984102B0704702204042FAE7C9B2821882
:10D2D000904201D10020704703788B42FBD001308F
:10D2E000F6E7000070B50500002910D00C1F236878
:10D2F000002B00DAE418280000F034FB1D4A136804
:10D30000002B05D163601460280000F02CFB70BD79
:10D31000A34209D9216860188342F3D118685B6879
:10D3200041182160EEE713005A68002A01D0A2429A
:10D33000F9D919685818A0420BD120680918581853
:10D3400019608242E0D110685268411819605A6031
:10D35000DAE7A04202D90C232B60D5E721686018D8
:10D36000824203D1106852684118216062605C609B
:10D37000CAE7C046341C0020032370B5CD1C9D4372
:10D38000083506000C2D1ED20C25A9421DD83000F0
:10D3900000F0E8FA254A14682100002919D1244C2C
:10D3A0002368002B03D1300000F0CAF92060290067
:10D3B000300000F0C5F9431C2BD10C233000336042
:10D3C00000F0D1FA03E0002DDFDA0C2333600020F7
:10D3D00070BD0B685B1B19D40B2B03D90B60CC18E9
:10D3E000256003E04B688C420DD11360300000F0E3
:10D3F000BAFA200007220B30231D9043C31AE7D04E
:10D400005A42E250E4E763600C00EFE70C00496821
:10D41000C3E70323C41C9C43A042E1D0211A30007F
:10D4200000F08EF9431CDBD1C7E7C046341C002056
:10D43000381C0020F8B507000D001600002905D1A2
:10D440001100FFF799FF04002000F8BD002A03D166
:10D45000FFF748FF3400F7E700F086FA2C00B042EF
:10D46000F2D231003800FFF787FF041EECD029000C
:10D470003200FEF7BFFF29003800FFF733FFE3E774
:10D48000F0B58E6885B007000C00039201939E42B0
:10D490003CD890238A89DB001A4234D003250969DD
:10D4A00023685B1A0293636902985D43EB0F5D1971
:10D4B000019B6D1001331B18AB4200D91D005305B1
:10D4C00032D529003800FFF757FF061E09D10C237B
:10D4D0003B6040230120A28940421343A38105B051
:10D4E000F0BD029A2169FEF785FFA389144A1A400C
:10D4F00080231343A381029B2661F6182660656191
:10D50000019EED1AA560019B9E4200D9019E32004A
:10D5100003992068FEF777FFA36800209B1BA36098
:10D5200023689E192660DAE72A003800FFF782FF99
:10D53000061EE0D121693800FFF7D4FEC7E7C046D8
:10D540007FFBFFFFF0B59FB0029005938B890F0022
:10D5500016001B0611D50B69002B0ED14021FFF7D9
:10D560000BFF38603861002805D10C23029A01387E
:10D5700013601FB0F0BD40237B61002306AC6361E4
:10D58000203363761033A37635002B78002B01D03F
:10D59000252B46D1AB1B04930CD0320039000298E6
:10D5A000FFF76EFF431C00D1AEE06269049B944616
:10D5B000634463612B78002B00D1A5E00122002396
:10D5C0005242626002A9543252186E1C2360E3601A
:10D5D000A3601370A365317805225448FFF776FEE7
:10D5E000751C00281FD12268D30604D5532302A935
:10D5F0005B1820211970130704D5532302A95B1867
:10D600002B21197033782A2B16D0350000210A20DF
:10D61000E3682A786E1C303A092A4ED9002918D0BE
:10D6200010E00135B1E7414B2268C01A0123834065
:10D63000134323602E00CEE7059B191D1B6805913F
:10D64000002B01DB099304E05B42E36002231343F8
:10D6500023602B782E2B0AD16B782A2B35D1059B92
:10D6600002351A1D1B680592002B2BDB0793304EE9
:10D67000297803223000FFF729FE002806D0402336
:10D68000801B8340226801351343236029780622DA
:10D6900028486E1C2176FFF719FE00283CD0264B47
:10D6A000002B25D10722059B0733934308330593AD
:10D6B0006369039A9B18636166E7434301219B18E2
:10D6C0003500A6E701235B42D0E700230A201A00B9
:10D6D0000135636029786E1C3039092903D9002B84
:10D6E000C5D00792C3E74243012352183500F1E742
:10D6F00005AB00933A00114B2100029800E000BFF7
:10D700000390039B0133D3D1BB890B985B0600D4F4
:10D710002FE7012040422CE705AB00933A00074B6E
:10D7200021000298FFF736F8EAE7C046F8F3000058
:10D73000FEF3000002F400000000000081D40000AD
:10D74000002370B5064C05000800236000F060F966
:10D75000431C03D12368002B00D02B6070BDC04652
:10D76000C82F002070B504000D001F2904D916230E
:10D7700003600120404270BD436C002B04D08A003E
:10D780009B181A68002A08D1200000F031F82A00FE
:10D790000100200000F01AF8EDE70020012AEAD08D
:10D7A000511C03D1162301302360E4E70024280034
:10D7B0001C6090472000DEE710B5034B010018689D
:10D7C000FFF7D0FF10BDC0468C000020002370B5CD
:10D7D000064C050008001100236000F001F9431C0D
:10D7E00003D12368002B00D02B6070BDC82F002010
:10D7F00010B500F0E5F810BD70B50C000E25495FBE
:10D8000000F0BAF8002803DB636D1B18636570BD78
:10D81000A389024A1340A381F9E7C046FFEFFFFF47
:10D82000F8B51F008B8905000C001600DB0505D537
:10D830000E23C95E0022022300F080F8A389054A66
:10D8400028001340A38132000E23E15E3B0000F06C
:10D850002BF8F8BDFFEFFFFF70B50C000E25495FF8
:10D8600000F06CF8A389421C03D1054A1340A38140
:10D8700070BD802252011343A3816065F8E7C04662
:10D88000FFEFFFFF10B50E23C95E00F021F810BDB9
:10D890000B1E04D0FF2A04D98A2303608B3B180097
:10D8A00070470A700123FAE770B5050008001100FF
:10D8B0000022064C22601A0000F0B8F8431C03D185
:10D8C0002368002B00D02B6070BDC046C82F0020FD
:10D8D000002370B5064C05000800236000F060F8D6
:10D8E000431C03D12368002B00D02B6070BDC046C1
:10D8F000C82F0020002370B5064C05000800110059
:10D90000236000F055F8431C03D12368002B00D09E
:10D910002B6070BDC82F0020002370B5064C050099
:10D920000800236000F054F8431C03D12368002B47
:10D9300000D02B6070BDC046C82F002070B5050018
:10D94000080011000022064C22601A0000F050F876
:10D95000431C03D12368002B00D02B6070BDC04650
:10D96000C82F0020704770470B1F1B68181F002B23
:10D9700001DA0B58C018704770B505000800110097
:10D980000022064C22601A0000F03AF8431C03D132
:10D990002368002B00D02B6070BDC046C82F00202C
:10D9A00058220120014B40421A607047C82F0020C6
:10D9B00058220120014B40421A607047C82F0020B6
:10D9C00058220120014B40421A607047C82F0020A6
:10D9D0005822024B00201A607047C046C82F002012
:10D9E00058220120014B40421A607047C82F002086
:10D9F00058220120014B40421A607047C82F002076
:10DA000058220120014B40421A607047C82F002065
:10DA1000044A1368002B00D1034B1818106018003B
:10DA20007047C0463C1C0020D02F00205822012007
:10DA3000014B40421A607047C82F0020FEE7C046E5
:10DA4000F8B5C046F8BC08BC9E467047F8B5C0465D
:10DA5000F8BC08BC9E467047646174610000000019
:10DA6000EEDA0000EF010000F7DA0000E302000048
:10DA7000FFDA0000090B000006DB0000450C000087
:10DA80000BDB00000905000011DB0000F5060000BB
:10DA90001CDB00005303000021DB00009D0E000092
:10DAA0002DDB00001F02000037DB0000D50900005D
:10DAB00045DB00009506000052DB000081080000F5
:10DAC0005EDB00005506000072616E646F6D0061E0
:10DAD0006C6C006C61737400300066616C7365007F
:10DAE0007472756500252E3135732E2E2E006D61F2
:10DAF0006B654C697374006164644C617374006499
:10DB0000656C657465006A6F696E0073706C69742A
:10DB100000636F707946726F6D546F0066696E6452
:10DB2000006A6F696E537472696E677300756E690F
:10DB3000636F6465417400756E69636F64655374E7
:10DB400072696E67006E65774279746541727261C1
:10DB5000790061734279746541727261790066720D
:10DB600065654D656D6F727900000000D1DB0000C6
:10DB700091130000D6DB0000AF130000FFDA0000B5
:10DB8000B3130000DCDB000095130000E6DB0000AF
:10DB9000B7130000EFDB0000BB130000F9DB00004F
:10DBA000BF13000004DC0000C313000010DC000001
:10DBB0009913000019DC0000A713000023DC00000B
:10DBC0009D1300002EDC0000AB13000066696C653D
:10DBD000006F70656E00636C6F736500656E644FF7
:10DBE0006646696C6500726561644C696E650072B9
:10DBF000656164427974657300617070656E644C30
:10DC0000696E6500617070656E6442797465730059
:10DC100066696C6553697A650073746172744C69E6
:10DC20007374006E657874496E4C6973740073790F
:10DC30007374656D496E666F000000008417000004
:10DC400094170000AE1700002A18000062180000A8
:10DC500096180000CE180000F418000038190000D3
:10DC60007A190000CE190000121A0000741A000080
:10DC7000BC1A0000E21A00001A1B0000601B000022
:10DC8000861B0000B41B0000E21B0000BE32000037
:10DC90009A1C00006C1D0000E21D0000521E0000D6
:10DCA0009E1E0000BE1E0000E01E00003820000086
:10DCB0007C200000F42000002221000054210000FC
:10DCC00086210000062200006E220000CA22000009
:10DCD000282300009A2300000C2400006824000080
:10DCE000C2240000F8240000482500008E25000012
:10DCF000D62500002A2600007E260000BC26000053
:10DD0000282700005E270000A6270000EE2700005D
:10DD10003628000070280000B828000008290000FC
:10DD20006A2A0000B41B00001A1B000070290000C2
:10DD300084170000A6290000D2290000082A00004C
:10DD4000342A0000841700008417000084170000A4
:10DD500084170000E62A0000282B00006E2B00002C
:10DD6000BE2B0000EA2B0000622C0000B42C000047
:10DD7000182D000084170000841700003C2D0000BF
:10DD80006C2D00009C2D0000D22D0000FC2D000009
:10DD9000322E00005C2E0000842E0000AC2E00000D
:10DDA000DC2E00000C2F0000362F0000602F00003A
:10DDB000902F0000BA2F0000841700008417000085
:10DDC000841700008417000084170000EA2F000069
:10DDD00016300000423000006E3000009A30000023
:10DDE000D030000010310000463100007C310000CE
:10DDF000A8310000D43100000A320000841700006E
:10DE000084170000841700008417000084170000A6
:10DE10008417000084170000841700008417000096
:10DE200084170000841700008417000036320000B9
:10DE300036320000583300008E3300005B2564202A
:10DE40006974656D206C6973745D002825642062B7
:10DE5000797465732900286F626A65637420747928
:10DE600070653A2025642900537461636B20756ED8
:10DE7000646572666C6F7700626F6F6C65616E00CF
:10DE80006E756D62657200737472696E67006C699D
:10DE900073740062797465206172726179000000A8
:10DEA000070000000300000031DF0000B53400006F
:10DEB00039DF00006535000042DF000099370000BF
:10DEC0004BDF0000B934000054DF00009D37000034
:10DED0005CDF00001937000065DF000049360000F4
:10DEE00070DF0000293900007BDF00002D370000C3
:10DEF00086DF00009D38000092DF0000F53500004D
:10DF00009EDF0000F93800001C0000000100000046
:10DF100002000000040000000500000006000000F0
:10DF2000100000001100000043616C6C696F7065A7
:10DF300000686173546F6E6500706C6179546F6E28
:10DF40006500686173536572766F0073657453651D
:10DF500072766F00646163496E697400646163572F
:10DF600072697465007371756172655761766500D9
:10DF7000736574557365724C454400616E616C6FD6
:10DF8000675265616400616E616C6F675772697496
:10DF900065006469676974616C52656164006469F5
:10DFA000676974616C577269746500474320746FC8
:10DFB0006F6B2025642075736563733B2066726503
:10DFC0006520256420776F726473003C496E746528
:10DFD0006765723E003C4C6973743E003C4F626A58
:10DFE0006563743E003C4279746541727261793EAA
:10DFF000000D0A564D2050616E69633A2025730D5D
:10E000000A006D69736300003DE00000F943000001
:10E0100046E00000894300004AE00000DD420000C5
:10E0200052E00000834200005CE000001942000062
:10E0300068E000001B4100006E756C6C006865783C
:10E04000546F496E740073696E006A736F6E476532
:10E0500074006A736F6E436F756E74006A736F6ECF
:10E0600056616C75654174006A736F6E4B657941DA
:10E070007400000038E100006544000040E1000049
:10E08000694400004AE100008744000053E10000B9
:10E09000914400005EE100009B4400006AE1000042
:10E0A000A544000078E10000AF44000080E10000DA
:10E0B000B944000086E10000C34400009BE1000079
:10E0C000CD440000B0E10000D7440000BCE10000F6
:10E0D000E1440000CCE10000EB440000D8E1000086
:10E0E000F5440000E5E10000FF440000F4E1000019
:10E0F0000945000007E20000134500001DE2000092
:10E100001D45000029E200002745000039E200001B
:10E110003145000048E200003B45000056E20000A7
:10E12000454500005EE200007344000066E2000026
:10E130007D4400006E65740068617357694669002C
:10E140007374617274576946690073746F705769AC
:10E1500046690077696669537461747573006D79F7
:10E1600049504164647265737300737461727453CF
:10E170005349447363616E006765745353494400A7
:10E180006D794D41430068747470536572766572A1
:10E190004765745265717565737400726573706F4D
:10E1A0006E64546F48747470526571756573740051
:10E1B00068747470436F6E6E656374006874747015
:10E1C0004973436F6E6E6563746564006874747040
:10E1D00052657175657374006874747052657370FC
:10E1E0006F6E736500776562536F636B657453740C
:10E1F00061727400776562536F636B65744C617311
:10E20000744576656E7400776562536F636B6574F1
:10E2100053656E64546F436C69656E74004D515460
:10E2200054436F6E6E656374004D5154544973438B
:10E230006F6E6E6563746564004D51545444697328
:10E24000636F6E6E656374004D5154544C6173740A
:10E250004576656E74004D515454507562004D51B1
:10E260005454537562004D515454556E7375620089
:10E270000D0E0F04050C0B0A06070809000000002C
:10E280000008080800080A4A4000000A5FEA5FEA3E
:10E290000ED92ED36E19324489330C924C924D080C
:10E2A0000800000004880808040804848488000A20
:10E2B000448A4000048EC480000000048800000EE0
:10E2C000C000000000080001224488100C92525245
:10E2D0004C048C84848E1C824C901E1EC244924C32
:10E2E00006CA525FE21FF01EC13E02448ED12E1FAD
:10E2F000E24488100ED12ED12E0ED12EC4880008F3
:10E3000000080000048004880244880482000EC0D3
:10E310000EC008048244880ED126C0040ED135B345
:10E320006C0C925ED2521C925C925C0ED010100E5D
:10E330001C9252525C1ED01C901E1ED01C90100EBF
:10E34000D013712E12525ED2521C8808081C1FE294
:10E3500042524C1254981492101010101E113B751A
:10E36000B131113935B3710C9252524C1C925C9000
:10E37000100C92524C861C925C92510ED00C825C16
:10E380001FE4848484125252524C1131312A4411B8
:10E390003135BB7112524C9252112A4484841EC4EE
:10E3A00088101E0EC808080E10080482410EC242D2
:10E3B000424E048A400000000000001F0804800054
:10E3C00000000ED2524F10101C925C000ED0100EA6
:10E3D00002424ED24E0C925C900E06C81C88080E6B
:10E3E000D24EC24C10101C9252080008080802407D
:10E3F00002424C10149814920808080806001B7575
:10E40000B131001C925252000C92524C001C925C92
:10E4100090000ED24EC2000ED010100006C8049814
:10E4200008080EC807001252524F0011312A44004A
:10E43000113135BB00124C8C9200112A4498001EF9
:10E44000C4881E06C48C8486080808080818080CAE
:10E45000881800000C83600000000000010000002C
:10E46000020000000300000004000000050000009E
:10E47000060000000700000008000000090000007E
:10E480000A0000000B0000000C0000000D0000005E
:10E490000E0000000F00000010000000120000003D
:10E4A0001400000016000000180000001A00000010
:10E4B0001C0000001E0000002000000023000000DF
:10E4C00026000000290000002C0000002F000000A2
:10E4D00032000000360000003A0000003E0000005C
:10E4E00042000000460000004B0000005000000009
:10E4F000550000005A0000006100000068000000A4
:10E500006F000000760000007D0000008400000025
:10E510008B0000009200000099000000A0000000A5
:10E52000A7000000AE000000B5000000BC00000025
:10E53000C3000000CA000000D1000000D8000000A5
:10E54000DF000000E6000000ED000000F400000025
:10E55000FB000000FF000000A8E500006945000086
:10E56000B3E50000E14A0000BDE5000021470000DE
:10E57000CAE5000051480000D1E50000A1480000B4
:10E58000DAE50000F1480000E6E50000E947000098
:10E59000F7E50000E149000004E6000079470000CB
:10E5A000646973706C6179006C696768744C657636
:10E5B000656C006D62446973706C6179006D6244D2
:10E5C0006973706C61794F6666006D62506C6F7430
:10E5D000006D62556E706C6F74006D62447261778D
:10E5E0005368617065006D625368617065466F7253
:10E5F0004C6574746572006E656F506978656C5314
:10E60000656E64006E656F506978656C5365745013
:10E61000696E004E6F7420656E6F75676820726F4B
:10E620006F6D206576656E20616674657220636F1C
:10E630006D70616374696F6E00436F6D70616374B8
:10E64000656420466C61736820636F646520737431
:10E650006F72650A2564206279746573207573652D
:10E660006420282564252529206F66202564004222
:10E670006164207265636F726420666F756E6420DA
:10E68000647572696E6720696E697469616C697A14
:10E690006174696F6E00256420256420256420283C
:10E6A000256420776F726473290025642072656386
:10E6B0006F7264732C20256420776F7264732C2032
:10E6C0006D617849442025642C20636F6D7061630F
:10E6D00074696F6E206379636C65732025640052E2
:10E6E0006573746F7265642025642073637269704A
:10E6F0007473005374617274656400726164696F4D
:10E700000000000094E70000CD540000A1E70000E5
:10E7100069570000B1E70000E9560000BFE70000BC
:10E72000FD580000CAE70000F5540000DAE70000D9
:10E730007D550000EEE7000065550000FDE7000094
:10E74000DF5A000009E800005D5A000012E80000EE
:10E75000015A00001DE800004959000028E80000A7
:10E760008559000031E80000B95900003AE800007E
:10E770000555000049E80000E554000052E800009B
:10E78000155500006E6F6E65006F746865720070DD
:10E790006169720064697361626C65526164696F7A
:10E7A000006D65737361676552656365697665645D
:10E7B000007061636B6574526563656976650070AE
:10E7C00061636B657453656E640072656365697639
:10E7D0006564496E74656765720072656365697624
:10E7E00065644D6573736167655479706500726522
:10E7F000636569766564537472696E670073656EEC
:10E8000064496E74656765720073656E6450616912
:10E81000720073656E64537472696E670073657419
:10E820004368616E6E656C0073657447726F7570D6
:10E8300000736574506F776572007369676E616C01
:10E84000537472656E6774680064657669636549C0
:10E8500044006C6173744D6573736167654944006E
:10E86000556E6B6E6F776E207072696D6974697624
:10E8700065205B25733A25735D00000000000000F1
:10E88000963007772C610EEEBA51099919C46D07BD
:10E890008FF46A7035A563E9A395649E3288DB0E18
:10E8A000A4B8DC791EE9D5E088D9D2972B4CB609FB
:10E8B000BD7CB17E072DB8E7911DBF906410B71DD8
:10E8C000F220B06A4871B9F3DE41BE847DD4DA1A11
:10E8D000EBE4DD6D51B5D4F4C785D38356986C1342
:10E8E000C0A86B647AF962FDECC9658A4F5C0114BB
:10E8F000D96C0663633D0FFAF50D088DC8206E3B99
:10E900005E10694CE44160D5727167A2D1E4033CAA
:10E9100047D4044BFD850DD26BB50AA5FAA8B535D1
:10E920006C98B242D6C9BBDB40F9BCACE36CD832C0
:10E93000755CDF45CF0DD6DC593DD1ABAC30D92667
:10E940003A00DE518051D7C81661D0BFB5F4B4216A
:10E9500023C4B3569995BACF0FA5BDB89EB8022867
:10E960000888055FB2D90CC624E90BB1877C6F2FEC
:10E97000114C6858AB1D61C13D2D66B69041DC76E7
:10E980000671DB01BC20D2982A10D5EF8985B171C0
:10E990001FB5B606A5E4BF9F33D4B8E8A2C907786F
:10E9A00034F9000F8EA8099618980EE1BB0D6A7F06
:10E9B0002D3D6D08976C6491015C63E6F4516B6BBF
:10E9C00062616C1CD83065854E0062F2ED95066C74
:10E9D0007BA5011BC1F4088257C40FF5C6D9B065E9
:10E9E00050E9B712EAB8BE8B7C88B9FCDF1DDD6246
:10E9F000492DDA15F37CD38C654CD4FB5861B24DAC
:10EA0000CE51B53A7400BCA3E230BBD441A5DF4A75
:10EA1000D795D83D6DC4D1A4FBF4D6D36AE9694338
:10EA2000FCD96E34468867ADD0B860DA732D0444E3
:10EA3000E51D03335F4C0AAAC97C0DDD3C7105500E
:10EA4000AA41022710100BBE86200CC925B56857B5
:10EA5000B3856F2009D466B99FE461CE0EF9DE5EFE
:10EA600098C9D9292298D0B0B4A8D7C7173DB359AF
:10EA7000810DB42E3B5CBDB7AD6CBAC02083B8ED40
:10EA8000B6B3BF9A0CE2B6039AD2B1743947D5EA4D
:10EA9000AF77D29D1526DB048316DC73120B63E37C
:10EAA000843B64943E6A6D0DA85A6A7A0BCF0EE4DB
:10EAB0009DFF099327AE000AB19E077D44930FF096
:10EAC000D2A3088768F2011EFEC206695D5762F78D
:10EAD000CB67658071366C19E7066B6E761BD4FECA
:10EAE000E02BD3895A7ADA10CC4ADD676FDFB9F9A7
:10EAF000F9EFBE8E43BEB717D58EB060E8A3D6D669
:10EB00007E93D1A1C4C2D83852F2DF4FF167BBD196
:10EB10006757BCA6DD06B53F4B36B248DA2B0DD899
:10EB20004C1B0AAFF64A0336607A0441C3EF60DF3C
:10EB300055DF67A8EF8E6E3179BE69468CB361CB25
:10EB40001A8366BCA0D26F2536E2685295770CCC4A
:10EB500003470BBBB91602222F260555BE3BBAC58B
:10EB6000280BBDB2925AB42B046AB35CA7FFD7C27C
:10EB700031CFD0B58B9ED92C1DAEDE5BB0C2649B6D
:10EB800026F263EC9CA36A750A936D02A906099CA0
:10EB90003F360EEB8567077213570005824ABF9513
:10EBA000147AB8E2AE2BB17B381BB60C9B8ED29296
:10EBB0000DBED5E5B7EFDC7C21DFDB0BD4D2D386ED
:10EBC00042E2D4F1F8B3DD686E83DA1FCD16BE8160
:10EBD0005B26B9F6E177B06F7747B718E65A088831
:10EBE000706A0FFFCA3B06665C0B0111FF9E658FC2
:10EBF00069AE62F8D3FF6B6145CF6C1678E20AA06C
:10EC0000EED20DD75483044EC2B30339612667A7F1
:10EC1000F71660D04D476949DB776E3E4A6AD1AE40
:10EC2000DC5AD6D9660BDF40F03BD83753AEBCA9CF
:10EC3000C59EBBDE7FCFB247E9FFB5301CF2BDBD3C
:10EC40008AC2BACA3093B353A6A3B4240536D0BA45
:10EC50009306D7CD2957DE54BF67D9232E7A66B3E2
:10EC6000B84A61C4021B685D942B6F2A37BE0BB48F
:10EC7000A18E0CC31BDF055A8DEF022D416C6C2059
:10EC80007461736B732073746F7070656400763198
:10EC9000343200202573202573004D656D6F727925
:10ECA00020636C6561726564004E6F2066726565F5
:10ECB000207461736B20656E747269657300000067
:10ECC00038ED0000AD73000045ED00005D710000FF
:10ECD00051ED00002D71000057ED00003D71000066
:10ECE0005DED00004D71000063ED0000DD6E000081
:10ECF00079ED00009572000087ED0000816B000047
:10ED000091ED00002173000099ED00001D6F0000DF
:10ED1000A2ED0000456D0000AEED00005D6C00004E
:10ED2000B7ED0000A96C0000BFED0000316E0000DF
:10ED300073656E736F727300616363656C65726196
:10ED400074696F6E0074656D70657261747572655B
:10ED50000074696C74580074696C74590074696C3F
:10ED6000745A00736574416363656C65726F6D6599
:10ED700074657252616E6765006D61676E65746976
:10ED8000634669656C6400746F756368526561649D
:10ED90000069326352656164006932635772697455
:10EDA000650073706945786368616E6765007370AC
:10EDB0006953657475700072656164444854006DF0
:10EDC0006963726F70686F6E65000000D1DB0000D0
:10EDD000B9740000D6DB00006574000003EE00008B
:10EDE000FD75000008EE00008174000011EE0000C7
:10EDF0008575000017EE0000DD7400007365726910
:10EE0000616C00726561640072656164496E746F63
:10EE10000077726974650077726974654279746508
:10EE200073000000A0EE00002D760000AEEE0000A2
:10EE30003D760000BBEE000031760000C4EE00001D
:10EE400041760000CEEE000045760000D7EE0000CF
:10EE500049760000DCEE00004D760000E1EE000097
:10EE600051760000EDEE000055760000F4EE000053
:10EE700059760000FDEE00005D76000002EF000014
:10EE8000617600000DEF00006576000017EF0000CE
:10EE90003576000021EF00003976000074667400BA
:10EEA000656E61626C65446973706C61790073654D
:10EEB000744261636B6C6967687400676574576955
:10EEC0006474680067657448656967687400736591
:10EED00074506978656C006C696E65007265637466
:10EEE00000726F756E646564526563740063697265
:10EEF000636C6500747269616E676C650074657837
:10EF00007400746674546F75636865640074667425
:10EF1000546F7563685800746674546F75636859EC
:10EF200000746674546F756368507265737375729C
:10EF3000650076617273000058EF0000F57A0000FA
:10EF400062EF0000D57A00006BEF0000B17A00009C
:10EF500077EF00003F7A000076617245786973743C
:10EF600073007661724E616D6564007365745661FD
:10EF7000724E616D6564007661724E616D65466FBB
:10EF800072496E6465780057656C636F6D652074B7
:10EF90006F204D6963726F426C6F636B73210070F9
:10EFA0005F73706920213D204E554C4C002F686FD7
:10EFB0006D652F6769742F2E706C6174666F726D4A
:10EFC000696F2F7061636B616765732F6672616D26
:10EFD00065776F726B2D61726475696E6F6E6F729B
:10EFE0006469636E7266352F6C69627261726965FD
:10EFF000732F5350492F5350492E63707000535054
:10F0000049436C6173733A3A535049436C6173736B
:10F01000284E52465F5350495F547970652A2C2020
:10F0200075696E74385F742C2075696E74385F74FE
:10F030002C2075696E74385F742900000000000090
:10F0400000000000C97C0000857C0000AB7C000053
:10F05000B57C0000BF7C0000A97C0000000000001F
:10F060000100000002000000160000000400000083
:10F070000500000006000000070000000800000076
:10F08000090000000A0000000B0000000C00000056
:10F090000D0000000E0000000F0000001A0000002C
:10F0A0001B0000001400000013000000110000000D
:10F0B00017000000100000001C0000001D000000F0
:10F0C0001E000000120000001500000003000000F8
:10F0D00018000000190000000000000000000000FF
:10F0E000B5800000E98800003581000049810000FA
:10F0F0003F810000B1800000A58000005581000024
:10F10000D1800000A180000000000000000030431A
:10F1100000000000000030C3737172740000000032
:10F12000FB21F93FFB2109407CD91240FB2119400A
:10F130007A6A1F407CD92240BBFD2540FB21294033
:10F140003A462C407A6A2F405C4731407CD93240A5
:10F150009C6B3440BBFD3540DB8F3740FB21394091
:10F160001BB43A403A463C405AD83D407A6A3F4048
:10F170004C7E40405C4741406C1042407CD942404C
:10F180008CA243409C6B4440AC344540BBFD4540A1
:10F19000CBC64640DB8F4740EB584840FB214940F7
:10F1A00083F9A200444E6E00FC291500D1572700B8
:10F1B000DD34F50062DBC0003C99950041904300CE
:10F1C0006351FE00BBDEAB00B761C5003A6E2400A0
:10F1D000D24D42004906E00009EA2E001C92D100FF
:10F1E000EB1DFE0029B11C00E83EA700F5358200AA
:10F1F00044BB2E009CE98400B4267000417E5F0071
:10F20000D6913900538339009CF439008B5F840018
:10F2100028F9BD00F81F3B00DEFF97000F9805009E
:10F22000112FEF000A5A8B006D1F6D00CF7E360044
:10F2300009CB2700464FB7009E663F002DEA5F00CE
:10F24000BA277500E5EBC7003D7BF100F7390700F1
:10F2500092528A00FB6BEA001FB15F00085D8D00CF
:10F26000300356007BFC4600F0AB6B0020BCCF00A7
:10F2700036F49A00E3A91D005E619100081BE600C8
:10F2800085996500A0145F008D40680080D8FF005C
:10F2900027734D0006063100CA561500C9A8730031
:10F2A0007BE260006B8CC00000000040FB21F93F56
:10F2B000000000002D44743E000000809846F83C99
:10F2C0000000006051CC783B00000080831BF039C7
:10F2D0000000004020257A38000000802282E336BA
:10F2E000000000001DF3693502000000030000006B
:10F2F000040000000600000060A500000AA5000050
:10F300000AA5000038A6000006A5000006A500001A
:10F310002EA6000038A6000006A500002EA60000BC
:10F3200006A5000038A600003CA600003CA6000090
:10F330003CA6000044A600003CB00000AEAE0000B9
:10F34000F2AE000056AE0000F2AE0000E2AF0000E8
:10F35000F2AE000056AE0000AEAE0000AEAE000051
:10F36000E2AF000056AE00004EAE00004EAE000010
:10F370004EAE0000F0AF000064B7000066B60000BB
:10F3800066B6000084B9000060B6000060B60000F8
:10F390006CB9000084B9000060B600006CB90000D0
:10F3A00060B6000084B900007AB900007AB90000A4
:10F3B0007AB9000088B900002C2066756E63746904
:10F3C0006F6E3A2000617373657274696F6E2022EC
:10F3D000257322206661696C65643A2066696C65F4
:10F3E00020222573222C206C696E652025642573EC
:10F3F00025730A0090000020232D302B2000686C1C
:10F400004C00656667454647003031323334353647
:10F410003738394142434445460030313233343580
:10F4200036373839616263646566000000000000A9
:10F4300000000000000000000000000000000000CC
:10F4400000000000000000000000000000000000BC
:10F4500000000000000000000000000000000000AC
:10F46000000000000000000000000000000000009C
:10F47000000000000000000000000000000000008C
:10F48000000000000000000000000000504F534941
:10F490005800002020202020202020202828282854
:10F4A0002820202020202020202020202020202054
:10F4B00020202088101010101010101010101010A4
:10F4C00010101004040404040404040404101010B4
:10F4D0001010101041414141414101010101010160
:10F4E00001010101010101010101010101011010EE
:10F4F0001010101042424242424202020202020234
:10F5000002020202020202020202020202021010BF
:10F5100010102000000000000000000000000000AB
:10F5200000000000000000000000000000000000DB
:10F5300000000000000000000000000000000000CB
:10F5400000000000000000000000000000000000BB
:10F5500000000000000000000000000000000000AB
:10F56000000000000000000000000000000000009B
:10F57000000000000000000000000000000000008B
:10F58000000000000000000000000000000000007B
:08F59000000000000000000073
:08F59800700BFF7F0100000071
:10F5A000FFFFFFFFE803000001000000E803DC05A7
:10F5B000DC05DC05DC050000FFFFFFFFFFFFFFFFB0
:10F5C0001800000019FCFFFFFFFFFFFF0200000012
:10F5D00040420F00FF01FF000024F4000200000081
:10F5E00003000000FFFFFFFF00000000010000001B
:10F5F0000000020001000000FFFFFFFF000000000C
:10F60000020000000000040002000000FFFFFFFFF6
:10F6100000000000030000000000080003000000DC
:10F620000A00000008000000010000009000002017
:10F63000000000004CF400006CF400002CF400000A
:10F6400000000000000000000000000000000000BA
:10F6500000000000000000000000000000000000AA
:10F66000000000000000000000000000000000009A
:10F67000000000000000000000000000000000008A
:10F68000000000000000000000000000000000007A
:10F690004300000000000000000000000000000027
:10F6A000000000000000000000000000000000005A
:10F6B0004300000000000000000000000000000007
:10F6C000000000000000000000000000000000003A
:10F6D00043000000000000000000000000000000E7
:10F6E000000000000000000000000000000000001A
:10F6F00043000000000000000000000000000000C7
:10F7000000000000000000000000000000000000F9
:10F7100043000000000000000000000000000000A6
:10F7200000000000000000000000000000000000D9
:10F730004300000000000000000000000000000086
:10F7400000000000000000000000000000000000B9
:10F750004300000000000000000000000000000066
:10F760000000000000000000000000000000000099
:10F7700091D80000A9D200000000000092F400001F
:10F78000ECDA000001E0000001E0000001E0000010
:10F7900001E0000001E0000001E0000001E00000E5
:10F7A00001E0000001E00000FFFFFFFFFFFFFFFF9F
:10F7B000FFFFFFFFFFFF00000100415343494900E5
:10F7C0000000000000000000000000000000000039
:10F7D00000000000000000000000415343494900C0
:10F7E0000000000000000000000000000000000019
:10F7F000000000000000000000000000E900000020
:10F80000557C0000A97F000001840000C1000000B9
:040000030000804534
:00000001FF
